:04000005000080C1B6
:020000040000FA
:10800000D02B00200983000015830000A59F0000ED
:108010000000000000000000000000006D2EFEDFE8
:108020008F9E939B0B999697FF000000B9810000EB
:10803000000000003C5501005D820000BD82000090
:108040002783000027830000278300002783000088
:108050002783000027830000278300004DA700002E
:108060001F83000023830000278300002783000074
:1080700027830000C5A70000278300002783000096
:108080002783000027830000278300002783000048
:108090002783000027830000278300002783000038
:1080A00031B20000278300002783000027830000EF
:1080B000278300002783000027830000F9A8000021
:1080C00000F002F800F030F80CA030C8083824188E
:1080D0002D18A246671EAB4654465D46AC4201D100
:1080E00000F022F87E460F3E0FCCB6460126334202
:1080F00000D0FB1AA246AB463343184748EC0000B9
:1081000068EC00000023002400250026103A01D36B
:1081100078C1FBD8520700D330C100D50B6070473F
:108120001FB51FBD10B510BD00F04EFB1146FFF787
:10813000F7FF08F0BFF900F066FB03B4FFF7F2FFAA
:1081400003BC00F069FB000080F309887047EFF37F
:1081500009807047684680F3098806480078C007A0
:1081600003D1032080F314887047022080F3148821
:1081700070470000B8600100064B9C46EFF3058392
:108180001B0605D1EFF31483DB0701D000DF704736
:108190006047000085170100064B9C46EFF30583FE
:1081A0001B0605D1EFF31483DB0701D000DF704716
:1081B0006047000099190100EFF309808169891E69
:1081C0000978002933D1A6461FC8A4467446E04763
:1081D0001F4B06CB914224D0083B002910D00CB491
:1081E000203101234B70EFF30983203B4B60F0C338
:1081F00044464D4656465F46F0C309F063FE0CBC4C
:108200001A60203253681033F0CBA046A946B2461C
:10821000BB4683F30988203BF0CB5078002803D07D
:108220001078EFF3098318600223DB43184710B579
:10823000084A1268914209D8074C89006458A6463A
:108240001FC8A446F047EFF309840FC410BD000017
:10825000DCEEFF1F7C8800007C88000009F018FD20
:10826000154B06CB914223D0083B0CB420310023A0
:108270004B70EFF30983203B4B60F0C344464D46FF
:1082800056465F46F0C309F01DFE0CBC1A60203252
:1082900053681033F0CBA046A946B246BB4683F3E1
:1082A0000988203BF0CB5078002801D01078186165
:1082B0000223DB4318470000DCEEFF1F09F0BAFE83
:1082C000CEE7000008F0A4FB09F0B4FEC8E7000008
:1082D00070B505460C46164602E00FCC0FC5103EA1
:1082E000102EFAD2082E02D303CC03C5083E042E6A
:1082F00007D301CC01C5361F03E021782970641C27
:108300006D1C761EF9D270BD72B60B48804762B6FE
:108310000A480047FEE7FEE7FEE7FEE7FEE70848FB
:108320000047084800470848004700000748084938
:10833000084A094B70470000A1B10000C18000004D
:1083400039A0000051A0000027830000D0290020A0
:10835000D02B0020D02A0020D02A002000487047CF
:1083600070290020034610B50B439B070FD1042A48
:108370000DD308C810C9121FA342F8D018BA21BAE9
:10838000884201D9012010BD0020C04310BD002A41
:1083900003D0D30703D0521C07E0002010BD0378A0
:1083A0000C78401C491C1B1B07D103780C78401C1F
:1083B000491C1B1B01D1921EF1D1184610BD421E53
:1083C0005378521C002BFBD10B78491C1370521CA4
:1083D000002BF9D17047D2B210B513029A181304CA
:1083E0009A1800F020F910BD020A08704A70020CB9
:1083F0008A70020ECA7070477047704770477047A6
:108400004D4943524F424954F0FFFFFFBE39FFFF31
:1084100030B5441C03E00178401C00290DD08107D1
:10842000F9D10B4BDD0104C8D11A91432940FAD090
:10843000001B0A0603D0C01E30BD001B30BD0A045D
:1084400001D0801E30BD0902FCD0401E30BD0000AE
:10845000010101010346F0B50B439B072DD1244DCB
:10846000EF01042A29D308C810C95E1B9E43121FBE
:108470003E4017D0D8B2E1B2401A3106014310D1C4
:1084800098B2A1B2401A310401430AD11802210264
:10849000000A090A401A3102014302D1180E210EC6
:1084A000401AF0BDA342DCD018BA21BA884201D9E3
:1084B0000120F0BD0020C043F0BD002A01D1002002
:1084C000F0BD03780C78401C491C002B0DD0A34252
:1084D0000BD1521E09D003780C78401C491C002B8C
:1084E00003D0A34201D1521EEBD1181BF0BD0000F6
:1084F00001010101F8B5042A2CD3830712D00B78AF
:10850000491C0370401C521E83070BD00B78491C7A
:108510000370401C521E830704D00B78491C037063
:10852000401C521E8B079B0F05D0C91ADF00202369
:10853000DE1B08C90AE0FFF7CBFEF8BD1D4608C9DF
:10854000FD401C46B4402C4310C0121F042AF5D233
:10855000F308C91A521EF0D40B78491C0370401C52
:10856000521EEAD40B78491C0370401C012AE4D443
:1085700009780170F8BD431A70B593421BD289186F
:10858000801804E0491E401E0B78521E03709307AA
:10859000F8D106E01039103878C9103978C0103891
:1085A000103A102AF6D203E0091F001F0B6803607F
:1085B000121FF9D570BDFFF78BFE70BDF8B50646EA
:1085C00014460843800707D0751AA54219D2081926
:1085D000102D13D2311907E03046FFF7CCFFF8BD5C
:1085E000401E491E02780A70641EF9D2F8BD471B6E
:1085F0002A463946FFF77EFF641B3846A542F6D36C
:10860000011B22463046FFF775FFF8BD01E004C0AC
:10861000091F0429FBD28B0701D50280801CC907E2
:1086200000D00270704700290BD0C30702D002703F
:10863000401C491E022904D3830702D50280801CF6
:10864000891EE3E70022EEE70022DFE70378C27825
:108650001946437812061B0219438378C0781B041D
:10866000194311430902090A000608437047002212
:1086700003098B422CD3030A8B4211D300239C465F
:108680004EE003460B433CD4002243088B4231D3D7
:1086900003098B421CD3030A8B4201D394463FE06B
:1086A000C3098B4201D3CB01C01A524183098B42CB
:1086B00001D38B01C01A524143098B4201D34B01B4
:1086C000C01A524103098B4201D30B01C01A524117
:1086D000C3088B4201D3CB00C01A524183088B429E
:1086E00001D38B00C01A524143088B4201D34B0087
:1086F000C01A5241411A00D20146524110467047F9
:108700005DE0CA0F00D04942031000D340425340FD
:1087100000229C4603098B422DD3030A8B4212D3BD
:10872000FC22890112BA030A8B420CD389019211EF
:108730008B4208D3890192118B4204D389013AD02C
:10874000921100E08909C3098B4201D3CB01C01A01
:10875000524183098B4201D38B01C01A5241430914
:108760008B4201D34B01C01A524103098B4201D302
:108770000B01C01A5241C3088B4201D3CB00C01A6F
:10878000524183088B4201D38B00C01A5241D9D287
:1087900043088B4201D34B00C01A5241411A00D208
:1087A0000146634652415B10104601D34042002B04
:1087B00000D54942704763465B1000D3404201B583
:1087C0000020C046C04602BD7546FFF7C7FDAE4655
:1087D000050069465346C008C000854618B020B55C
:1087E000FFF7A4FD60BC00274908B6460026C0C5B7
:1087F000C0C5C0C5C0C5C0C5C0C5C0C5C0C5403D59
:1088000049008D46704710B50446C046C046204614
:10881000FFF793FC10BD000001491820ABBEFEE736
:108820002600020070B58C180578401C6B075B0FA2
:1088300001D10378401C2A1106D10278401C03E0C4
:108840000678401C0E70491C5B1EF9D12B0705D41D
:108850000023521E0DD40B70491CFAE70378401C0C
:10886000CB1A921C03E01D780D70491C5B1C521E34
:10887000F9D5A142D8D3002070BD0000000000004F
:10888000F8B504460026006A354640064027002811
:1088900003DA206A0126B8432062606AC0210843D7
:1088A000606206E0204600F099F8400601D50125F7
:1088B00005E00021204600F037F80006F2D52069D7
:1088C0000090002E02D0206A38432062204600F03B
:1088D00085F8400601D5012501E0002D01D028468C
:1088E000F8BDE06CA16C4018616C226C89184018CE
:1088F000E16B4018A16B401841080120C0030143FF
:108900000091E162E16EA26E8918626E236ED21848
:108910008918E26D8918A26D8918490801430091F0
:1089200021630020F8BD000070B50C460546022901
:1089300001D2012000E00020FF226A3204A105F0EC
:108940009BF90020A1006958090600D5802070BD60
:108950002E5C736F757263655C6869635F68616CD8
:108960005C667265657363616C655C6B6C32377AEB
:108970005C66736C5F61646331362E6300000000D7
:1089800010B509490024A2008A58824201D0641C13
:10899000F9D0002C06D00020462204A105F06CF985
:1089A000204610BD0120F7E7C05D01002E5C736F0B
:1089B000757263655C6869635F68616C5C6672654B
:1089C000657363616C655C6B6C32377A5C66736C83
:1089D0005F61646331362E630000000001460A6A5D
:1089E0000020120600D58020496A490601D54021A1
:1089F0000843704770B50C00054601D0012000E027
:108A000000204D2225A105F037F92846FFF7B8FFD1
:108A10002E49800009582E4A080C8018026801234C
:108A20008B401A4302606078217980078907800FA4
:108A3000090F08436179042901D010210843E17826
:108A40008907490E0143E079002801D080200143C5
:108A5000A960E868617900090001042902D089074A
:108A6000890F0843A179002901D004210843A27885
:108A70000821002A00D00843E860286A227880088C
:108A800080009207920F02432A62207A0028686AC7
:108A900001D0084300E08843686270BD2E5C736FAC
:108AA000757263655C6869635F68616C5C6672655A
:108AB000657363616C655C6B6C32377A5C66736C92
:108AC0005F61646331362E6300000000C45D010005
:108AD0000070044070B514460D460646022901D2C6
:108AE000012000E00020FF2254320EA105F0C4F85E
:108AF000002C01D0012000E00020FF22553209A106
:108B000005F0BAF82078C3066079DB0E002801D0A2
:108B1000202003432079002801D040200343A800EF
:108B2000335070BD2E5C736F757263655C686963EA
:108B30005F68616C5C667265657363616C655C6BD4
:108B40006C32377A5C66736C5F61646331362E63B6
:108B50000000000010220029C16802D01143C1604A
:108B600070479143FBE7426AD208D200042903D040
:108B70008907890F091D0A4342627047044A010CA4
:108B800089180A68012383409A430A6070470000ED
:108B900000700440044A010C89180A6801238340CC
:108BA0001A430A60704700000070044010B5114875
:108BB0000068800C8007800F05D002280CD00328A5
:108BC00015D0002010BD00F091F80121C9038842A2
:108BD00000D00021084610BD074C6068002800D076
:108BE0000120912205A105F047F8606810BD7D20A5
:108BF000C00010BD00700440C4ECFF1F2E5C736FFA
:108C0000757263655C6869635F68616C5C667265F8
:108C1000657363616C655C6B6C32377A5C4D4B4C91
:108C200032375A345C66736C5F636C6F636B2E63B0
:108C30000000000010B5194C030004F06BFF140B8A
:108C40000B102D102D2D1E212D2D2D242D2D2D2DD4
:108C500027272A2D00F07CF86168090F09E000F051
:108C600077F86168090F491CFFF701FD6168490346
:108C7000490F491CFFF7FBFC10BDFFF797FF10BD24
:108C800000F034F810BD00F00BF810BD00F0A4F8AF
:108C900010BD7D20C00010BD002010BD40800440EC
:108CA00070B50648017A007E09074C0F45076D0F25
:108CB00000F006F86119C84070BD00000040064091
:108CC00008480178890706D481790907890F0129A5
:108CD00001D00020704740780349C007400F085872
:108CE0007047000000400640B85D010010B508481C
:108CF000007800060AD5074C2068002800D0012023
:108D0000782205A104F0B8FF206810BD002010BD36
:108D100000500640C4ECFF1F2E5C736F75726365D4
:108D20005C6869635F68616C5C66726565736361EA
:108D30006C655C6B6C32377A5C4D4B4C32375A3415
:108D40005C66736C5F636C6F636B2E630000000086
:108D500010B5104CA07980088007800F05D001283D
:108D600005D002280AD0002010BD0B4810BDFFF727
:108D7000A7FF217A0907490FC84010BD074C20689A
:108D8000002800D00120FF226B3205A104F074FFFF
:108D9000206810BD00400640006CDC02C4ECFF1FE0
:108DA0002E5C736F757263655C6869635F68616C84
:108DB0005C667265657363616C655C6B6C32377A97
:108DC0005C4D4B4C32375A345C66736C5F636C6F2E
:108DD000636B2E63000000000548017E090605D480
:108DE00080790007800F01D000207047014870474C
:108DF00000400640006CDC02F8B502787F2A02D001
:108E000000F04EF8F8BD0A704478861C4C708D1C3A
:108E1000074F08E02946304600F042F8010C3F18A1
:108E20008E1980B24519641EF4D23846F8BD000090
:108E3000020002000A4670B50146002003460629DA
:108E400016D006DC0B0004F065FE0513131314188E
:108E50001300FD290CD003DCF02909D111201CE0FE
:108E6000FE2919D0FF2903D1402010705370022031
:108E700070BD154607F0BEF902E0154607F0C2F9CD
:108E80000646FFF7C5FA401CC4B2224631462846C2
:108E9000FFF730FB204670BD05201070012070BD2B
:108EA000F8B502781346803B1F2B02D800F032F948
:108EB000F8BD1346A03B5E2B02D800F0C5F9F8BD03
:108EC0000A7007784C1C421C0025FF218848894EF7
:108ED0003B0004F01FFE1E10182140A9B6D3F1F28A
:108EE0005264F1F1F1F1F1686D728190A63DF1F1FA
:108EF000F1F1F1F18BF11078611CFFF79BFF7E49D6
:108F000020704018F8BD1078002846D0012844D0C1
:108F100021707948401ED5E01178002903D001293D
:108F200002D0002114E00121012202707348402385
:108F3000436020254560724A4703576047691F43D5
:108F4000476143692B4343615069EB031843506108
:108F500021703046B6E0057068484169402291436F
:108F60004161426920218A43426165484269C903DF
:108F70008A43426125700120A4E0507811780702ED
:108F800061480F435F490068FFF771FB0321801CB4
:108F9000FFF76DFB7843401EFDD12570B9E7657082
:108FA000257002208EE02146104600F0F1FB89E09A
:108FB0002146104600F0B6FB84E01778511C002FC4
:108FC00001D1FF270137384602F0C4F8FF1D257094
:108FD000F8080004801975E011788A07920F521C76
:108FE00049070276C90F41762570B2E7214610463F
:108FF00000F030F966E02170012113780C46521C14
:109000000AE01078521C8006800E00D14020C01D5E
:10901000C00812180918491C5B1EF2D2080420432C
:1090200050E010782170D4E7117801739378577865
:109030001902394301821179D27809021143418220
:1090400050E000782146012814D01346521C1078B5
:10905000521C002808D01778521CBC0701D5FC060A
:1090600000D5121D401EF6D1D01A0D7000044D70AF
:10907000801C27E0104600F031F923E00078174605
:10908000214601280AD00D704D70A5700320F97893
:109090001E4A890706D5104301460AE0104600F033
:1090A000AFFAF4E7B9787B78090219438904891883
:1090B0000143084606E000E016E00078012803D0EE
:1090C000217013488019F8BD1746501CFFF7BEFAEF
:1090D00039790002000A0906084300906946002019
:1090E00001F052FD2570ECE7203CE1773046F8BDF9
:1090F00034F8FF1F0100010002000200800000F8A8
:1091000000F00F4040420F00CCECFF1F00000400B5
:1091100001000500FEB502780A704D1C0178484C2C
:10912000401C8039064667000B0004F0F3FC0E0873
:10913000152137447D7D7D4E5C686C707F7D07F026
:1091400059F80746FFF764F9C6B22E70681C32461C
:109150003946FFF7CFF92BE00724684602F0A4FA5E
:10916000224669462846FFF7C5F9354C08345BE0CE
:10917000684602F099FA002002900422314602A8C3
:10918000FFF7B8F902980090684602F0ADFA0020A7
:1091900002F02AFB012028702A4C45E03E21681C81
:1091A0000AF028FD060002D0012007F097F92E7082
:1091B000A419641C38E03778701C39460AF09AFD0F
:1091C000012007F08BF901202AE001202870307877
:1091D000002805D0012803D0002028703C4623E059
:1091E00007F01AFBFAE70120287005F099F800282B
:1091F00002D102200AF0BAFA114C641C14E0007883
:1092000009F0B6F9E9E709F083F92870F4E737784F
:10921000461C012007F072F93946304609F042FA3F
:1092200028703904081904192046FEBD0020287052
:109230003078002800D0012006F0A2F9CEE7000027
:109240000100010002000500FF200870004870477F
:1092500001000100F3B583B000220A70491C01250A
:10926000009504910178441C01912AE02778641C40
:10927000B806800E00D14020C01DC608380616482A
:10928000416902D52022914301E02022114341612E
:1092900021463846049A01F02BFC0198002804D19D
:1092A0000D484169202211434161380606D50498D2
:1092B0008019049000988019009001E0A419AD195C
:1092C0006D1C0198401E0190401CCFD100992804CC
:1092D000084305B0F0BD0000800000F8F0B589B08B
:1092E0000890044600208D1C0391C3490290087029
:1092F000049005906678A41C002E6FD02778641C1B
:10930000B9076CD50499002935D0BC48008A019072
:109310001120384001280FD16946384601F034FC4D
:1093200002281AD10199491E0191491C03D0B24962
:1093300009780029F0D012E169460E2001F024FCE2
:10934000022808D10199491E0191491C03D0AA495C
:1093500009780029F0D0002104910128EBD100996F
:1093600029700099090A69700099090CA97000997F
:10937000090EE9702D1DF90658D52046FFF766F94C
:10938000E1780002000A0906084307909B48241D63
:10939000408A0690F80715D09848008A019000216D
:1093A000384601F0F1FB022802D00128C3D109E0C0
:1093B0000199491E0191491CBDD08F4909780029A6
:1093C000EDD0CCE08D48008A01906946384601F026
:1093D000DBFB022804D001281CD10BE0E0E064E0B4
:1093E0000199491E0191491C14D08349097800292B
:1093F000EBD00FE08149009A49691140079A9142E8
:1094000008D00699491E0691491C03D07A4909786B
:109410000029D7D07949009A49691140079A9142A9
:1094200001D01021084301281AD13CE07349098A70
:109430000191F90718D00499002934D10021384648
:1094400001F0A2FB022802D0012809D109E001990C
:10945000491E0191491C03D0674909780029EDD0C4
:109460007DE0012104911EE06946384601F08CFB45
:10947000022802D0012872D109E00199491E019108
:10948000491C6CD05C4909780029EDD067E000994F
:1094900029700099090A69700099090CA97000994E
:1094A000090EE9702D1D00214DE00498002823D0FD
:1094B0005248008A019069460E2001F065FB02289F
:1094C00002D001284BD109E00199491E0191491CA4
:1094D00045D0494909780029EDD040E0009828702E
:1094E0000098000A68700098000CA8700098000EA0
:1094F000E87000202D1D04902046FFF7A7F8E178C2
:109500000002000A09060843241D0090B90603D58D
:109510003A494861012017E03848008A01906946BD
:10952000384601F031FB022802D0012817D109E0AA
:109530000199491E0191491C11D02F490978002930
:10954000EDD00CE0012105910299491C02912A49B4
:109550000978002903D1761E00D0CFE60AE0002E5C
:1095600008D02178641C8A0701D5C90600D5241DBE
:10957000761EF4E7012832D1049900291ED01F4835
:109580001D4F068A69460E2001F0FEFA022802D01D
:10959000012824D105E0761E21D339780029F1D0A5
:1095A0001DE0009929700099090A69700099090C59
:1095B000A9700099090EE9702D1D10E00599002988
:1095C0000DD00E480C4F068A00210E2001F0DCFA67
:1095D000022804D1761E02D339780029F4D0039AE8
:1095E000029911700399487008980399201A000491
:1095F000691A084309B0F0BD2FE8FF1F34F8FF1FB8
:10960000F3B583B00025CE1C02914449024628469A
:109610000D70917853780C02D21C1C4373D01178D2
:10962000521C0091039289075DD50099C90737D074
:109630003B48078A0021009801F0A6FA022802D0D0
:10964000012860D12CE07F1E5DD3344909780029C0
:10965000F0D058E0002C04D10098C00701D00E20B3
:1096600000902F48078A01A9009801F08DFA02287E
:1096700002D0012847D106E07F1E44D3274909784C
:109680000029F0D03FE00199317001996D1C090A61
:1096900071700199090CB1700199090EF170361DB4
:1096A000641ED7D22FE00398FEF7D0FF0399000283
:1096B000C978000A0906084301900398001D039029
:1096C0001748078A01A9009801F05EFA022802D023
:1096D000012818D106E07F1E15D31049097800290A
:1096E000F0D010E06D1C641EDDD20D480B4F048AD3
:1096F00000210E2001F048FA022804D1641E02D392
:1097000039780029F4D002990D70029A290A517013
:1097100002998870029805B0301AF0BD2FE8FF1F3B
:1097200034F8FF1FF8B50D460646FEF78FFF04021A
:10973000F078240A000604430CD012480621006881
:109740000090FEF794FF00270F4EA04205D801209D
:10975000707012E0FF20287011E0777000982146A9
:1097600040080019401EFEF782FF012804D903219A
:10977000401CFEF77CFF00E0012070602F70034862
:10978000F8BD0000CCECFF1F34F8FF1F01000400FF
:10979000F3B506460578447881B0801CFEF756FF85
:1097A00001027079090A000601432A48E20706D03F
:1097B000EB074022002B01D0426000E08260A2074C
:1097C00006D5AB072022002B01DA426000E0826060
:1097D000214A230606D5EB09DE07204B01D0536052
:1097E00000E09360002923D001260023E10704D084
:1097F00001694906C90FA94217D1A10705D5016919
:109800006F088906C90FB9420FD1610701D5A908B0
:109810000BD1A10601D5690907D1210608D5116927
:10982000EF09C902C90FB94202D05942B142DDD392
:10983000016900694906C90F8006C00F4000014355
:109840001069C002C00FC0010143029801700448B2
:10985000FEBD0000800000F800F00F400000100086
:109860000100060010B5224C0020207020736421F6
:10987000218260820122606122761E496076096839
:109880001D4B4908994202D8627062600FE0607017
:109890001A4808181949491CFEF7E9FE012804D99D
:1098A0000321401CFEF7E3FE00E001206060144944
:1098B000886B1F22520210438863FF20114A033035
:1098C0009061114840234360416919434161FF2180
:1098D00004315161202242604369934343610B4844
:1098E00001610B48D103416042690A43426110BDE6
:1098F00034F8FF1FCCECFF1F02366E01FF117A0017
:109900000080044000B00440800000F84090044013
:1099100000F00F40F8B5C41D0546F934E06C1E4652
:109920000F46002823D0402A00DD4022401EE0647C
:10993000606D80014019FEF7DDFD606D8001411909
:109940003846FFF759FA616D49004919FF31413135
:109950000880606D0521800140193060606D401CF9
:10996000FEF785FE6165206D401C20650120F8BD75
:1099700010B5C41DF934236D002B17D05B1E236571
:10998000A36D9B011B180B60A16D49000818FF30E7
:10999000413000881060A06D0521401CFEF767FE75
:1099A000A165E06C401CE064012010BD002010BDEA
:1099B000FF30002201304265826505210265C164E5
:1099C00070470000002805DBC106C90E0120884051
:1099D000014908607047000000E100E070B50546ED
:1099E000EFF31080C407E40F72B6094E094B294605
:1099F0003046F26800F010F8002805D1002329460F
:109A00003046F26800F030F9002C00D162B670BD2B
:109A1000181100206B66656BFFB589B016460C46C1
:109A20006A46099805F088FC32462146049B09984D
:109A300005F06BF905002BD1009C019FA619761E3D
:109A400039463046FEF713FE00291BD0401C7843F0
:109A5000461E17E021020920090A000609180D48D0
:109A600041600C9805F06AF9002811D1099805F0B9
:109A70006FF9054609980069002800D08047002D3D
:109A800002D1E419B442E5D9099805F011F9284644
:109A90000DB0F0BD0000024070B5040027D016489C
:109AA000C0680001000F0F2823D014494000085A55
:109AB00080020025256060600220A0606561A561CC
:109AC00040022561E060204605F011F900280AD027
:109AD0000B48014680390560416040318160E0619A
:109AE000204600F00FF825620020656270BD04205A
:109AF00070BD01208004DCE740800440985D0100D7
:109B0000CC110020F8B500280FD0C56922484024A8
:109B1000460822487600400840006F68B0420ED9DF
:109B2000841B402C03D8012002E00420F8BD002053
:109B30001B4A1CA104F0A0F8402C00D94024224666
:109B400031463846FEF7D6FC21487F1C0760214885
:109B5000402446082048760040084000AF68B042E4
:109B60000DD9841B402C01D8012000E000200C4AB4
:109B70000CA18E3204F080F8402C00D940242246FB
:109B800031463846FEF7B6FC11487F1C476002207C
:109B900028600020F8BD000041F600004DF60000EE
:109BA0008E0700002E5C736F757263655C68696375
:109BB0005F68616C5C667265657363616C655C6946
:109BC00061705C66736C5F666C6173682E63000025
:109BD000BCECFF1FD9EC0000EDEC0000FFB589B034
:109BE0001F4614000D460DD06A46099805F0A4FBE7
:109BF0003A462946039B099805F087F8060002D1EA
:109C0000009D28E004200DB0F0BD02CC1548816015
:109C10000399042902D0082907D00EE02902032263
:109C2000090A52068918416007E002CCC160290286
:109C30000722090A120689184160099805F088F878
:109C4000064609980069002800D08047002E04D1FC
:109C5000039845193F1A002FD7D1099805F028F825
:109C60003046D0E700000240FFB589B014460D46EB
:109C70006A46099805F060FB22462946059B09982B
:109C800005F043F800282FD16A462946099805F0C7
:109C900053FB009D029808906942404201404F42A8
:109CA000AF4201D108983F18002C1CD07E1BA64261
:109CB00000D9264630460599FEF7D9FC2902012233
:109CC000090A12068A1809494A600C9A000412020D
:109CD0001043FF308860099805F03AF8002803D156
:109CE000A41BAD19DEE700200DB0F0BD000002405E
:109CF000FFB589B0129F1D0016460C4610D06A466B
:109D0000099805F019FB32462146079B099804F093
:109D1000FCFF002805D1154A39068F18009C22E067
:109D200004200DB0F0BD21020120090A40060918E7
:109D30000F48416087602968C160099805F008F8FC
:109D4000002809D01399002900D00C60149900292B
:109D5000E7D000220A60E4E70799761A89088900AB
:109D60004D1907990C19002EDDD1DAE7FFFFFF002E
:109D70000000024010B5040001D0012000E00020E6
:109D80008B2207A103F078FF04212046FEF75AFC3E
:109D90000121217000206070A170E07010BD0000F2
:109DA0002E5C736F757263655C6869635F68616C74
:109DB0005C667265657363616C655C6B6C32377A87
:109DC0005C66736C5F666C6578696F2E630000007B
:109DD00010B509490024A2008A58824201D0641CAF
:109DE000F9D0002C06D00020412204A103F044FF4A
:109DF000204610BD0120F7E7C85D01002E5C736F9F
:109E0000757263655C6869635F68616C5C667265E6
:109E1000657363616C655C6B6C32377A5C66736C1E
:109E20005F666C6578696F2E6300000070B50C4644
:109E30000546FFF7CDFF124980000858114A010C72
:109E400089180A68012383401A430A60284600F0F3
:109E50001DF8A8680C490840A178C9074A08E178AC
:109E6000C907490F0A432178C907C90F0A430243AA
:109E70006078002802D10120C0070243AA6070BDAB
:109E8000CC5D010000700440FAFFFF3F81680222B0
:109E90001143816000218160704710B5937BD47BB2
:109EA0009B07A4079B09A40A2343147C8900640729
:109EB000640B2343547C08186407640C2343947C8C
:109EC00009216407640D2343D47CC901A407A40EAF
:109ED0002343147DE407A40F234341180B60118B27
:109EE00005231B0289B2C318196011781379090779
:109EF000DB0709091B0A19435379DB075B0A19437E
:109F000093799B079B0B1943137A5B075B0D1943EE
:109F1000137B527BDB071B0E92071943920F1143F1
:109F2000012292028018016010BD000070B515007A
:109F30000E46044601D0012000E0002064220AA160
:109F400003F09AFE29780120B040002907D06978F3
:109F5000002907D0606061690143616170BD61697A
:109F60008143FAE7A060F6E72E5C736F7572636554
:109F70005C6869635F68616C5C6672656573636188
:109F80006C655C6B6C32377A5C66736C5F677069AA
:109F90006F2E630001238B40002A01D0436070477D
:109FA00083607047EFF3088470460007000F0D28A8
:109FB00001D1EFF309842546A08B2035800500D51B
:109FC0002D1D7046C00600D44835704604F020FAB6
:109FD000EFF3098004F01CFAEFF3088004F018FA9C
:109FE000EFF3148004F014FA284604F011FA6069C3
:109FF00004F00EFAA06904F00BFAE06904F008FA24
:10A000004A2203A1002003F037FE01F003F9FEE726
:10A010002E5C736F757263655C6461706C696E6BE6
:10A020005C486172644661756C745F48616E646C13
:10A0300065722E630000000010B5034801680348F4
:10A0400000F012FB10BD0000D8ECFF1F00600640BE
:10A0500010B503484168034800F006FB10BD00003E
:10A06000D8ECFF1F007006404A0603D58278BF2354
:10A070001A408270890603D581798F22114081713F
:10A0800070470029817802D08022114301E04906FF
:10A09000490E817070474A0603D5827840231A43DF
:10A0A0008270890605D58179AF22114020221143A3
:10A0B0008171704710B50A490024A2008A58824273
:10A0C00002D0641C022CF8D3022C01D2012000E043
:10A0D0000020AF2203A103F0CFFD204610BD0000F9
:10A0E000DC5D01002E5C736F757263655C6869638B
:10A0F0005F68616C5C667265657363616C655C6BFF
:10A100006C32377A5C66736C5F6932635F6D6F6463
:10A110002E6300000A04CB04120E002B02DA8379AE
:10A12000134383714B0402D5837913438371C17048
:10A1300070470146C0788A79520602D501229203FF
:10A1400010438979C90602D50121090308437047E4
:10A15000F7B586B00020009001900F460120002640
:10A160007D210490F6430025C9001046FEF77FFAD2
:10A17000039004981649A8400024484302901548CB
:10A180006200805A029A03995043FEF770FA8742A0
:10A1900001D9381A00E0C01BB04203D200950194E7
:10A1A000060003D0641CE4B2402CE8D36D1CEDB271
:10A1B000022D01D8002EDCD1009801998007000EF5
:10A1C0008906890E08430699487009B0F0BD000061
:10A1D00020A10700E45D010010B504460021FFF74F
:10A1E00050FF2046FFF766FF024980000858FEF73F
:10A1F000C5FC10BDD45D010010B5040001D00120E4
:10A2000000E00020084A09A103F036FD002020608C
:10A210006060A06020726070A070E0707D204001DE
:10A22000E0600120207010BD030700002E5C736FFA
:10A23000757263655C6869635F68616C5C667265B2
:10A24000657363616C655C6B6C32377A5C66736CEA
:10A250005F6932635F6D6F642E63000070B51646F0
:10A260000D00044601D0012000E00020294A2AA167
:10A2700003F002FD2046FFF71DFF33498000085818
:10A28000FEF788FC002020706070A070FF21E17054
:10A2900060715021A171E071287A002802D0022853
:10A2A0001AD103E028794000207015E0A888E988D9
:10A2B000884201D2012000E00020164A16A11D327A
:10A2C00003F0DAFC287940002070A8794000E071A2
:10A2D0006079082108436071A078FD210840A978C1
:10A2E000C907890F01432878C007000E0143A170F8
:10A2F00060796F210840E9786A78C907C90ED207EA
:10A30000120E11430143617132462046E968FFF79E
:10A310001FFF70BDA90600002E5C736F7572636528
:10A320005C6869635F68616C5C66726565736361D4
:10A330006C655C6B6C32377A5C66736C5F69326338
:10A340005F6D6F642E630000D45D0100F8B51D469B
:10A3500016460C00074601D0012000E000200C4A00
:10A360000CA103F089FC3846FFF7A4FE0746242120
:10A370002046FEF769F91349E661B80025620C50E2
:10A380001148083948601148C057FFF71BFBF8BD5A
:10A39000C70700002E5C736F757263655C68696344
:10A3A0005F68616C5C667265657363616C655C6B4C
:10A3B0006C32377A5C66736C5F6932635F6D6F64B1
:10A3C0002E630000D8ECFF1FD1A30000D05D010078
:10A3D000FEB50C00064601D0012000E00020714AC5
:10A3E00071A103F049FC00206946019008700878CB
:10A3F000401C08703046FFF79CFE87B2251D78048C
:10A400001AD5012189033046FFF784FE0220F0703F
:10A41000207801280ED1202028700021E9602170C9
:10A42000A169014206D0E369002B03D029463046DA
:10A43000226A9847780634D5F80414D50121090317
:10A440003046FFF767FE0220F07010202870A169E7
:10A45000014206D0E369002B03D029463046226A28
:10A46000984778061DD50220F070F8071AD0B0780A
:10A47000E7210840B070307969460870E06800282C
:10A480000FD0202129705448E86000202070A06976
:10A49000084206D0E369002B03D029463046226AE1
:10A4A0009847FEBD780634D50120207028707807C3
:10A4B00009D5B17810200143B170012001903079A5
:10A4C000694608700BE0B078E7210840B070307939
:10A4D000694608700878002801D140202870297842
:10A4E000A06908420BD0E069002808D068460078CF
:10A4F000216A0870E36929463046226A9847019824
:10A500000028CED0A868696800292BD0002829D05F
:10A5100033E0380622D57807F4D4A86869680029A2
:10A5200001D000280AD104202870E369002B03D051
:10A5300029463046226A9847002028613179E06830
:10A540000028AED0A068421CA2600170E068401EE6
:10A55000E0602869401C2861E068FEBD30796946EA
:10A560000870FEBD02202870E369002B03D0294645
:10A570003046226A984700202861E06800280BD006
:10A58000A068411CA16000783071E068401EE06066
:10A590002869401C2861FEBDB078E7210840B070F2
:10A5A000DCE70000560800002E5C736F757263656F
:10A5B0005C6869635F68616C5C6672656573636142
:10A5C0006C655C6B6C32377A5C66736C5F693263A6
:10A5D0005F6D6F642E6300004E04000070B5154679
:10A5E0000C00064601D0012000E000200F4A10A117
:10A5F00003F042FB2078012816D060213046FFF797
:10A6000033FD1421201DFEF71FF801202070462085
:10A61000054330461249A561FFF77CFD60213046B5
:10A62000FFF739FD002070BD0E4870BDF607000031
:10A630002E5C736F757263655C6869635F68616CDB
:10A640005C667265657363616C655C6B6C32377AEE
:10A650005C66736C5F6932635F6D6F642E630000CC
:10A66000125000004C04000010B5C37882789406A4
:10A67000054A01D4DB0601D5126800E05268904714
:10A68000BFF34F8F10BD0000D0ECFF1F10B5EFF3EC
:10A690001080C007C00F72B60021064A1160002862
:10A6A00000D162B60448FFF7F7F9002800D0012076
:10A6B00010BD000000810440181100201CB508F0F6
:10A6C00085FA00281AD09E2069460870E720487055
:10A6D000102000F03FFD012408F078FA00280DD08A
:10A6E000002069460870082000F034FD01A9002010
:10A6F00008F002FA012802D1002C00D01CBD002075
:10A700001CBDCA080AD0012A07D1801D002804D028
:10A710004A07520F0121914001707047401DF5E733
:10A72000CA0802D0012A0ED101E0401D00E0801DC0
:10A73000002808D000784A07520F012191400840B4
:10A7400000D00120704700207047000070B50D4D0B
:10A750000E212846FFF7E4FF0124002805D00E2132
:10A760002846FFF7CEFF0848047008212846FFF767
:10A77000D7FF002805D008212846FFF7C2FF03486D
:10A78000047070BD00C0074018E0FF1F19E0FF1FF4
:10A7900010B58B0806D0012B10D0022B10D0032B44
:10A7A0000BD1C01C002808D003788907490F032467
:10A7B0008C40A3438A401A43027010BD401CF1E74D
:10A7C000801CEFE7F8B5354D6C68A868800202D4AC
:10A7D000012040058443A868314E000200D4B443F0
:10A7E000304F200313D5686801213840C904401850
:10A7F000686003F0ADFD002809D02B4803F088FC09
:10A80000132804D3132229A1274803F038FD20027E
:10A8100018D52B4803F08DFC002800D00120FE2223
:10A8200028A103F029FA264803F0A4FCE860244894
:10A8300003F07FFC002805D1A868B043A8600D2074
:10A8400003F076F9A0020BD56003800FE86808D00A
:10A8500069460870686803213840490440186860F8
:10A86000F8BDC5B2104803F053FC0446132804D9C0
:10A8700029460D4803F0B6FCF8BD03F069FD002839
:10A8800007D0132CF8D1132208A1074803F0F7FCD6
:10A89000F8BD054803F06EFCEAE7000000500540F3
:10A8A000000080000000E03FE81300203C444150DD
:10A8B0004C696E6B3A4F766572666C6F773E0A0034
:10A8C000D81100202E5C736F757263655C686963D4
:10A8D0005F68616C5C667265657363616C655C6B17
:10A8E0006C32377A5C756172742E63000A7849782D
:10A8F00009010A438270704710B5144C1348803424
:10A90000216AC90605D50022042100F02DF8102087
:10A9100020620F49086AC0060ED51020086206F0B2
:10A92000F3FB0C4908700C480069C006C017401CB6
:10A9300003D00A490120087010BD02F0DDFF09F0C4
:10A94000B9FE0749002008700649F4E700C004403A
:10A9500080B0044028E0FF1F80F00F4019E0FF1F87
:10A960001AE0FF1F3CE9FF1F10B5890043580F2470
:10A9700024041207A343120B1343435010BD10B518
:10A9800089004358072424025207A343520D13435E
:10A99000435010BD10B589004358072424025207C4
:10A9A000A343520D1343435010BD10B589004358C3
:10A9B000072424025207A343520D1343435010BDF2
:10A9C00010B589004358072424025207A343520DAF
:10A9D0001343435010BD10B5890043580724240287
:10A9E0005207A343520D1343435010BDFEB5074613
:10A9F00016460D46EFF31080C407E40F72B60B46FF
:10AA000039460948FFF7EAF8002809D101210190E9
:10AA10000091029033462A4639460348FFF768F909
:10AA2000002C00D162B6FEBD18110020034800685A
:10AA300080F31088BFF36F8F70470000E0ECFF1FBA
:10AA4000EFF3108072B602490860BFF36F8F704752
:10AA5000E0ECFF1F10B504460878002806D14878BE
:10AA60000128A0781AD020221043A0706078042317
:10AA7000C008C00018436070A078C2080878D200EF
:10AA80001043A070084801691943016160780748C4
:10AA900080476078000704D5054810BDDF221040CC
:10AAA000E3E7002010BD000000ED00E0E5ECFF1F33
:10AAB0003C0F000010B5044640780221C008C000D9
:10AAC00008436070074801690422114301616078FE
:10AAD000054880476078000701D5044810BD002074
:10AAE00010BD000000ED00E0E5ECFF1F3C0F000092
:10AAF000F0B583069B0E00D14023224C0006402671
:10AB00001F4D646800281BDB37E00021082012E09D
:10AB1000AE601C4C646827467F1EFDD12F696E60B5
:10AB2000BF06FF0F641EFDD14C08F9012143401EF2
:10AB30005B1E002801D0002BEAD1C1401170521CCD
:10AB4000002BE2D1F0BD0A780827491C12E0D0079B
:10AB500002D02020686001E02020A860AE6020467E
:10AB6000401EFDD16E602046401EFDD152085B1E86
:10AB70007F1E02D0002BEAD1F0BD002BE3D1F0BD47
:10AB8000800000F834F8FF1F10B5054A5278002AFB
:10AB900002D000F007F810BD00F04EF910BD000023
:10ABA00034F8FF1FF0B5A24F20228C467A60402176
:10ABB000B96000BF00BF796000BF00BFC30701D00C
:10ABC0007A6000E0BA60B96000BF00BF796000BF82
:10ABD00000BF4308DD0701D07A6000E0BA60B960C9
:10ABE00000BF00BF796000BF00BFC4188308DD0745
:10ABF00001D07A6000E0BA60B96000BF00BF796040
:10AC000000BF00BFE418C308DD0701D07A6000E090
:10AC1000BA60B96000BF00BF796000BF00BFE31831
:10AC2000DB0701D07A6000E0BA60B96000BF00BF06
:10AC3000796000BF00BFBA60B96000BF00BF796033
:10AC400000BF00BF7A60B96000BF00BF796000BF7D
:10AC500000BF7B69202293437B61764A127E131EDC
:10AC600007D0B96000BF00BF796000BF00BF521EAF
:10AC7000F7D1B96000BF00BF3A6979609206D20F80
:10AC800000BF00BFB96000BF00BF3C697960A40687
:10AC9000E40F00BF00BF64001443B96000BF00BFF1
:10ACA0003A6979609206D20F00BF00BF920022433A
:10ACB000012A14D0022A70D0042A6ED0213307D082
:10ACC000B96000BF00BF796000BF00BF5B1EF7D155
:10ACD000796920200143796178601046F0BD8407CE
:10ACE00033D5002425462023B96000BF00BF3E694C
:10ACF0007960B606F60F00BF00BFAD196408F6070D
:10AD000034435B1EF0D1B96000BF00BF3B6979607E
:10AD10009B06DB0F00BF00BF5D40EB0700D00822A1
:10AD20006346002B00D01C60424B1B7E002B07D0DB
:10AD3000B96000BF00BF796000BF00BF5B1EF7D1E4
:10AD40007B69202423437B6130E0002B07D0B9606E
:10AD500000BF00BF796000BF00BF5B1EF5E77B69E5
:10AD6000202633437B6163461B6800253446DE079B
:10AD700002D020267E6001E02026BE60B96000BFC0
:10AD800000BF796000BF00BFED185B08641EEED104
:10AD9000EB0703D020237B6002E01CE02023BB6094
:10ADA000B96000BF00BF796000BF00BF000602D5D8
:10ADB0002048002383601F48007B002809D02023FF
:10ADC000BB60B96000BF00BF796000BF00BF401E1C
:10ADD000F7D1202080E7174C657E002D0AD084072C
:10ADE00008D52124B96000BF00BF796000BF00BF53
:10ADF000641EF7D1002B07D0B96000BF00BF796097
:10AE000000BF00BF5B1EF5E77C6920231C437C610B
:10AE1000002D0BD0800709D4BB602120B96000BF92
:10AE200000BF796000BF00BF401EF7D17B6054E7D0
:10AE3000800000F834F8FF1FF3B50023C34E202232
:10AE400072604024B460C24F79680D466D1EFDD11A
:10AE500074600D466D1EFDD1C50701D0726000E023
:10AE6000B260B4600D466D1EFDD174600D466D1E5E
:10AE7000FDD11D184308DF0701D0726000E0B26009
:10AE8000B4600F467F1EFDD174600F467F1EFDD15A
:10AE9000ED188308DF0701D0726000E0B260B46093
:10AEA0000F467F1EFDD174600F467F1EFDD1ED1849
:10AEB000C308DF0701D0726000E0B260B4600F46E3
:10AEC0007F1EFDD174600F467F1EFDD1EB18DB079E
:10AED00001D0726000E0B260B4609D4D0B465B1E15
:10AEE000FDD174600B465B1EFDD1B260B4600B46B1
:10AEF0005B1EFDD174600B465B1EFDD17260B460B9
:10AF00000B465B1EFDD174600B465B1EFDD1736961
:10AF10002022934373612B7E1D1E09D0B4600A4624
:10AF2000521EFDD174600A46521EFDD15B1EF5D142
:10AF3000B4600A46521EFDD1326974609206D20F87
:10AF40000B465B1EFDD1B4600B465B1EFDD1336921
:10AF500074609B06DB0F0F467F1EFDD15B00134321
:10AF6000B4600A46521EFDD132699206D70F4022C4
:10AF700072600A46521EFDD1BA001A43012A17D048
:10AF8000022A70D0042A6ED021350AD04023B36043
:10AF90000846401EFDD173600846401EFDD16D1E5F
:10AFA000F5D1716920200143716170601046FCBDCC
:10AFB00083073ED50024254620234027B7600F464F
:10AFC0007F1EFDD13769BF06FF0FBC464027776063
:10AFD0000F467F1EFDD167086446E4073C43654485
:10AFE0005B1EEAD14023B3600F467F1EFDD1376957
:10AFF0007360BF06FF0F491EFDD17D40E90700D0F9
:10B0000008220199002900D00C6051490C7E002CC7
:10B010000AD04D68B3602946491EFDD173602946A8
:10B02000491EFDD1641EF5D171692024214371614F
:10B030003AE0002D0AD04024B4600B465B1EFDD1DF
:10B0400074600B465B1EFDD16D1EF5D17369202423
:10B0500023437361019B00271B682546DC0703D04F
:10B060002024746002E038E02024B4604024B460FE
:10B070000C46641EFDD1402474600C46641EFDD154
:10B08000FF185B086D1EE9D1FB0702D02023736017
:10B0900001E02023B36040243546B4600B465B1EBC
:10B0A000FDD16C60491EFDD1000602D52849002063
:10B0B0008860274B197B00290DD02020B0605B6889
:10B0C0004024B4601846401EFDD174601846401EEE
:10B0D000FDD1491EF5D1202067E71D4B5B7E9C46C4
:10B0E000002B0DD083070BD521244027B7600B46DA
:10B0F0005B1EFDD177600B465B1EFDD1641EF5D152
:10B10000002D0AD04024B4600B465B1EFDD1746054
:10B110000B465B1EFDD16D1EF5D1746920231C43C7
:10B1200074616446002C0ED080070CD4B3602124D7
:10B130004025B5600846401EFDD175600846401E9A
:10B14000FDD1641EF5D1736030E70000800000F887
:10B1500034F8FF1FF0B50023104C1A460E4E40275E
:10B16000656815E0002A02D10B780822491CDC072B
:10B1700002D02024746001E02024B460B7602C4623
:10B18000641EFDD177602C46641EFDD15B08521E03
:10B19000401EE7D2F0BD0000800000F834F8FF1F29
:10B1A00015488178090703D58178082211438170F9
:10B1B000124800210160012210481204C038426088
:10B1C0000F48026803239B049A4302600D484268BB
:10B1D0000D4B1A4003231B06D21842600B48017224
:10B1E00080220276017001224270094A1170817931
:10B1F0000907890FFBD1704700D007400081044048
:10B200000070044000800440FFFFFBC00040064087
:10B2100000500640BFF34F8F04490348C860BFF396
:10B220004F8F00BFFDE700000400FA0500ED00E0CD
:10B23000F8B52E4E002435780095280741D5317C8D
:10B240000A090807C00F4B07DB0F154605431AD143
:10B25000950040002818C018254BC0001D5CAD06A5
:10B260002D0F012D0FD1C5186F88002F0BD1214F45
:10B27000BA5C6A801A5C520601D5882200E0C822B6
:10B280001A5401200143EFF31080C507ED0F72B689
:10B29000194A184F143FB86811541921401CFDF782
:10B2A000E6F9B960002D00D162B608203070002C9C
:10B2B00002D1307D800601D5012400E000243578DC
:10B2C000BBE700990B482943083805F005FF002C1F
:10B2D00001D0012000E00020064914390A7810430B
:10B2E0000870357002F0C2FBF8BD000080200740F6
:10B2F000001A0020BCEEFF1FC02000201CB500205B
:10B3000001906A4601A90948FEF732FB002808D0DF
:10B31000074880210078009A0843019902F0CEFB8B
:10B320001CBD0449012008701CBD00008C260020B3
:10B330008C5E010034EFFF1F38B5174D174C28887D
:10B340006188421A16486168007801F041FF61681F
:10B3500080B209186160618809188AB26280298800
:10B360008A4206D20F49104B09784900595A814246
:10B3700011D96B460D490E48FEF7CCFA002500287E
:10B3800006D02078002803D00020FFF7B7FF2570F3
:10B3900065800648606038BD925E010034EFFF1F93
:10B3A0008D5E0100DFEFFF1F8E5E0100421800205E
:10B3B0008C26002010B50446400702D50020FFF778
:10B3C000BBFF200702D50020FFF798FF10BD00202B
:10B3D00070470000034801694069081A024909885A
:10B3E000081A70473CEFFF1F825E010070B50B4DDD
:10B3F0000C460346696B286B88420BD9401A84427D
:10B4000000DD044622461846FDF774F8686B001903
:10B41000686300E00024204670BD00003CEFFF1F81
:10B4200000207047F8B5184F0C4606467969386910
:10B43000401A16490988081A002801DC0020F8BDC6
:10B44000844200DD0446FA69B869002590420DD3B4
:10B450000F4A031951188B4208D30D1A2A46314658
:10B46000FDF748F876190A48641BB861002C06D02D
:10B4700022463146FDF73EF8B8690019B8613969CE
:10B48000601909183961F8BD3CEFFF1F825E0100A9
:10B49000C217002010B5054C6068002805D10120B6
:10B4A000606000F005F80020606010BD3CEFFF1FF9
:10B4B000F8B5234CA06800283DD0616920690026BA
:10B4C000421AE06811460143002935D021461D4F3C
:10B4D000C9691D4D002A10D0A069814205D3388862
:10B4E0008B182818834200D3421A1848007843006A
:10B4F0001748C05A904200DA02461648E6600078C3
:10B500008023184302F0DAFAE1690918E1616269FF
:10B51000121862613B88EB188B4200D1E56121690A
:10B5200091420BD1094909784A000949895A814257
:10B5300004D10120E060F8BDA660F8BDE660F8BD6A
:10B540003CEFFF1F825E0100C2170020DFEFFF1FEC
:10B55000865E0100805E010010B50C4C206A002858
:10B5600003D0A06A401CA06210BD0120206260626E
:10B5700000F00EF8002060622062616B206B884250
:10B58000F2D0401AFFF74CFF10BD00003CEFFF1F48
:10B5900010B5134C1348216B154B0A1A124800883A
:10B5A000821A124800784000185A82420EDB114875
:10B5B000007801F00DFE216B08182063A06A0028B6
:10B5C0000CD0616A002909D1401E06E00120E0622A
:10B5D000606A002802D0A06A401CA06210BD000072
:10B5E0003CEFFF1F02180020845E0100DFEFFF1F09
:10B5F000865E0100815E010010B50446400702D559
:10B600002046FFF7A9FF200702D52046FFF742FF9B
:10B6100010BD7047002070470020704710B50C48DF
:10B6200000F042F8002812D00948FDF70FF8094948
:10B63000020A08704A70020C8A70000EC870044832
:10B6400002790A7142794A7180798871012010BDAE
:10B6500074EFFF1FC016002010B51048002444608E
:10B660008460C46004610E49816144610462446283
:10B670008462C462C1610B49016341630146048075
:10B680004B203831C001FCF7AFFE044808213830A8
:10B6900004714471817100F019F810BD3CEFFF1F77
:10B6A000C21700200218002070B50446064D21463E
:10B6B0002868FCF799FE2879A07168796071A879EB
:10B6C0002071012070BD00006CE9FF1F10B508F06B
:10B6D00049FA04F025FF012010BD10B508F094FAD6
:10B6E000012010BD0120704710B50446FCF7AEFFE5
:10B6F00006490860A07908716079487120798871DD
:10B700000020C871084608F093FA10BD6CE9FF1FCD
:10B7100010B51148002444608460C46004610F497E
:10B7200081614461046244628462C462C1610C4903
:10B73000016341630480FFF7D0FF07494B20383194
:10B74000C001FCF751FE04480821383004714471EF
:10B750008171FFF7C9FF10BD3CEFFF1FC21700202A
:10B760000218002010B5FFF7D3FF10BD70B51B48BD
:10B770000078002831D01A4C0025206A01260028C4
:10B780000AD1616B206B884206D11649884203D0EA
:10B790002163E56225626163A06A002810D0206AF7
:10B7A00000280DD1E06A00280AD12662FFF7F0FEDA
:10B7B0002562616B206B884202D0401AFFF730FE91
:10B7C000A1686068084308D161692069884204D093
:10B7D0006660A660FFF76CFE656070BDDDEFFF1F61
:10B7E0003CEFFF1F0218002070B505460F480068A7
:10B7F000C1698847002816D10D4C002D06D005F0F0
:10B800002DF82060002007F0B1FF0CE005F026F8CD
:10B810002168401AFF212D31884201D3012000E028
:10B82000002004F091FE012070BD0000F05A0100DC
:10B8300068E9FF1F002070470020704710B50249DB
:10B840000880FFF74FFF10BD3CEFFF1F10B50B48FE
:10B85000FCF7FCFE094C0002E178000A09060843E7
:10B860000749FCF7C1FD06482179017161794171F1
:10B87000A1798171FFF738FF10BD0000C0160020CC
:10B8800074EFFF1F01078A0E044910B551180A789A
:10B89000FD231A400A7002F081F810BDC020074055
:10B8A00010B501464A790B798078110219430206D6
:10B8B00001D4024A115402F071F810BDBCEEFF1F12
:10B8C000704710B500F016FB10BD0000094A094989
:10B8D00080320028087D04D0012318430875102009
:10B8E00005E0400840000875107AEF21084010720A
:10B8F000704700008020074010B50C4C0C48A2880F
:10B900000078824200D90246002A03D1074900206C
:10B91000143908718020216802F0D0F821680918D4
:10B920002160A188081AA08010BD0000F0EFFF1F61
:10B93000675E010010B5064C0020A288216801F066
:10B9400047FC216809182160A188081AA08010BD51
:10B95000F0EFFF1F704700000749020605D50007FA
:10B96000800E40180178FA2203E080004018017828
:10B97000F622114001707047C020074007490206B7
:10B9800005D50007800E40180178052203E08000ED
:10B99000401801780922114301707047C020074008
:10B9A000F8B504466F4F704D704E800720D502F0F9
:10B9B00053F83878C009FFF7CDFFF888A8803878A9
:10B9C0004106890F04D001295CD0022975D169E0B4
:10B9D00079780B0002F09EF80C070D71137119288D
:10B9E000712D333B4A7101F095FD1FE0FFF784FF95
:10B9F00070E0002004E002F043F85D483DE00120E3
:10BA000001F0CAFD002858D0F5E7C006C00E54D199
:10BA1000B8788021084330704006400E012102F0C2
:10BA200005F802F02DF855E001F05EFC002844D046
:10BA3000DCE7C006C00E40D14C48401C14E001F0C9
:10BA4000FFFD002839D002F01BF84A4815E0C00677
:10BA5000C00E012831D1707800282ED03879B17805
:10BA600088422AD2444940182860BFE701F0ACFE62
:10BA7000002822D002F004F840480068002829D0AD
:10BA8000804727E0C006C00E17D0012815D100F06E
:10BA900017F900281ED100F06FF900281AD100F024
:10BAA000BBF808E0C006C00E07D100F09FF90028DF
:10BAB00010D100F0E7F900280CD13878C00904D182
:10BAC000F888002801D0002000E0802001F0B8FFB5
:10BAD0000020A880600704D53878C0090DD001F097
:10BAE000D7FF200733D53878C00927D0A888317907
:10BAF00008432CD0FFF700FF29E0A8880028F0D0E9
:10BB0000FFF718FFA8880028EBD138784106890F85
:10BB10000ED001290CD1C006C00E09D0012807D1D2
:10BB200000F05CF80028DCD100F02AF80028D8D119
:10BB3000802001F085FF0020A880D2E73078010640
:10BB400005D54006400E3070002101F06FFF600601
:10BB500002D50020FFF796FE200602D58020FFF7D1
:10BB600091FEF8BDF8EFFF1FF0EFFF1FDCEFFF1FA6
:10BB7000F05E0100E85E010097EEFF1FEC5E010041
:10BB800010B51349134A08791278904203D0124A2B
:10BB90001278904219D14878002804D0022805D0A4
:10BBA000202812D10EE0FFF745FE05E0C87889781D
:10BBB00000020843FFF740FE002806D001F060FFB6
:10BBC000012010BDFFF742FEF6E7002010BD000087
:10BBD000F8EFFF1FFCECFF1FFDECFF1F10B50B493A
:10BBE0000B4A08791278904203D00A4A12789042A0
:10BBF0000AD14878092807D100F082FB002803D039
:10BC000001F03EFF012010BD002010BDF8EFFF1F26
:10BC100000EDFF1F02EDFF1F70B52449244A08798B
:10BC20001278904203D0234A127890423BD11F48A9
:10BC30004978C278837810021F4C204D184304299C
:10BC400020D008DC00290FD001290FD002290BD009
:10BC5000032928D111E0202906D0212919D0222931
:10BC60001AD023291FD11AE02C6010E0FFF7D4FC72
:10BC700005E02C60FFF740FE09E0FFF7CBFC002851
:10BC8000F7D110E0FFF7A3FB0BE001F0F9FE012074
:10BC900070BDFFF7C3FCF2E7FFF7D0FD01E0FFF74F
:10BCA000A3FD0028F1D1002070BD0000F8EFFF1FB8
:10BCB000FCECFF1FFDECFF1FC0160020F0EFFF1F84
:10BCC000F8B5254E254930790978884203D02449B2
:10BCD000097888423DD17078224C234D234F0300D0
:10BCE00001F018FF0C3707232D3737373737182661
:10BCF000333700F023FA00282BD0F078012802D047
:10BD0000032803D003E01A48206000E02560FFF715
:10BD1000F3FD12E0F078022802D0032803D00CE0F3
:10BD20001448206009E0256007E000F0EFF908E022
:10BD300000F0BEFA0BE001F0A3FE0120F8BD00F018
:10BD4000F3F9002805D02760E1E700F0CFFA0028DA
:10BD5000F1D10020F8BD0000F8EFFF1F00EDFF1F3C
:10BD600002EDFF1FF0EFFF1FA4EEFF1FC016002023
:10BD7000011700204217002010B51848184A017911
:10BD80001278914227D142780146C8788B78000218
:10BD90001843CB798C7919022143FE2A0CD0FF2A53
:10BDA00019D1002817D1002915D101F051F9002827
:10BDB00011D001F065FE0CE000280CD101290AD158
:10BDC00000F03AFE002806D0074906480860FFF751
:10BDD00093FD012010BD002010BD0000F8EFFF1FF3
:10BDE00001EDFF1FC0160020F0EFFF1F70B51F4DC3
:10BDF0001F49687809780026884235D16879297901
:10BE00000002084302282FD1AA781A4C002A2BD00E
:10BE1000002004E02178002900D00C19401C411CAE
:10BE20008A42F7D82078002819D004F089F9014611
:10BE3000E01CFCF7C4FA104A01261460E979AB79DA
:10BE400020780902194381420BD90C499080097866
:10BE5000491E084206D10A490120087002E0002666
:10BE600002E09180FFF748FD304670BDF8EFFF1FFC
:10BE70008A5E010058EEFF1FF0EFFF1F675E0100B2
:10BE8000E0EFFF1F10B5154A1549507809780024D6
:10BE9000884220D1507911790002084307281AD12D
:10BEA000114B10481860417A007A09020143D07999
:10BEB0009279000201241043884209D90B489980E5
:10BEC0000078401E014204D109490120087000E0B9
:10BED0009880FFF711FD204610BD0000F8EFFF1F0E
:10BEE0008B5E010008EDFF1FF0EFFF1F675E010092
:10BEF000E0EFFF1F074800214170C160016141610F
:10BF0000418081808161C161C18001810162418183
:10BF1000704700007CEFFF1FF8B54A4EB08871886B
:10BF2000494F00257C1C884218D3B069002815D1E0
:10BF30007561B580012339787A1C184608F076FAC5
:10BF400070807088002809D0404877610078012807
:10BF500001D8746102E07088401C708070880028ED
:10BF60003AD1F068002801D0F56035E0306900284A
:10BF700032D03649097801290ED83D70B5800223A8
:10BF80007A1C0021012008F051FA70807088002886
:10BF900000D0746135611FE03C780127202C00D36C
:10BFA00000243946A14001421AD0601CC1B2264A81
:10BFB00002231170B5800120521C08F037FA7080FE
:10BFC0007088002804D0204870617088401C708000
:10BFD0003069A740B84330617088002806D102E07C
:10BFE000641CE4B2DAE7B069002828D07088B18810
:10BFF000174F401A84B2387841001648405AA04280
:10C0000000D2044614480078002805D08021084357
:10C010002246716901F052FD706910490019706182
:10C02000B088001980B2B0800988884208D2387878
:10C0300041000848405AA04202D10120B061F8BD39
:10C04000B561F8BD7CEFFF1F00170020725E010094
:10C05000DFEFFF1F6E5E0100685E0100745E01008D
:10C06000F8B51C4C002620891B4D1C4F002803D11D
:10C07000E5613888E0802681E0882189421A1848E5
:10C08000E169007801F0A4F8E16980B20918E16182
:10C09000218909188BB22381002809D039888B4265
:10C0A00006D21049104A09784900515A814210D9E4
:10C0B0000E48017801200129009003D80021064A8A
:10C0C000022003E029786A1C02205B1E08F046FA71
:10C0D0002681F8BD7CEFFF1F41170020765E01002E
:10C0E000695E0100DFEFFF1F6E5E0100735E0100FD
:10C0F00010B50446000702D52046FFF70DFF600784
:10C1000002D52046FFF7ACFF10BD000003480449EC
:10C110008078085C0349087001207047F8EFFF1F22
:10C12000A2EEFF1FC016002010B508F07DF90249ED
:10C130000870012010BD0000C016002010B50B498A
:10C140000022C878012804D0022804D0032806D190
:10C1500003E0074A02E0002010BD064A521C89781D
:10C16000002308F063F9012010BD0000F8EFFF1F65
:10C1700000170020A3EEFF1FFEB5444800780028FA
:10C180007ED0434E002031788446481C30704148B0
:10C19000042300784200821893405B1E019299426A
:10C1A00003DB0021317001218C463B4A00251188B8
:10C1B000FF2901D2491C118041003848405A3649B4
:10C1C00000900988884200D101253549002009786E
:10C1D0008E4648E000216246002A0DD0314A135CA9
:10C1E000FF2B01D25B1C13542F4B1B5C002B03D085
:10C1F000125C9A4200D301212B4A0223145C019A5B
:10C20000934022469A40009B9A4203DA002C01D0C8
:10C21000012200E00022002D06D0002A04D00123D4
:10C22000376983403B433361204B1B5C9C420CD0FD
:10C230001C4C245C9C4206D30124376984403C4357
:10C24000346100243470184C2354002909D0002A8A
:10C2500004D101213269814011433161114A002129
:10C260001154401CC0B27045B4D3002D02D00A490D
:10C27000002008803069002806D07088002800E07F
:10C2800002E001D1FFF748FEFEBD0000DDEFFF1F19
:10C290007CEFFF1FDFEFFF1F9EEEFF1F6A5E0100B6
:10C2A000725E0100A0EEFF1FA1EEFF1FA2EEFF1FB6
:10C2B0000A480A498078C978002802D0084A81547F
:10C2C00009E0094B0020074A1B7802E01154401C8A
:10C2D000C0B29842FAD3012070470000F8EFFF1F68
:10C2E000A1EEFF1FA2EEFF1F725E010010B5034812
:10C2F000807808F031F9012010BD0000F8EFFF1F31
:10C3000038B50D490022C878012804D0022804D08D
:10C31000032806D103E0002038BD084A00E0084A9F
:10C32000521C00230093CB798C791B02234389781C
:10C3300008F014F9012038BDF8EFFF1F4117002065
:10C34000A3EEFF1FF8B5EFF31080C007C00F72B661
:10C35000564D0021EC68E9602A7800922970002887
:10C3600000D162B6E00708D001F0C6FA08F0A2F9E1
:10C370004F480068002800D08047E00606D501F04D
:10C3800093FB4C480068002800D08047A00606D5E3
:10C3900001F03CFB48480068002800D08047600757
:10C3A00004D546480068002800D08047022C09D1F7
:10C3B00043480168002902D04248007A8847414832
:10C3C000FF210172200767D53F4FEFF31080C207AE
:10C3D000D20F72B6A9686868884257D1012156E029
:10C3E000EFF31081CE07F60F72B638490C5C1921B5
:10C3F000401CFCF73CF96960002E00D162B6204673
:10C400002207D30F21066207090FD20F002908D196
:10C410005C00A418E4003C5D0026A406240F0D2C4B
:10C420000AD08C005B00E3189A18D600BA5D920619
:10C43000120F012A13D01DE02869022188432861C8
:10C44000387E4006400E3876387C4006400E387400
:10C450001F486E7001680029B7D0022014E000293F
:10C4600002D1C007C00F687019480159002901D0D6
:10C4700004208847B85D8006000F0928A5D114481C
:10C4800001590029A1D0082088479EE70021002AF1
:10C4900000D162B60029A3D00098002804D0094931
:10C4A000087DDF2210400875F8BD0000A8EEFF1FD0
:10C4B000945E0100985E01009C5E0100A05E010098
:10C4C000A45E010080200740001A0020C020002048
:10C4D000A85E010010B519484024047003F0AEFABC
:10C4E000182001F059FB1648017B8022114301738B
:10C4F000017B0906FCD41349114B090A803B1977CB
:10C5000010490F4A090C603A11740E49090E117551
:10C51000FF2119700C490968002900D004210B4A39
:10C520001268002A00D00222114319221143197106
:10C530000470017B2143017310BD0000BCEEFF1F9E
:10C5400000210740001A0020A05E0100A45E010047
:10C5500070B500F015F900282AD01648022404709E
:10C560004470154E03203463307014480546FCF7C0
:10C570006DF8022808D9114920461F39FBF734FF0E
:10C5800029462046FBF730FF0D48802100782246DF
:10C590000843084901F092FA2846FCF757F8316B36
:10C5A000401A2946FBF720FF044901200839087387
:10C5B00070BD000082170020A4EFFF1F6B29002030
:10C5C000785E010010B510490878022808D00328C9
:10C5D0000FD0042810D0052801D10020087010BD0C
:10C5E0000A48C07B282801D0A828F8D100F068FAB2
:10C5F00010BD00F06FFD10BD054880210078084394
:10C6000000F082FDF5E70000A4EFFF1F44290020A1
:10C61000785E010010B51D4A117800290FD001295C
:10C6200010D01B48052900781BD0072927D000F01F
:10C630006BFD18490220087300F04CFD10BD00F09E
:10C640000BF910BD13481F38C07B2A2803D02F28B0
:10C6500004D0AA28F5D100F011FB10BD00F09EFA1D
:10C6600010BD012181400C480068014201D0012029
:10C6700000E00020094A0AA101F0FEFA10BD0020E6
:10C680001070106B1F28DAD010BD0000A4EFFF1F40
:10C69000795E010063290020E8EFFF1F3F040000DE
:10C6A0002E5C736F757263655C7573625C6D73632A
:10C6B0005C757362645F6D73632E630010B5144C18
:10C6C0006068E060002801D0012010BD1148FBF730
:10C6D000BDFF002814D00F480838007B000604D5A1
:10C6E0000D4880210078084308E00A481F30FBF716
:10C6F000ADFF216B884203D00848007800F004FDAC
:10C70000044901201731087300F0E4FC002010BD3B
:10C71000A4EFFF1F4C290020785E0100795E010024
:10C7200010B5124801798F200140080605D5080789
:10C73000000F01221204824001E001228A400C48CD
:10C740000478802004438C420ED10A4800681042CD
:10C750000AD00948FBF77AFF0849884204D10D2224
:10C760000549204601F0AAF910BD0000F8EFFF1FAF
:10C77000785E0100E8EFFF1F632900205553425304
:10C7800070B50C48FBF762FF0A4C022517340028ED
:10C7900008D020461F38007B000608D406480078E1
:10C7A00000F0B2FC257300F095FC002070BD012064
:10C7B00070BD00004C290020795E010070B5114861
:10C7C000FBF744FF104C216B884202D82063032002
:10C7D00000E0042020700D4880210078226B08437F
:10C7E0000B4901F06BF907481F300546FBF72EFF98
:10C7F000216B401A2946FBF7F7FD0249002017314B
:10C80000087370BD4C290020A4EFFF1F785E010063
:10C810008217002010B506480649028806480078AD
:10C8200000F0D6FC05490863FFF7F4FE10BD0000D8
:10C830007E5E010082170020795E0100A4EFFF1FD9
:10C8400010B50446400702D50020FFF7E3FF20079C
:10C8500001D5FFF7B7FE10BDF8B5704E316B1F293B
:10C8600001D20A4600E01F2200206D4D6D4B02E010
:10C870001C5C2C54401C9042FAD36B4880220078F8
:10C880000127104300901F2970D16548FBF7DEFE99
:10C89000664988426AD1281DFBF7D8FE604C1F34D8
:10C8A000211DFBF7A1FD20461738FBF7CFFE2146DF
:10C8B0000831FBF799FD687B002804D1A87B00288C
:10C8C00001D0102801D9277374E0E87B2A283BD0D7
:10C8D00020DC1A2847D00EDC0428F4D006DC00281F
:10C8E0003BD00328EFD100F071FBF8BD1228EAD14C
:10C8F00000F0AAF8F8BD23283CD006DC1B282FD076
:10C900001E28E0D100F0CCF8F8BD252835D0282825
:10C91000D9D13BE09E2836D00EDC5528D3D004DC9C
:10C920002F2842D03528CED103E05A281FD0912895
:10C93000C9D100F019FCF8BDA12821D0A3284ED000
:10C94000A82823D0AA28BED100F080FA0028F2D06F
:10C95000287B00063BD43770F8BD00F00FFCF8BD13
:10C9600000F0E8FBF8BD00F043FAF8BD3BE000F052
:10C970000DFAFAE700F0EEFAF7E700F0C5FAF4E78F
:10C98000FFF7E6FDF1E700F079FBEEE700F05EFA75
:10C990000028EAD0287B000604D50220307000F081
:10C9A0008FF8E2E72248007815E0287C800704D45D
:10C9B0000020207300F08EFBD7E700F047FA002834
:10C9C000D3D0287B000602D437703762CDE71648F3
:10C9D00080210078084300F097FB0220E9E70098E7
:10C9E00000F092FB6FE7104C009800F08DFB207870
:10C9F000104C0107090F01200004884021680C4DEC
:10CA000008432060287800F07FFB28788740206862
:10CA10000743062027603070A7E70000A4EFFF1F40
:10CA20004429002082170020785E010055534243BC
:10CA3000795E0100ECEFFF1F024900200870012021
:10CA400070470000C016002010B5FFF799FE0028BF
:10CA50001FD0104B0020187080215970022199704E
:10CA6000D97020241C7158719871D8710A480168D6
:10CA700008200A78002A02D01A54491C00E01C54ED
:10CA8000401CC0B22428F4D3044924200863FFF7D3
:10CA900095FE10BD8217002054EEFF1FA4EFFF1F6C
:10CAA00010B50548C07CC107044800D001210173BE
:10CAB00000F010FB10BD0000442900206329002075
:10CAC000F8B5314D314FA969686A002688420AD30A
:10CAD000387880210024084300F016FB2C480673A8
:10CAE00000F0F8FA08E02B48007841002A48445A40
:10CAF000E86A844200D30446FFF7E0FD002800D135
:10CB00000024A86A00282DD0002C0ED0A96AE8695C
:10CB10008022411838781043224600F0CFFFA86ADF
:10CB20000019A862E86A001BE86229696869AA6AB4
:10CB30004143914203D1AE62696A081868621448A1
:10CB400008300746FBF782FD001B3946FBF74CFC1B
:10CB5000002C06D0E86A002803D1032028700C4876
:10CB60000673F8BD002CE0D02969E86A4018401E21
:10CB7000FBF77DFD69690246884200D90A46E969EA
:10CB8000686A07F057FDC1E7A4EFFF1F785E010058
:10CB900063290020DFEFFF1F7A5E0100F8B5334CF8
:10CBA0000025A169606A884208D33148256300786E
:10CBB00000F0AAFA2F48057300F08CFAFFF77EFD0B
:10CBC000002806D0206B002824D0A06A002802D0BC
:10CBD00010E025631EE02169E06A4018401EFBF763
:10CBE00046FD61690246884200D90A46E169606AE9
:10CBF00007F020FD00202049A76A266B08E0E369C2
:10CC00003A189A5C0B5C9A4201D0256202E0401C03
:10CC1000B042F4D3266BA06A8119A162E06A871B37
:10CC2000E7622269606942438A4203D1A562616A70
:10CC3000081860620F4808300546FBF707FD801BA7
:10CC40002946FBF7D1FB002E0CD0002F02D0207814
:10CC5000052807D1206A002805D00020054908735F
:10CC600000F038FAF8BD0120F8E70000A4EFFF1F3C
:10CC7000795E01006329002082170020F8B5384D45
:10CC8000384FA969686A0026884207D336482E6360
:10CC9000007800F039FA3E7300F01CFAFFF70EFD41
:10CCA000002800D12E63296BA86A401829698842A0
:10CCB00005D9FE222DA1002000F0DEFFF8BD0020E6
:10CCC000314905E0AB6A0A5C1B18EC69401CE25470
:10CCD0002A6B9042F6D3A86A8018A862E96A891A7A
:10CCE000E962002A25D0002914D1002812D0296930
:10CCF0004018401EFBF7BBFC69690446884200D916
:10CD00000C462246E969686A07F0ACFCAE62686AC4
:10CD100000190DE069692B690A465943814208D11F
:10CD2000E969686A07F09EFCAE626969686A401842
:10CD300068620C4808300090FBF788FC2C6B009967
:10CD4000001BFBF751FB002CB8D0E86A002802D08A
:10CD500028780528B2D13E7300F0BCF9F8BD000078
:10CD6000A4EFFF1F63290020795E01002E5C736F22
:10CD7000757263655C7573625C6D73635C75736219
:10CD8000645F6D73632E63008217002070B5FFF738
:10CD9000F7FC002824D0FFF791FC002820D0114890
:10CDA00000210170062242700F4B81701A7A08240C
:10CDB000D201C270017141718171C1710B481C6354
:10CDC0000546FBF743FC082808D9084920461F39C7
:10CDD000FBF70AFB29462046FBF706FBFFF7EEFCB4
:10CDE00070BD000082170020A4EFFF1F6B290020F8
:10CDF00070B5FFF7C5FC002820D0FFF75FFC0028C6
:10CE00001CD00F480321017000210E4B41701A7A8B
:10CE10000424D2018270C1700B481C630546FBF7E5
:10CE200015FC042808D9084920461F39FBF7DCFA0D
:10CE300029462046FBF7D8FAFFF7C0FC70BD00007A
:10CE400082170020A4EFFF1F6B290020F8B52A48A5
:10CE5000FBF7FCFB284D00BA040A113D287D240293
:10CE60000443264E00207462B062E87B2F280AD06B
:10CE700004DC28280BD02A281CD104E0A82810D0D4
:10CE8000AA2817D109E0FFF719FC002830D0E87D67
:10CE9000A97D0002084344BA0CE0FFF70FFC00280C
:10CEA00026D01548001DFBF7D1FB00BA040A287EE6
:10CEB00024020443306944430F48F4620938FBF705
:10CEC000C5FB0D4F01260E3700280DD0A04210D013
:10CED000287B000604D50A4880210078084301E039
:10CEE0000848007800F010F93E7300F0F3F80020D5
:10CEF000F8BD0120F8BD000055290020A4EFFF1F58
:10CF0000785E0100795E010010B5FFF739FC00285A
:10CF10001AD0FFF7D3FB002816D00C4A0C489169B1
:10CF2000491E0B0E03700B0C43700B0A8370C1700B
:10CF300011690B0E03710B0C43710B0A8371C171E4
:10CF400008201063FFF73AFC10BD0000A4EFFF1F9C
:10CF50008217002070B5FFF713FC00282ED0FFF7D2
:10CF6000ADFB00282AD01648002101704170817065
:10CF70000821144AC17091690C240B0E03710B0C2B
:10CF800043710B0A8371C1710221017211690B0C8B
:10CF900043720B0A8372C1720B4814630546FBF798
:10CFA00055FB0C2808D9084920461F39FBF71CFA05
:10CFB00029462046FBF718FAFFF700FC70BD000079
:10CFC00082170020A4EFFF1F6B29002070B5FFF728
:10CFD000D7FB00282ED01B487021017000211A4B6E
:10CFE00041705A68DD681446AC4306D0062484704C
:10CFF000282404734173DA600AE0002A1BD0134A24
:10D00000127B002A1BD005228270202202734173FA
:10D01000C1700171417181710A22C2710172417244
:10D020008172C1728173C1730174417412201863DB
:10D03000FFF7C4FB70BD022282703A22E6E78170DE
:10D040000173E4E782170020A4EFFF1F632900208B
:10D0500010B50549002008600449FBF7C5F90449EB
:10D0600007200870012010BDECEFFF1F632900208E
:10D07000A4EFFF1F10B5FFF7EBFF10BD70B5FFF772
:10D080007FFB00281DD00F48202202700021417034
:10D09000C1770D4C0320226320700C48802100785A
:10D0A0000843084900F00AFD09480546FBF7CEFA97
:10D0B000216B401A2946FBF797F9054901200839E9
:10D0C000087370BD82170020A4EFFF1F785E010077
:10D0D0006B29002010B508490848FBF785F9084876
:10D0E000802100780D220843034900F0E7FC054940
:10D0F0000520087010BD00006329002055534253DD
:10D10000785E0100A4EFFF1F10B5044600F098FC04
:10D11000200605D52107090F01200004884001E001
:10D120000120A04002490A681043086010BD0000B9
:10D13000E8EFFF1F10B50A48817C04461F34002920
:10D1400004D001202073FFF7C5FF10BDC07C054946
:10D15000C007C00F486007F083FA0020F2E7000024
:10D1600044290020A4EFFF1F10B5034900200873D5
:10D17000FFF7B0FF10BD00006329002010B5104874
:10D18000FBF764FA0E4C173400280FD020461F38E6
:10D19000007B000604D50B4880210078084301E09D
:10D1A00009480078FFF7B0FF012004E0FFF786FA96
:10D1B000002803D000202073FFF78CFF10BD000073
:10D1C0004C290020785E0100795E01007047000064
:10D1D000F7B5074682B0002000903807860E334826
:10D1E000F500281801904488002F15D13048407868
:10D1F000002809D07008012181402D48103003F02B
:10D2000077FF002005B0F0BD2848405D8006000F84
:10D210000D2801D1012000900498A04206D2FF22DF
:10D22000E83224A1002000F027FD049C1F4A0020C2
:10D23000B101C032891803E0039A0B5C1354401CFF
:10D24000A042F9D31A481430C15D0198174F4180AC
:10D25000174876080069795DF040C0074906C00F9D
:10D26000C90F88420FD10398C179827908020099C9
:10D270001043002901D000280CD001210C48B140F6
:10D28000103003F035FF0A480069F040C00708D0AD
:10D29000C82007E006480121C943103003F010FF01
:10D2A000F1E7882078552046ACE70000001A0020FE
:10D2B000A8EEFF1F2E5C736F757263655C6869630F
:10D2C0005F68616C5C667265657363616C655C75F3
:10D2D0007362645F6B696E657469732E630000002E
:10D2E00010B5FFF71DFA10BDFEB5574A574D10781F
:10D2F000574CC006C00E02D001287CD18CE05549A5
:10D30000D0780B785149544E544FC978062810D024
:10D3100006DC012809D0022815D003286BD14FE084
:10D32000072832D00F2866D166E04D4820601220D1
:10D3300070E0002B5FD0002903D04A4820600A200B
:10D3400068E04948FAE7002B01D1012979D0022091
:10D35000002904D000977870002092780DE00096A4
:10D360007070F9E700990B78002B05D0CB788E7898
:10D370001B02334359180091401C8242F2D100989D
:10D38000017800295DD0206040E0002B59D00720B3
:10D39000002904D000967070002092780DE000976C
:10D3A0007870F9E700990B78002B05D0CB788E7850
:10D3B0001B02334359180091401C8242F2D1DEE730
:10D3C0002A4800909078032801D0002009E002F05C
:10D3D00015FF0DE000990B78002B01D05918009132
:10D3E000401C91788142F5D100980178002928D01D
:10D3F000206000780EE024E01D48007800281FD04F
:10D400001C4800902060017800291AD0C1788278E9
:10D4100008021043019005E001A9684600F02EF8CB
:10D4200000280DD0A1880198814208D980B2124904
:10D43000A0800978491E084201D1012028710120ED
:10D44000FEBD0020FEBD0000F8EFFF1FDCEFFF1F58
:10D45000F0EFFF1F655E0100F8150020FFECFF1FD5
:10D46000185F01002B5F01002A5F0100665F010069
:10D47000665E01002C5F0100675E010070B51A4A0C
:10D480001A4CD3781A4A25781478174A194E12790B
:10D49000212B02D0222B24D118E0AA4201D0A24293
:10D4A0001FD1154A1378154A002B127801D1012A91
:10D4B00017D0002A08D0124A02601046114A12887A
:10D4C00080183060092009E00F4AF5E7AA4201D030
:10D4D000A24206D10D4830600D4800880860012046
:10D4E00070BD002070BD0000F8EFFF1F00EDFF1FB2
:10D4F00002EDFF1FF0EFFF1F655E0100DFEFFF1F72
:10D50000FFECFF1F06EDFF1FF8150020F45E010081
:10D51000165F010070B51D481D4B0078C106C90E8D
:10D520000AD01D461948143D1A4C6A780079012921
:10D5300006D0022928D10AE015480E38186021E0EB
:10D54000002A21D0A97888421ED2002016E08F211F
:10D550000840010605D50607360F01210904B14030
:10D5600001E001218140002A01D100070CD1A86807
:10D57000084209D0E868084000D001202070000A65
:10D5800060701C60012070BD002070BDF8EFFF1FAF
:10D59000F0EFFF1FC016002070B5274B0246187829
:10D5A0001946C0064988254EC00E04D001282BD04C
:10D5B000022829D111E0012926D10224002A05D010
:10D5C000012000F079FAF088204304E0002000F008
:10D5D00073FAF088A043F0802CE01C798F2004407F
:10D5E000200605D52007000F01252D04854001E008
:10D5F0000125A5407078002806D0200704D0B06827
:10D60000284201D0002901D0002070BD002A05D099
:10D61000204600F015FAF06828430AE030692842F5
:10D6200008D12046FEF72EF92046FFF759FEF06894
:10D63000A843F060012070BDF8EFFF1FDCEFFF1F73
:10D64000F8B55A4800260178C906C90E7ED1574F51
:10D6500080781C3F00287AD0554801783846C07839
:10D66000002901D1012871D0002801D0514C70E06F
:10D67000514C6EE06078022805D0042847D0052878
:10D6800047D0072860D1494861798078814239D1F3
:10D6900078702079B8704A490020484A0B8802E027
:10D6A00000211154401C9842FAD301250120B96889
:10D6B000A840084202D02846FEF74EF90120000497
:10D6C000B968A840084204D0284680210843FEF7E4
:10D6D00043F96D1C102DE9D33A48B8600020F8607A
:10D6E00038613D460120FEF7EBF8E079400604D5AD
:10D6F000E98801200143E98026E0E88840084000ED
:10D70000E88021E0E078A178000208431DE0E67897
:10D710001AE0002E18D1A5788F200540280605D5DF
:10D720002907090F01200004884001E00120A840DA
:10D73000B96801432046B960FEF7B2F82846FEF703
:10D740001DF9284600F02AF9207801E02AE004E0DB
:10D750000419207800288DD11FE0002501247D7058
:10D7600080260120B968A040084202D02046FEF77A
:10D77000F3F801200004B968A040084203D0204615
:10D780003043FEF7E9F8641C102CEAD3FD600D4825
:10D790003D61B8600020FEF793F8044879788078FE
:10D7A000884201D00020F8BD0120F8BDF8EFFF1F2E
:10D7B000655E0100FFECFF1FF815002097EEFF1FCC
:10D7C00004EDFF1F01000100F0B585B000274548BA
:10D7D0000397019700783E46C006C00E01287ED10F
:10D7E00040491C394878002876D0002002903E48F5
:10D7F00002780846C078002A01D101286FD000289D
:10D8000001D03A4C64E03A4C62E06078022805D0DE
:10D8100004280ED005281ED0072857D13148617939
:10D820001C384078814251D0E078A178000208434A
:10D830004DE0A778E678002001902A480179B942A6
:10D8400044D18078B04241D1012002902948C15D85
:10D850000391C6553AE023490879B84236D1A078F9
:10D860008F22104000900006009804D50007000F9A
:10D8700001252D0400E0012585408878B04214D1AF
:10D8800018481C38816829438160C168A943C16078
:10D890002046FEF705F80098FEF770F8009800F0B3
:10D8A0007DF801982843019010E0039886420DD13D
:10D8B000019828420AD10B481C388168A94381602D
:10D8C000C168A943C1600098FEF746F820780419A2
:10D8D0002078002899D1029805B0F0BDFFE700201C
:10D8E000FAE70000F8EFFF1F655E0100FFECFF1F85
:10D8F000F815002097EEFF1F70B501201F490006A4
:10D900000860BFF34F8FBFF36F8F01201C4D0024C1
:10D91000810049190C70401C1028F9D319211948AD
:10D92000FAF792FE1848194944608460C460047094
:10D93000447040220B464A80C0334B60C8230B70B2
:10D940000C72134BCC614B610D212970114901619F
:10D950000B484038017D022319430175FF210170F6
:10D960000172017304760C480168090A0902114327
:10D970000160182000F010F970BD000080E100E0A7
:10D98000C0200740C0200020A8EEFF1F001A002082
:10D99000401B00205555555518E400E0F8B50546E4
:10D9A000154F2C073E4600060121C03E240F0028DB
:10D9B0000EDA6000401C8140104803F08DFB20020D
:10D9C000C11960018019803141610021C161F8BD38
:10D9D00068008140C943094803F072FB07486101B0
:10D9E000001D425D881942802202D21942608822BD
:10D9F000725400210172F8BDC01A0020B8EEFF1F5A
:10DA000010B5FDF7AFFEFFF735FB10BD02480179F9
:10DA1000DF221140017170478020074010B5FEF7EA
:10DA2000ABFBFDF7A3FE00F0E7FA10BD002903D120
:10DA300040060249400E08767047000080200740EB
:10DA40000007810E03480818017802221143017073
:10DA500070470000C020074010B50822024900208E
:10DA6000FFF7B6FB10BD0000F8EFFF1F10B503482D
:10DA700001214902006902F01FFF10BD34E9FF1FB8
:10DA800010B500221146802000F018F810BD0000EB
:10DA900010B50348034902780020FFF799FB10BD39
:10DAA000675E0100C0160020024801792022114360
:10DAB000017170478020074070470000F8B50007EB
:10DAC000114F840E1646A41CE200D01946803D4634
:10DAD0000023A001C035451902E0C85CE8545B1C76
:10DAE000B342FAD3094960080969C140C90701D0A6
:10DAF000882100E0C821B954012181400348103039
:10DB000003F0F6FA3046F8BD001A0020A8EEFF1F19
:10DB10000020704730B47446641E2578641CAB4204
:10DB200000D21D46635D5B00E31830BC184700005F
:10DB3000002805DBC106C90E0120884001490860A4
:10DB40007047000080E200E0002809DBC106C90E32
:10DB50000120884003490860BFF34F8FBFF36F8FE8
:10DB60007047000080E100E0002805DBC106C90E17
:10DB700001208840014908607047000000E100E092
:10DB8000002805DBC106C90E012088400149086054
:10DB90007047000000E100E0002805DBC106C90E67
:10DBA00001208840014908607047000000E100E062
:10DBB0008307FF22DB0E9A408907090E994000284F
:10DBC00008DB830809489B001818036893430B433C
:10DBD000036070470007000F0838830804489B0063
:10DBE0001818C36993430B43C361704700E400E016
:10DBF00000ED00E010B5002A06DA52005208D21DEE
:10DC0000D308DB00102203E0D21C93089B000C22F7
:10DC1000002B02D09C188C4201D9012010BD821823
:10DC20008360411802604160C91AD018884202D846
:10DC300010600246F9E70020106010BDB0B5044640
:10DC400004F090FA002804D0034F0249BC46206833
:10DC500000DFB0BDFFFF0000251C0100B0B5044689
:10DC600004F080FA002803D0024F2068BC4600DF91
:10DC7000B0BD00007D1B0100F8B516460F46002818
:10DC80001BD1EFF31080C507ED0F72B600231A46C3
:10DC90001946184600F0E0FB040003D1314638462F
:10DCA00000F03AFC002D00D162B6002C05D1EFF354
:10DCB0000380C00601D106F0F7FFF8BD3EB5002095
:10DCC0006A4610700321517001219170D07011715A
:10DCD00050719071D071074C107269462046FAF766
:10DCE00089FE01212046FAF73EFF2046FAF7C8FDDB
:10DCF0003EBD000000B003407CB50446009100200A
:10DD00006946087148710F4DD1B22846FAF722FFD3
:10DD10006A4621462846FAF7DDFE21462846FAF7EC
:10DD200003FE0006F9D5022C01D2012000E00020FC
:10DD3000FF22F83204A1FFF79FFFA00040190069FD
:10DD40007CBD000000B003402E5C736F757263658C
:10DD50005C6869635F68616C5C667265657363616A
:10DD60006C655C6B6C32377A5C66736C5F616463A4
:10DD700031362E6800000000FEB56D496D4A087806
:10DD8000FF2700256C4C022802D0002805D007E0B0
:10DD9000FF2301331360277202E0156064222272B0
:10DDA00063780622002B04D06271002801D1012083
:10DDB0000870E078002801D0401EE0700978002942
:10DDC00015D1A078002812D1607900280FD1E07A0F
:10DDD00000280CD059480078002808D1E0780028A5
:10DDE00005D12079002802D0227305206071607966
:10DDF000514A0300567AFFF78DFE0B0A770C162264
:10DE000058318C7907091B00A67114E06571207ADE
:10DE100007E0A08A3146503948435021FAF731FCD7
:10DE2000301AA07107E05020A07101F03DFDE071B3
:10DE30006079042808D0A07901F036FD05E0E0798A
:10DE4000002801D0401EE071E07901F027FCA07BA2
:10DE5000002802D0A57306F027FFFEBD384E002231
:10DE600001213046FCF7A1FD00950195112069467E
:10DE70000295087009204870012088706178002997
:10DE800005D002216A46D1706570A07202E00320BD
:10DE90006946C8700B220021684601F04FFE01223E
:10DEA00011463046FCF781FD17E0207C022809D09E
:10DEB000002904D00229BED108206071BBE7A078F8
:10DEC0000028B8D102F036FBA07A002804D0207BCD
:10DED000082804D0062804D0A5716571ABE7A771A6
:10DEE000FBE76420A071F8E7A571A4E7A0790A28F0
:10DEF00001D2401C08E00A2803D0F52803D8A571F8
:10DF000003E0A77101E0401EA071002993D1A07821
:10DF100007E0E07B002807D0401EC0B2E073052870
:10DF2000E2D00028D9D086E70A20E073A77182E703
:10DF30003CE9FF1F00A0044018E0FF1F10F8FF1F7E
:10DF40000090044010B5164C6278204641688078F5
:10DF5000002A10D0A268002A04D0702802D1C9B2C9
:10DF6000104890472269002A16D0A078722813D151
:10DF700021790C480FE0E268002A04D0702802D111
:10DF8000C9B2094890476269002A05D0A078722872
:10DF900002D121790448904704490120087010BD3E
:10DFA00000E0FF1F08F4FF1F00F0FF1F1CE0FF1F31
:10DFB0000EB5084910300EC90192009102930C224F
:10DFC0006946FAF7CFF90006000E01D000200EBD19
:10DFD00001200EBD1C55010010B50648007B062827
:10DFE00004D0082801D102F04BFE10BD02F04DFE16
:10DFF00010BD000018E0FF1F014901208870704724
:10E0000018E0FF1F10B507480021417301228272FA
:10E01000417101F081FD002201210348FCF7C5FC9C
:10E0200010BD000018E0FF1F009004407047000082
:10E0300010B528220D490E48FAF74AF906F0EEFE0F
:10E040000C4806F0E5FE06F019FD0B4901220860B8
:10E050000A4952020A600A4A012111600949400A2C
:10E0600008600A490848086010BD0000E455010036
:10E07000D0030020D9EA0000D8EFFF1FB4EFFF1F44
:10E08000B8EFFF1FBCEFFF1FD0010020C0EFFF1F44
:10E0900000B591B0FDF79EF9402801D9402001E07C
:10E0A00000280DD081B2684605F0A4FD010007D01C
:10E0B0006846FDF7B7F9002802D0012002F00EFAF9
:10E0C00005F038FE0146402801D9402101E0002931
:10E0D0000DD06846FDF78AF9002808D081B268465D
:10E0E00005F008FE002802D0012002F0F7F902F046
:10E0F00017FA11B000BD00000448417880788142D1
:10E1000001D001207047002070470000B8E8FF1FD1
:10E1100030B50546EFF31080C407E40F72B6284609
:10E1200000F007F8A968081A401E002C00D162B65A
:10E1300030BDEFF31081CB07DB0F72B606C808388D
:10E140008A4201D3501A02E080681018401A002B4E
:10E1500000D162B67047EFF31083DB07DB0F72B6B6
:10E160008260C160002101604160002B00D162B675
:10E170007047000070B50446EFF31080C507ED0F3F
:10E1800072B603CC083C884201D0012000E0002098
:10E1900042220DA1FFF770FDE16820680E5C401C73
:10E1A0002060A16888420AD3884201D1012000E0A2
:10E1B0000020472204A1FFF75FFD00202060002D12
:10E1C00000D162B6304670BD2E5C736F75726365A8
:10E1D0005C6461706C696E6B5C636972635F6275CD
:10E1E000662E630070B50446EFF31080C507ED0F8F
:10E1F00072B66268E06881546068401C6060A16823
:10E2000088420AD3884201D1012000E00020302258
:10E2100009A1FFF731FD0020606003CC884201D0E6
:10E22000012000E00020352203A1FFF725FD002D8D
:10E2300000D162B670BD00002E5C736F75726365AD
:10E240005C6461706C696E6B5C636972635F62755C
:10E25000662E6300F8B514460E460746FFF769FFC1
:10E26000844200D220460546002404E03846FFF7E9
:10E2700081FF3055641CAC42F8D32846F8BDF8B590
:10E2800014460E460746FFF743FF844200D220465D
:10E290000546002404E0315D3846FFF7A3FF641C07
:10E2A000AC42F8D32846F8BD10B50C4880682B2244
:10E2B0000002C0170AA1401CFFF7DEFC124901242E
:10E2C0006402084622461038FFF745FF0F492246F0
:10E2D00008461038FFF73FFF10BD00000050054012
:10E2E0002E5C736F757263655C6869635F68616CEF
:10E2F0005C667265657363616C655C6B6C32377A02
:10E300005C756172742E6300E8110020F813002020
:10E3100010B500F03BFD10BD10B500F037FD10BD8D
:10E3200002488079002800D001207047FC100020AE
:10E330000248C079002800D001207047FC1000205E
:10E340000248407A002800D001207047FC100020CD
:10E350000248007A002800D001207047FC100020FD
:10E36000F8B58E212748FAF76DF98E272648FAF777
:10E370006DF9244C254E244D4034B04213D16879B8
:10E380002A79010211438E2901D20A4600E08E2229
:10E390008E2901D90F4600E08E271B491948FAF74C
:10E3A000A9F80020E0718E211748FAF74BF91649B9
:10E3B0003046FAF719F82F71390A6971114941226B
:10E3C000C91DE81DFAF796F8607A227A01020E4814
:10E3D000114340300172090A4172A17A8172E17AD7
:10E3E000C1728A0007490C304C31FAF783F80548AE
:10E3F00005498030027B80310A73407B487300F00E
:10E40000C9F8F8BD6D100020005F0020646C766BC9
:10E4100010B5094CE17A102901D3002010BD064A3D
:10E420008900403A89184C31F9F7DEFFE07A401C48
:10E43000C0B2E07210BD0000405F002010B5412165
:10E440000448FAF7FFF8034800213930017241729D
:10E45000C17210BD075F0020FFB581B01D46164692
:10E460000F461A48F9F7D4FF441C0198002802D03F
:10E470003946FAF7E7F80020002E00D03080002D52
:10E4800000D028701149C91FC87900281BD0BC4290
:10E4900001D8224602E0E01B41183A460B4C019895
:10E4A000C91D3934002804D0607A237A0002184349
:10E4B0003080002E02D00198FAF71CF8002D01D010
:10E4C000A07A2870012005B0F0BD0000075F002091
:10E4D0000148007B70470000805F00200549CA7A30
:10E4E000002A04D00A460C320260C87A7047002025
:10E4F00070470000405F002002488079002800D06B
:10E5000001207047005F00200248407B002800D0B7
:10E5100001207047805F0020F3B581B00746F9F70E
:10E5200077FF124D441C41263146E81DFAF78AF860
:10E53000412C02D83946224602E0413CE1193246DC
:10E54000E81DF9F7D7FF094C029840342072000A01
:10E55000607200F020F9002801D0012004E000F0F2
:10E560001CF9002800D00220A072FEBD005F002030
:10E570000149087370470000805F002001498871DD
:10E5800070470000005F0020014948737047000099
:10E59000805F002070B5002211461046FCF776F827
:10E5A0000A2220492048F9F7A5FF204C227810467E
:10E5B000627812021043A278E1781204104309062F
:10E5C0001B4D0843A8420FD160792179000208430E
:10E5D0000A2804D26079217902020A4300E00A2263
:10E5E00012491148F9F786FF0F492846F9F7FCFE52
:10E5F0000D490A2088802078014660780002014396
:10E60000A07800040143E07800060143A94205D147
:10E6100060792179000208430A2802D2024802F0F8
:10E6200061FC70BDF45A0100FC10002000FC0100E8
:10E63000646C766B10B503498871084602F052FC91
:10E6400010BD0000FC10002010B50349C871084639
:10E6500002F048FC10BD0000FC10002010B503497A
:10E660004872084602F03EFC10BD0000FC1000207D
:10E6700010B503490872084602F034FC10BD0000D2
:10E68000FC100020F8B50024E4430F4606460025A0
:10E6900012E0705D082103F049F8000644400A4981
:10E6A0000820002C02DA64004C4000E06400401EA8
:10E6B0000006000EF5D16D1CBD42EADB202120468C
:10E6C00003F034F8C043F8BDB71DC104F8B50E46D9
:10E6D00017462021C04303F029F80446002512E024
:10E6E000705D082103F022F8000644400A49082022
:10E6F000002C02DA64004C4000E06400401E00067A
:10E70000000EF5D16D1CBD42EADB2021204603F04E
:10E710000DF8C043F8BD0000B71DC10470B5144624
:10E720000D460646FF2A07D8FF22DE320AA1002046
:10E73000FFF7A2FA022070BD00F0ACFD002801D066
:10E74000102070BD2A462146304600F06DFF00289B
:10E75000F7D0202070BD00002E5C736F757263656A
:10E760005C6461706C696E6B5C647261672D6E2DA8
:10E7700064726F705C6961705F666C6173685F6919
:10E780006E74662E63000000C1060007000F0029AA
:10E7900000DB09307047002070470120704710B53A
:10E7A00000231A4600F02AFB002800D0012010BDEB
:10E7B00010B506F06DF8012800D0002010BD000053
:10E7C000F8B5164E012530780024ED03012806D057
:10E7D000FF22383212A10020FFF74EFA0AE0B0788B
:10E7E0000227002808D0FF223E320DA10020FFF7AB
:10E7F00043FA37700220F8BD204600F029F80028BF
:10E8000002D037702220F8BD012080022418AC42CB
:10E81000F2D30120B0700020F8BD00008CE8FF1F8B
:10E820002E5C736F757263655C6461706C696E6B8E
:10E830005C647261672D6E2D64726F705C696170CB
:10E840005F666C6173685F696E74662E63000000BA
:10E85000F8B5254E05463078012805D0FF2223A1C2
:10E860000020FFF709FA1AE00127BF0239462846BF
:10E87000F9F7FDFE0224002902D0FF22083209E048
:10E88000F07800280DD0F168B0684018A84208D090
:10E89000FF220F3215A10020FFF7EEF9347002209D
:10E8A000F8BD01227F20D20380020121954203D3CB
:10E8B000854201D2002000E00846002810D0F17007
:10E8C000F7602846B56001F0A5FD262803D0002892
:10E8D000E6D03470F8BD284600F0DCFC0028F9D002
:10E8E00034702120F8BD00008CE8FF1F2E5C736F90
:10E8F000757263655C6461706C696E6B5C64726197
:10E90000672D6E2D64726F705C6961705F666C61FB
:10E9100073685F696E74662E6300000001208002D8
:10E920007047000070B5084D04460146074B284665
:10E93000EA68FBF771F8002805D100232146284634
:10E94000EA68FBF791F970BD181100206B66656BE2
:10E9500010B5282804D2064980000858002805D19F
:10E96000F02204A10020FFF787F908A010BD0000E5
:10E97000205A01002E5C736F757263655C64617070
:10E980006C696E6B5C6572726F722E6300000000C2
:10E9900001460120282901D20148405C704700004F
:10E9A000E8E8FF1FF3B581B00446009000E0641C66
:10E9B0002078402802D00028F9D164E060786228ED
:10E9C00048D012DC522854D008DC422842D04428D7
:10E9D00049D0482841D04D2817D134E054283FD0A1
:10E9E000552833D0562810D140E0722841D006DC9B
:10E9F000642838D0682830D06D2806D123E07428E8
:10EA00002ED0752822D0762830D020A52046F9F7C0
:10EA1000FFFC07462846F9F7FBFC0646A019029BB7
:10EA2000009AC119D218891E91422BD2BA1EA11C7C
:10EA3000F9F7C4FD324629462046F9F75BFD2078F8
:10EA40000028B5D11FE001F0CDFB01E001F0D2FBC1
:10EA50000546DBE701F074FBFAE701F0A1FBF7E7FD
:10EA600001F0C4FBF4E701F097FBF1E701F0CAFB0A
:10EA7000EEE70848807A002802D0064D0A35C5E73F
:10EA800005A5C3E7E4190098201AFEBD4552524F70
:10EA9000520000005C55010068747470733A2F2FA7
:10EAA0006D6265642E6F72672F6465766963652F8A
:10EAB0003F636F64653D40553F76657273696F6E65
:10EAC0003D40563F7461726765745F69643D4054B0
:10EAD0000000000070470000F8B51E4615460C46C1
:10EAE000074606F0B1FA2C480178032912D00146F6
:10EAF0002039022C0FD0002C1FD0012C0AD10A681B
:10EB0000AA4207D18078002833D00020421E086036
:10EB10008A608861F8BD0868A842FBD1304605F0DC
:10EB200085FF0446304605F087FF0646384603F069
:10EB30009FFD03462246314617E0384603F098FD14
:10EB40000328E7D0304605F06FFF8007E2D438464F
:10EB500003F08EFD0746304605F068FF0446304658
:10EB600005F06AFF01463B462246284604F0FAFEBD
:10EB7000F8BD0948282209492038F9F7A9FB04F013
:10EB8000A7FB07488178012903D14178022900D1E8
:10EB9000817004F0A7FBF8BDF0030020E4550100EC
:10EBA000B8E8FF1FF7B51C4E0446B078550217466B
:10EBB00000280BD12946019803F01CFD032802D040
:10EBC000214604F07FFEB078002812D01249203987
:10EBD0004868A0420DD8C868A0420BD0A04208D90E
:10EBE0000869401C00D10C610869A04200D20446AB
:10EBF0000C61FEBDC8692A468018C861E019C8606A
:10EC0000F078002803D0002004F0FAFEFEBD204674
:10EC1000019904F0FDFDFEBDF0030020F0B585B0C4
:10EC200018A1096804910378002104AA545C9C424D
:10EC300026D0491C0329F9D313A10A688E68964689
:10EC40004A68CD6800239446C25C714664466F46AC
:10EC5000039552C711466139192911D9202A01D2C9
:10EC6000052A0DD100216C46675C974208D0491CEB
:10EC70001029F9D35B1C0B2BE6D3012005B0F0BDA6
:10EC80000020FBE7E5002000222A2B2C2E2F3A3B08
:10EC90003C3D3E3F5B5C5D7C10B50448F9F7D6FC1B
:10ECA000002801D0012010BD0020FCE74C550100D8
:10ECB00070B50446204600F01AF80546002D00D035
:10ECC00070BD044902480968884700BFF8E70000A2
:10ECD0000C3000F0C0ECFF1F0168012292021143CA
:10ECE0000160BFF36F8FBFF34F8F704770470028ED
:10ECF00007D0C069002802D00068022803D06D2028
:10ED00007047042070470020704710B5002806D0D7
:10ED10005B1E194201D11A4203D0652010BD0420A8
:10ED200010BD03688B4204D84068891818188842BF
:10ED300001D2662010BD002010BD000003498842AA
:10ED400001D06B2070470020704700006B66656B38
:10ED500010B50C4C70212170FFF7C9FF002807D1B6
:10ED600009492046096888472078810601D567202F
:10ED700010BDC10601D5682010BDC007FCD06920B8
:10ED800010BD000000000240BCECFF1F70B50E4D2E
:10ED900000202C78002C0FD000212970A9780029A0
:10EDA00001D000F0F7FB022C05D06978032902D0CE
:10EDB000002800D1252070BDFF226F3203A1002062
:10EDC000FEF75AFF022070BD5CE8FF1F2E5C736FD8
:10EDD000757263655C6461706C696E6B5C647261B2
:10EDE000672D6E2D64726F705C666C6173685F6412
:10EDF00065636F6465722E6300000000FEB51C46FB
:10EE00000546302901D3012000E00020472217A148
:10EE1000FEF732FF29460C2220316846F9F76AFBDB
:10EE20001E4E002C01D1002030711D4901988842EE
:10EE30000BD11C490098884201D10220FEBD19491E
:10EE4000FC3988420FD10120FEBD284605F0BAFCEE
:10EE5000002804D0002C04D10120307101E0002CE6
:10EE600001D00320FEBD0020FEBD00002E5C736FAC
:10EE7000757263655C6461706C696E6B5C64726111
:10EE8000672D6E2D64726F705C666C6173685F6471
:10EE900065636F6465722E63000000005CE8FF1F0D
:10EEA0000B9996978F9E939BFFB581B006460024E1
:10EEB00004982546002813D00A98002810D00499F9
:10EEC000002008600A9907460860FFF764FC0028E4
:10EED00012D00120C003022E06D0032E04D03FE042
:10EEE000712253E0074618E003990029FAD00299ED
:10EEF0008142F7D01B2434E0FFF74FFC00282FD0CD
:10EF0000012E02D0032E0AD02AE00398002804D054
:10EF10000298002801D01A2423E01F4819E01F4856
:10EF2000F9F794FB00281BD005460C3506E028466F
:10EF30000830F9F78BFB01280DD014352846F9F776
:10EF400085FB0028F3D1281DF9F780FB0028EED1BE
:10EF50001348056805E02846F9F778FB0746F7E708
:10EF60001C24FFF7E5F9002801D1012E04D0002C64
:10EF700004D0204605B0F0BD1C24FAE7002D04D0D3
:10EF8000049807600A980560F3E7B82205A10020FD
:10EF9000FEF772FE0220EDE7E05501004C5501003E
:10EFA000F05A01002E5C736F757263655C6461706A
:10EFB0006C696E6B5C647261672D6E2D64726F702C
:10EFC0005C666C6173685F6465636F6465722E6311
:10EFD00000000000F7B51E490646487800250128C4
:10EFE00004D0022805D0032830D105E00125ED0327
:10EFF00026E07F25AD0223E00879002826D01548B9
:10F00000F9F724FB002821D004460C340CE0B74269
:10F0100009D8201DF9F71AFBB04204D3201DF9F7D7
:10F0200015FB05460AE014342046F9F70FFB0700EC
:10F03000EDD1201DF9F70AFB0028E8D1002D05D0FD
:10F0400002983018A84201D30120FEBD0020FEBD69
:10F050005CE8FF1F4C55010010B50D4C20780028CE
:10F0600006D0DD220BA10020FEF706FE022010BD17
:10F07000FF2230211348F9F7AEF90120207000205B
:10F080006070A060E0602061A070E07010BD0000C2
:10F090005CE8FF1F2E5C736F757263655C64617062
:10F0A0006C696E6B5C647261672D6E2D64726F703B
:10F0B0005C666C6173685F6465636F6465722E6320
:10F0C0000000000054F9FF1FF8B516460F4604462D
:10F0D0000025FFF762FB002817D0032C15D10C4840
:10F0E000F9F7B4FA002810D031463846FEF760FF31
:10F0F00000280AD0074C1D2520680068804720683A
:10F10000006980472068406880472846F8BD0000B5
:10F110004C550100F05A0100F7B506464F4884B03F
:10F1200001781546012907D0F2224DA10020FEF7F3
:10F13000A3FD022007B0F0BDC178002903D1C6604D
:10F1400001210661C17045480327807800286FD1EE
:10F15000424A11698E4201D1012000E000203F4A5D
:10F160004919116100282AD0114688683022141AE2
:10F17000AC4200D92C46464A059910182246F9F7A8
:10F18000B9F93648354980682D1B00198860059902
:10F19000361909190591302839D3304C0DD000208B
:10F1A000FF2215322EA1FEF767FD01233848E268E1
:10F1B000A168FFF723FE607003E00120F0E7274815
:10F1C000477001A8254C009002AB01226078E168ED
:10F1D000FFF76AFE002826D1FFF7B2F8002806D014
:10F1E0002B496078A268FFF76FFF00281BD1A07839
:10F1F00001214840FF22383219A1FEF73DFD019858
:10F2000000F058F900280ED10120A07003E0134847
:10F210008078002816D0114C1D49A268E06800F0E3
:10F22000A7F8002801D0277084E7A078002809D02B
:10F230002A463046059900F09BF8002802D007497D
:10F240000F7077E72A4630460599FFF7C3FE00287E
:10F25000EAD002480221017013206BE75CE8FF1F2F
:10F260002E5C736F757263655C6461706C696E6B44
:10F270005C647261672D6E2D64726F705C666C6188
:10F2800073685F6465636F6465722E6300000000DD
:10F2900054F9FF1F10B5EFF31081CC07E40F72B6DD
:10F2A000FAF79CFB002C00D162B610BDFEB5214FD1
:10F2B00005467E787C68AE4238D0002E17D02046B6
:10F2C0003830F9F7C3F9800701D5002D11D1201D81
:10F2D000F9F7BCF901460020009001900346029026
:10F2E00020463246183003F02DFA00280BD0002DAE
:10F2F0001BD020463830F9F7A9F9800705D5787872
:10F30000002802D011E00C20FEBD2046F9F79EF93E
:10F310000021019102910B460146009520461830CC
:10F32000FA6803F00FFA002802D07D700020FEBDBD
:10F330000B20FEBD58E9FF1F70B50E4605001446B0
:10F3400013D020211046F9F77FF92660E868606045
:10F35000A9686868F9F78BF9A0600420E060206173
:10F360006061A061E061002070BD042070BD0000FC
:10F37000F7B5424E04467078002582B01746012842
:10F3800007D07B223EA10020FEF776FC022005B0CC
:10F39000F0BDF07800280AD1204602F0DDFF05001C
:10F3A00002D00220707066E00120F0707461334872
:10F3B000816820460091F9F75AF93048661A009999
:10F3C00040690090F9F753F90098401A864208D036
:10F3D000204600F0EBF9050003D0284902204870D0
:10F3E00049E02648016920460091F9F740F9234891
:10F3F000661A009940690090F9F739F90098401AA7
:10F40000864204D0204602F0A7FF0500E5D11B4E3E
:10F41000B16870684018A04204D8204600F0C6F9D0
:10F420000500DAD1002F24D03169F0684018A042DD
:10F4300004D8204602F090FF0500CED10F4948685D
:10F440008968201A0E1AB74200D23E461849324641
:10F4500008180399F9F74EF8002E08D00020074944
:10F46000A419887003988019BF1B0390CFE701206F
:10F47000F5E702484461284689E7000070E8FF1F6D
:10F480002E5C736F757263655C6461706C696E6B22
:10F490005C647261672D6E2D64726F705C666C6166
:10F4A00073685F6D616E616765722E6300000000B6
:10F4B00084F9FF1F70B5244D04466878002801D0F8
:10F4C00047222FE0002C2CD06068002829D0A068AB
:10F4D000002826D0E068002823D02069002820D00A
:10F4E000606900281DD0A06900281AD0E0690028B2
:10F4F00017D00121FF2289021448F8F76CFF01267A
:10F50000AE700020E8706860A860E8602861AC61B7
:10F51000686120688047040009D12878002807D056
:10F5200010E04D220AA10020FEF7A6FB022070BDCC
:10F53000A86900698047040004D0A8694068804732
:10F54000204670BD6E70FBE770E8FF1F84F9FF1F57
:10F550002E5C736F757263655C6461706C696E6B51
:10F560005C647261672D6E2D64726F705C666C6195
:10F5700073685F6D616E616765722E6300000000E5
:10F5800010B50446FFF700F80148047010BD0000F4
:10F5900070E8FF1F70B5164C00256078002802D077
:10F5A000012807D00AE0CC2212A10020FEF764FB5C
:10F5B000022070BD002000F0F9F80546A0694068FF
:10F5C000804706460121FF2289021648F8F703FF0B
:10F5D00001200021A070E1706160A160E160216103
:10F5E00061616170002E01D0304670BD284670BD4B
:10F5F00070E8FF1F2E5C736F757263655C646170E9
:10F600006C696E6B5C647261672D6E2D64726F70D5
:10F610005C666C6173685F6D616E616765722E63B5
:10F620000000000084F9FF1F10B5EFF31083DC0722
:10F63000E40F72B6FBF7DAF9002C00D162B610BD08
:10F640008021017001780906FCD5704770470000E1
:10F6500008B50A4801780322114301700849486837
:10F6600092059043104348606846FAF783FB0120F7
:10F67000694648700348FAF7D9FB08BD00400640C8
:10F680000080044000F0054010B506220721024822
:10F69000FBF775F910BD000000C0044030B504460A
:10F6A00087B0334D0C20F9F7C5FA4008A84207D3BC
:10F6B0000C20F9F7BFFA000AA84201D8012000E0A7
:10F6C00000203F222BA1FEF7D7FA34488021344B8B
:10F6D000FF2C05D34269FE240A434261416040E0A9
:10F6E000002C39D0FFF7D0FF012069460090487107
:10F6F0000871032088710020087307210291694670
:10F7000048738873C8734874887408740875C8741B
:10F710000C20F9F78FFA40002946F8F7A8FF401CA3
:10F7200045082A4662437F211046F8F7A0FF401C97
:10F730004008291A0902FF39401E01390143069188
:10F740006A4600211748FAF7A8FB17490868022201
:10F750001043086007B030BD426901240A4342618A
:10F760008160012207211846FBF709F9BCE7000078
:10F77000127A00002E5C736F757263655C626F6154
:10F7800072645C6D6963726F62697476325C666C18
:10F790006578696F5F70776D2E630000C0F00F4071
:10F7A00000C0044000F0054000F4054070B50E4D67
:10F7B0000646A8780024002808D1A8690B49836868
:10F7C000AA686868984704460120A870FF22074885
:10F7D000A968F8F700FE3046A968F8F748FF701AE4
:10F7E0006860204670BD000070E8FF1F84F9FF1FAD
:10F7F00010B50748F8F72AFF002805D0FF309D30E4
:10F80000F8F724FF002801D101480C3810BD000092
:10F810004C55010010B50948F8F718FF002806D02C
:10F82000FF30A130417802780802104305D1034827
:10F830001038C17882780802104310BD4C55010081
:10F84000034601220149002018470000F803002068
:10F85000F8B505461248F8F7F9FE04460C34114F86
:10F8600010E0AE420DD8201DF8F7F0FEA84208D3F4
:10F870002046F8F7EBFEF86020461030F8F7E6FE79
:10F88000F8BD14342046F8F7E1FE0600E9D1201D4A
:10F89000F8F7DCFE0028E4D1BC68002CE8D1F8BD04
:10F8A0004C55010058E9FF1F0146414341437F2069
:10F8B000000210B508180249F8F7D9FEC0B210BD11
:10F8C00001FE000002480069C006C017401C7047D6
:10F8D000C0F00F400020704708B51748816B1F2209
:10F8E00052021143816315490020086008600860D6
:10F8F000881513490861002000F034F8002000F05A
:10F9000027F8002000F038F80E48426901210A4328
:10F91000426142690A43426142690A4342610948BD
:10F920008030416910229143416107480090401E98
:10F930000090FCD108BD00000080044000A00440FD
:10F9400000C0044040F00F4040420F0070470000EC
:10F9500001220349012801D08A6070474A6070473C
:10F9600040F00F4001220349012801D08A6070470E
:10F970004A60704740F00F4001220349012801D03E
:10F980008A6070474A60704740F00F4070B5264863
:10F990000068C0698047002835D1244C0025607B71
:10F9A0000126002811D1FFF78DFF002802D1207811
:10F9B000002807D0012003F0D9FE6673A5822570C8
:10F9C000092022E0607B00281DD0FFF77BFF002884
:10F9D0000DD0607B002816D0FFF774FF002812D0EE
:10F9E000A08A02210A2812D9502810D311E002203F
:10F9F00003F0BCFE6573A672A08A07210A2801D90C
:10FA0000502801D2617170BD0620607170BD6171B6
:10FA100007E0782801D20321F9E7042161717828F1
:10FA2000F4D8401CA08270BDF05A010018E0FF1FFE
:10FA3000092800D927303030C0B2704730B50B48A4
:10FA4000017E8023194301760948416BDC02214382
:10FA5000416308490A7D02252A430A750A781A4338
:10FA60000A7041682143416030BD000000400640FB
:10FA700000800440402107401CB501AA69460A489D
:10FA8000F9F776FF002807D00198402805DD3222DB
:10FA900006A10020FEF7F0F81CBD402200200099CE
:10FAA00004F000FD1CBD0000E82700202E5C736FF1
:10FAB000757263655C7573625C6869645C757362BA
:10FAC000645F757365725F6869642E63000000008F
:10FAD00002460020064B702905D0712902D07229F8
:10FAE00003D001207047DA6070475A617047000008
:10FAF00000E0FF1F02460020064B702905D0712947
:10FB000002D0722903D0012070479A6070471A61B1
:10FB10007047000000E0FF1F10B58121C9000248B6
:10FB2000F8F792FD10BD000000F0FF1F10B502486D
:10FB3000FAF752FB012010BD0070064070B5812419
:10FB40008B18E400A34208D80023044C03E0C55CF2
:10FB5000CE18A5555B1C9342F9D370BD00F0FF1F72
:10FB60007FB5204801680124C214114301601E4D75
:10FB7000022221462846FAF70DFF022211462846A6
:10FB8000FAF708FF6846FAF737FB02206946087261
:10FB9000702088807220C8808C700020F9F74AF8A5
:10FBA000124C024669462046FAF758FB104A116883
:10FBB000FF20000281430025116024210D48F8F741
:10FBC00043FD0D4B0D4A0B492046FAF7BFFB21229E
:10FBD00008492046FAF702FD06480570012004B0E6
:10FBE00070BD00003880044000B004400070064042
:10FBF00008E400E010F8FF1F02E0FF1F45FC0000D2
:10FC000010B50178132905D14078072802D105499C
:10FC100005204871FFF780FF002201210248FAF712
:10FC2000C4FE10BD18E0FF1F0090044010B5FFF7A0
:10FC300073FF002201210248FAF7B7FE10BD000051
:10FC400000900440F8B50C4609781D4D00200129AC
:10FC50000BD08122D200022910D00126194F04298D
:10FC600011D020291AD02870F8BD6060A0601078EB
:10FC700015494008A87003200870F8BD1349616059
:10FC8000A2606870F8BD8121C9000E48F8F7DCFC5D
:10FC900067608120C000A0606E70F8BD2E700646BF
:10FCA0006060A060206968606878002802D03878B9
:10FCB000002801D000F02AFC05480670F8BD0000BD
:10FCC00000E0FF1F08F4FF1F1BE0FF1F00F0FF1FF5
:10FCD0001CE0FF1FF0B585B0002101910291039156
:10FCE000017801255B4C2022122966D006DC002910
:10FCF00074D010290AD0112904D15AE0132922D036
:10FD0000202920D069460A71322050E011216B462B
:10FD1000197141785971417802200B00FDF7FAFE04
:10FD20000895050C141D233E44956A469071494878
:10FD3000817CD171C07C0EE069460D8088710878A5
:10FD4000C8714878087269E0FF216A461180907195
:10FD50001078D0715078107260E001F0D5F92074FD
:10FD600069468D711EE001F017FA7D21C9004843F4
:10FD7000009001F0EBF97D21C90048430490082070
:10FD80006946887101AC042204A9E01CF8F7B2FBB3
:10FD900004226946E01DF8F7ADFB3FE069462E48B6
:10FDA0008D710078C87139E069460A713620487152
:10FDB00034E069460A713320F9E747781321352684
:10FDC0003B00FDF7A7FE0B420707070707070C1DBF
:10FDD0004237420069460A713720E8E728E0837815
:10FDE000012B09D1C378082B03D069460A7138204A
:10FDF000DDE7082222730DE06846027146710DE0CE
:10FE00008378012BF8D1C278002A01D0A57201E0D5
:10FE10000022A2726A461171407850710B220021B3
:10FE200001A8FFF78BFE012211460C48FAF7BDFD31
:10FE300005B0F0BD8378012BDED1C278002A01D055
:10FE4000E572E7E70022E272E4E769460A713420CE
:10FE5000ADE7000018E0FF1F3CE9FF1F00900440E1
:10FE6000F0B5044685B00020049060780D4601048A
:10FE7000A07800020143E078014381208002081845
:10FE80000290201DF8F7E2FB00BA019020460830EE
:10FE90000090FFF741FE8B4F2278394620260F3124
:10FEA000700303911300FDF735FE0DE75089B5CCC3
:10FEB000E1FDFBFAE71C0822E700019808308542C3
:10FEC00031D1009A0199029801F0E2F80028F7D1A7
:10FED000082200212046FFF731FE0821019A0298EE
:10FEE0008FE0019A0299891881421CD8F0E7617865
:10FEF000A278090412021143E278A3791143812206
:10FF000092028D1861791B0209041943E3791943A0
:10FF10008F18294639438905D2D1BD42E5D885429B
:10FF200001D2874207D3A7E02846FEF7FBFC0490E6
:10FF3000012080022D180498BD4202D80028F3D079
:10FF40009AE0002805D10122B5E0012D02D00C2D48
:10FF500009D091E0012200212046FFF7EFFD0B229E
:10FF60000121381D4DE0601CFEF758FE002829D005
:10FF7000661C142254496846F8F7AAF90025083689
:10FF8000A9006846415803223046F8F7EBF90028EB
:10FF90000ED06D1C052DF3D30822611C381DF8F717
:10FFA000A9FA4848032249A10C30F8F791F9D1E7A2
:10FFB0000B22611C381DF8F79DFACBE7012D02D00A
:10FFC000052D04D058E00846F8F740FB0FE0601C10
:10FFD000F8F73CFB00BA000A2179000208437F21B0
:10FFE00089020090884247D80399F8F7FDF900BAD2
:10FFF0000090012200212046FFF7A0FD04220121EC
:020000040001F9
:100000006846FFF79BFD012211463148FAF7CDFC07
:1000100005B0F0BD2B4813300090012D02D0022D09
:1000200009D029E0012200212046FFF787FD0122A7
:1000300011460098E5E76078002800D00120F874A8
:10004000F0E701256D04142229461E48F8F78AF9C5
:10005000002800D177E72846FEF764FC00280BD182
:10006000184A1421284601F013F86CE701204004D7
:10007000FEF758FC002801D0267064E711491548A6
:10008000F8F7B2F90B2214A1381DF8F721F93F2037
:10009000C0020399F8F7A8F90020F87453E70DE0BF
:1000A00004E0FFE77F206070022204E0042060701B
:1000B0000020A070032200212046A2E70949012068
:1000C000887340E718E8FF1F2855010042494E0099
:1000D00000900440646C766B444154412020202001
:1000E00042494E0018E0FF1F10B50F49002008607C
:1000F0000E4908600E4908600E4908600E49FEF777
:10010000C1FA0949086001200C49C003FEF7BAFA98
:100110000649086001217F2089028002FEF7B2FAB9
:100120000449086010BD000014E9FF1F18E9FF1F13
:100130001CE9FF1F20E9FF1FFC7F0000FC7B010082
:100140000048704724E9FF1F01200021096A054A81
:10015000914200D000200021496A034A914200D018
:1001600000207047939D939B0B99969700B5FFF7DE
:10017000EBFF002800D100BD0020806AFBE70000F3
:10018000014800687047000014E9FF1F014800683B
:100190007047000018E9FF1F00487047001000205A
:1001A00000487047BE0F00200120C103096A064ABB
:1001B000914200D000200121C903496A034A9142BB
:1001C00000D00020704700008F9E939B0B9996975C
:1001D00000B5FFF7E9FF002800D100BD0120C003F2
:1001E000806AFAE700487047B10F00200048704766
:1001F000DF0F002000487047800F00200048704744
:1002000009100020004870472EE9FF1F10B5FFF7C6
:100210006BFF054801F00EFA01F0D6FF02F058F925
:1002200002F02AF910BD0000600F002010B5134C39
:100230002078002806D0622211A10020FDF71CFDC5
:10024000022010BD002211461046FAF71FFA0028BE
:1002500001D01E2010BD00206070A070E070A06072
:10026000E0602071206160610121A0618902104875
:10027000F8F7E8F901202070002010BD8CE8FF1F7E
:100280002E5C736F757263655C6461706C696E6B14
:100290005C647261672D6E2D64726F705C69617051
:1002A0005F666C6173685F696E74662E6300000040
:1002B00084FDFF1F10B50024FFF7ACFA0D4A0E4B6A
:1002C0001168002914D10AE00988002905D081426B
:1002D00003D1A0001858106006E0641CE4B2A1002D
:1002E00059580029F0D11068002801D10348106046
:1002F00010BD0000F0EEFF1FF4EEFF1FD060010004
:1003000030B5002305E0DD000C46EC40C4545B1C16
:10031000DBB29342F7D330BDF7B504462F48012531
:100320000078ED0382B01746012808D0FF227A3208
:100330002BA10020FDF7A0FC022005B0F0BDAC42CF
:1003400001D32320F9E7FEF728FA002844D02E1B1A
:10035000301FB84201D93A4600E0321F1F480399C6
:100360008069FEF7B3F91D49886100900120800281
:10037000844207D226483A4600190399F8F7BAF89A
:100380000020DAE7E019A84226D103988519281F32
:10039000F8F75CF90102203DE87F090A00060143F5
:1003A00000980E4D884201D02720C6E739462046E6
:1003B000039AFFF739F9002801D02020BDE7012278
:1003C000920213490020FEF7A9F90446FFF78CFEBC
:1003D000012068702046B0E72620AEE78CE8FF1FBA
:1003E0002E5C736F757263655C6461706C696E6BB3
:1003F0005C647261672D6E2D64726F705C696170F0
:100400005F666C6173685F696E74662E63000000DE
:1004100084FDFF1F70B50546104801240078E403F1
:10042000012807D0FF22BC320DA10020FDF724FCDB
:10043000022070BDA54201D3232070BDFEF7ADF9A7
:10044000002801D0002D01D0262070BDFF22002001
:1004500001322146FEF762F970BD00008CE8FF1FF3
:100460002E5C736F757263655C6461706C696E6B32
:100470005C647261672D6E2D64726F705C6961706F
:100480005F666C6173685F696E74662E630000005E
:1004900002468800064910B540188038C06F002811
:1004A00004D0114601F03CFC01F02AFC10BD000014
:1004B0006422002001200749C003886001F05AFE31
:1004C00000F0D4F900221146034800F021FA00F0B0
:1004D000D3F9FEE700ED00E05D05010002490122CD
:1004E0004A7008717047000034E9FF1F0249012279
:1004F0000A70C8707047000034E9FF1F02490122EA
:100500008A7048717047000034E9FF1F10B5034836
:100510000821006900F0D0F910BD000034E9FF1F88
:1005200010B503480121C902006900F0C5F910BDEA
:1005300034E9FF1F10B503481021006900F0BCF931
:1005400010BD000034E9FF1F10B503480421006905
:1005500000F0B2F910BD000034E9FF1F1CB5012006
:100560000746064616250090FDF7FAFEFDF75EFDEC
:1005700000F0C6F99A4C2061FFF7AEF90098FFF73A
:10058000F1F93846FFF7E4F93046FFF7F5F9F9F7E6
:1005900069F994484178027808021043012800D094
:1005A0000020FF2290A1FDF767FB8E486A30F8F724
:1005B0004DF8002800D08047FFF77CFE9348006884
:1005C000002803D0C068002800D0804785480C3040
:1005D0000190F8F73BF8800702D5012002F006FBF6
:1005E0000198F8F733F8C00702D00120FEF7C8FFE2
:1005F000FFF70CFE03F0FAFFFDF76AFF00285AD060
:10060000002004F03DFB002003F00AFF74480121A4
:1006100001720B20002301901A467D4800F0A0F9DA
:10062000032100F0A5F90022D2430021794800F00F
:1006300057F984B2A00508D569488079002802D00E
:10064000012000F001F9FBF77DFE600702D50220D2
:1006500003F08CF8E00613D5032003F087F80020A0
:10066000FFF774F9002003F0DBFE0020FFF77AF9B2
:100670000020FFF76DF90020FFF77EF9FDF7ACFCD5
:10068000A00602D5032003F071F8200501D5FDF77F
:10069000FFFC200701D5FDF755FCE00742D05A20AA
:1006A00004F01CFB4E48007A0300FDF733FA062FD6
:1006B0000F2F1C3B063B0120A3E74949002008728D
:1006C000FFF744F9002003F0ABFE2BE0019800286F
:1006D00002D0401E019025D1012003F0A1FE404828
:1006E000032101721DE003F093FE002803D00120D6
:1006F000FFF72CF90EE0002D01D06D1E12D1012064
:10070000FFF724F90020364908720BE003F080FE61
:10071000002801D00220F6E73149002008720B20A2
:1007200001901625A00700D47DE7FFF72FF9FDF70C
:1007300023FB2B4C207800280BD0E078012825D013
:10074000022823D001200090002020700098FFF79D
:1007500009F9A07800280AD06079012825D002285C
:1007600023D001260020A0703046FFF705F96078FD
:100770000028D9D02079012824D0022822D00127AE
:10078000002060703846FFF7E3F84CE70099012934
:1007900001D0012100E0002100910029D6D00128DC
:1007A000D4D100202070E070D0E7012E01D00126C6
:1007B00000E00026002ED7D00128D5D10020A0705F
:1007C0006071D1E7012F01D0012700E00027002F41
:1007D000D8D00128D6D1002060702071D2E7000067
:1007E00034E9FF1F3C5501002E5C736F7572636521
:1007F0005C6461706C696E6B5C696E746572666175
:1008000063655C6D61696E2E63000000F0EEFF1F92
:10081000E53701003F0A0000014988717047000078
:1008200034E9FF1F10B5FEF717FC10BD10B5FF210E
:1008300004460231F7F706FF00F08CFF002020701D
:10084000FEF70AFC10BD000080B5034F80B2BC4625
:1008500000DF002080BD00009918010080B5024F24
:10086000BC4600DF80BD000071200100014900206E
:1008700008607047C8EEFF1F0020704780B5034F27
:1008800089B2BC4600DF002080BD0000251C0100AD
:1008900080B5044F0248BC4600DF014880BD00001F
:1008A000202600206D1B010080B5024FBC4600DFF2
:1008B000002080BD7D1B0100B0B50C460146EFF362
:1008C0000380C00603D0A0B2FFF7E2FD03E0034FB0
:1008D000A0B2BC4600DF2046B0BD0000FD180100FC
:1008E00080B5054F91B280B20022BC4600DF034FB5
:1008F000BC4600DF80BD000059190100A5180100A9
:1009000080B5024FBC4600DF80BD000065210100BC
:10091000F8B50E4C06462068002500280CD00023B0
:100920000B4F1A460B213046BC4600DF05462068B7
:10093000401C20602846F8BDF7F70CFC074F054A1D
:1009400005493046BC4600DFF1E70000C8EEFF1F56
:10095000E9200100782200200A200300FD1E01008A
:100960000146024A0020516070470000C8EEFF1F98
:1009700080B50548084F81600023044A04490548B2
:10098000BC4600DF002080BDC8EEFF1F9825002078
:100990000B8800007D200100E9200100012805D01E
:1009A000022805D003280BD0C72202E0BB2200E0BA
:1009B000BF2204A10020FDF75FF9FAF72BFCFEE748
:1009C000C322F6E72E5C736F757263655C72746F99
:1009D000735C5254585F436F6E6669672E63000004
:1009E000FEE7000007480168074841610021816176
:1009F000072101610548016AFF22120611430162C5
:100A000040177047B460010000E000E000ED00E036
:100A100070477047FFB583B0054604980E9C2818B0
:100A200000900020924F2060F878924E00281BD052
:100A30000020F870701E0278011D0698F7F75AFD25
:100A4000701E0078069941180691216808182060E8
:100A5000F8683278010C70780904000210430143F1
:100A6000701E00780818F860E6E028780A2829D077
:100A70000D28FCD03A281CD03978002973D0FDF716
:100A800083FE02077B497878491E0B5C120F1A43DC
:100A90000A54401CC0B2787009780291491D8842FE
:100AA00044D3744A0021521E137808465B1D9C46AD
:100AB0000EE070482521401EF7F7C4FD0020387075
:100AC0007870B870B7E0135C5918401CC9B2C0B256
:100AD0008445F8D8002901D00426B3E0B87800286E
:100AE00024D10120B870707831780002084340BAF0
:100AF0003070010A717001905E48401EC078042871
:100B00006CD006DC002812D001284AD002280DD172
:100B100049E00A2802D00D2808D108E05548401EB7
:100B2000417900790902014348BAB8807EE0514911
:100B30002522491E8818F7F7DDFCB888002807D061
:100B40004D49098888427CD34C490988884278D825
:100B5000F868019A010C09041143814204D0012074
:100B6000F87002266EE057E04249029AC91C0698C6
:100B7000F7F7C0FC3F480699401E007841180691DF
:100B8000216808182060F86871783278000C090232
:100B90000004114308433749491E09784018F8609A
:100BA00044E001264EE021680C98FF22411A069885
:100BB000F7F711FC2068F968091A0D980160009890
:100BC000411B0498411A059801602A48401E01798A
:100BD0004079090300010143F9601AE021680C988B
:100BE000FF22411A0698F7F7F6FB2068F968091A00
:100BF0000D9801600098411B0498411A0598016006
:100C00001C48401E417902790802104340BA000492
:100C1000F860022007B0F0BD7978252926D2FDF7CB
:100C2000B3FD144900017A78491E885438780028A9
:100C30001CD0002038706D1C0098854201D014E74C
:100C4000FFE7002621680C98FF22411A0698F7F763
:100C5000C2FB2068F968091A0D9801600098411BD1
:100C60000498411A059801603046D3E70120E1E776
:100C7000A8E8FF1F850100202CE8FF1F2AE0FF1FC6
:100C800010B5082000F006F810BD10B5062000F0E1
:100C900001F810BDF8B504463C48C078601E0A282B
:100CA00072D23B4841684902FCD503F009F8394F3C
:100CB000002212213846F9F783FE0022132138461C
:100CC000F9F77EFE002211463348F9F779FE334DDD
:100CD0000026AE616E61082C09D100220121284650
:100CE000F9F76EFE002202212846F9F769FE0A2272
:100CF00004212B48F9F738FE022C12D0052C10D015
:100D0000062C0ED0032C0CD002220E212548F9F718
:100D10003FFD022208212348F9F73AFD0720FCF79E
:100D200023FF012069464870062C02D0082C0FD101
:100D300005E0F9F785FE1548F9F7BCFE06E00E70F0
:100D4000F9F77EFE69461148F9F784FEF9F76EFE61
:100D5000FF200330A86114484021416042690A43E2
:100D60004261FF2004306861032212213846F9F7FE
:100D700027FE032213213846F9F722FE02F0F2FE85
:100D8000FEF7D4FEFEF7ECFEF8BD000000E00740E1
:100D9000005005400090044000A0044000B0044012
:100DA00000C0044000C00740800000F810B5194C96
:100DB000012204212046F9F703FE17492A20087072
:100DC00016480278417808021043C00704D014483E
:100DD0008178082211438170124948680122120665
:100DE0001043486008684000400808600B22042156
:100DF0002046F9F7B9FD03210720FCF7D9FE0720AB
:100E0000FCF7B2FE03211F20FCF7D2FE1F20FCF7E7
:100E1000ABFE10BD00B0044000E0074000F007400A
:100E200000D007400070044038B500F0FDF901F033
:100E3000A3F9FFF7BBFF00F0C1F900F065F91F4C03
:100E40002074FEF705FCFEF71FFC207C022833D03F
:100E5000FF202072C0B2FEF727FDFEF71FFCFEF751
:100E60007FFE70211648FEF745FE70211548FEF7FB
:100E70002FFE72211448FEF73DFE72211348FEF743
:100E800027FE134800224068009001211148F9F71D
:100E90008CFD6A4601211048F9F748F8012040040A
:100EA0000446F7F7D3FB0D4A904204D114222146A1
:100EB0000B48F7F71FFB38BD6420CAE718E0FF1F97
:100EC000D5FC000001FC000061FE00002DFC0000CC
:100ED0000C5501000090044000F00F40646C766BEC
:100EE00018E8FF1F70B5134D0646EFF31080C407D6
:100EF000E40F72B62846F8F771FD002C00D162B6F7
:100F0000002816D1FF2210210B48F7F764FA0A22B5
:100F100031460948F7F7EEFAEFF31080C407E40F03
:100F200072B6054A10212846F9F760FD002C00D161
:100F300062B670BD00FC010008110020F7B5044640
:100F4000012084B0C003434F029038781646012830
:100F500005D0A22240A10020FCF78EFE41E0FF2137
:100F600001318800009001912046F7F780FB0225AF
:100F7000002901D0AB222FE00198864205D301461B
:100F80003046F7F774FB002901D0B22224E0204656
:100F90000099F7F76CFB00988919814201D9B922B1
:100FA0001AE0B87800280DD1F878002808D0B96880
:100FB0008C4203D3F8680818A04203D8C7220BE07C
:100FC000C12209E03979384600290DD07A6939699A
:100FD0008918A14208D0CF221FA10020FCF74CFEA7
:100FE0003D70022007B0F0BD7F218902A7198C4215
:100FF00005D20121C9038F4201D9002100E001215E
:10100000002910D013480121017146610461324664
:1010100020460599FFF780F9262807D00028E1D05F
:101020000C490D70DEE705702020DBE731462046D5
:10103000059AFEF7F9FA002801D00648F3E702986E
:10104000874204D3FFF750F802490120487000207E
:10105000C8E700008CE8FF1F2E5C736F7572636534
:101060005C6461706C696E6B5C647261672D6E2D7F
:1010700064726F705C6961705F666C6173685F69F0
:101080006E74662E63000000FF2001307047000080
:10109000FEB50C460B460646014615460748F8F7CE
:1010A0009DFD002809D101210190009102902B465D
:1010B000224631460148F8F71BFEFEBD18110020FC
:1010C000EFF31082D207D20F72B603680B400360B1
:1010D000002A00D162B67047EFF31082D207D20F18
:1010E00072B603680B430360002A00D162B67047F2
:1010F000EFF31082D207D20F72B603684B40036041
:10110000002A00D162B6704770B50E48002400690D
:10111000C006C617761C00F019F8054600F03CF82A
:101120000949002E05D08D4201D2012407E0032495
:1011300005E08D4203D3C835854200D902242046FC
:1011400070BD000080F00F40DC05000070B5104C51
:10115000012203212046F8F71DFF0E48401EFDD155
:10116000002209211046FCF7C7FD05460022032195
:101170002046F8F70FFF0B204543002000F03CF815
:1011800001467D20C0006843F7F771FA70BD00008A
:1011900080F00F4080BB000010B500221D211046DA
:1011A000FCF7AAFD0446002000F026F801467D2049
:1011B000C0006043F7F75BFA10BD000008B50A48AD
:1011C00000680090FCF77AFD6A4603210748F8F7AB
:1011D000ADFE012203210648F9F7FDFB00220121A3
:1011E0000448F9F7F8FB08BDB855010080F00F403E
:1011F00000B0044000A00440F8B5094C0646207831
:10120000002807D1012569460D7048700548F9F797
:101210006DFB257000221B213046FCF76DFDF8BDEB
:101220002EE8FF1F00D00740F8B52448244F00687F
:101230000090002206213846F9F7B7FBB869402430
:10124000A0432043B8611F4E6A4606213046F8F796
:101250006DFEFCF733FDB460012206213846F9F734
:10126000A4FB194D2C46641EFDD14020706019204E
:101270008001401EFDD1002206213846F9F795FB7A
:10128000012207210020FCF737FD1049484310498F
:10129000F7F7EDF904464020B060012206213846F8
:1012A000F9F783FB6D1EFDD10A48FF3C0E3C8442DA
:1012B00001D20120F8BD0020F8BD00000C5501004E
:1012C00000C00440C0F00F4080BB0000E40C0000F0
:1012D000FF0F00009A02000070B514460E46054646
:1012E0000019012140028902884206D90B4A0CA14B
:1012F0000020FCF7C1FC002070BD012149023046EE
:10130000F7F7A0F9002D06D11048114900694201F4
:101310003046F7F7EFF8600270BD0000630200008E
:101320002E5C736F757263655C6461706C696E6B63
:101330005C647261672D6E2D64726F705C76697289
:101340007475616C5F66732E63000000D0E8FF1F48
:10135000600B002010B5012464020B46002801D068
:10136000002010BD224603491846F7F7C3F820466F
:1013700010BD0000A0080020F8B50C4600210E4664
:101380000091002801D00020F8BD314800780128E4
:1013900042D0022842D0002720462EA103F0CEF9E9
:1013A000054660192EA103F0C9F9451960192E49A7
:1013B00003F0C4F9451960192CA103F0BFF94519D0
:1013C00060192BA103F0BAF9214945196019498820
:1013D00003F0BDF94519601924A103F0AFF94519CF
:1013E000002F0ED0601924A103F0A8F94519601947
:1013F000394603F0A3F9451960191CA103F09EF9C1
:1014000045196846FDF76AF807001FD000980028C4
:101410001CD060191BA10EE01DA7BDE71FA7BBE7ED
:10142000B0000099761C0958F6B2601903F060F913
:10143000451960190DA103F081F94519BE4205D285
:10144000284601210A3049028842E9D32846F8BDDE
:10145000C8E8FF1F4173736572740D0A0000000035
:1014600046696C653A2000005C0600200D0A000009
:101470004C696E653A200000536F757263653A20BF
:101480000000000048657864756D70730D0A0000F7
:10149000426F6F746C6F6164657200004170706CB4
:1014A00069636174696F6E000B464102812080029E
:1014B000091810B5012080044412814203D222464B
:1014C0001846F7F717F8204610BD000070B50D4616
:1014D0000646012801D9002070BD992189000948DC
:1014E00002F06AFC0446700206490122231A5202E5
:1014F0004118934200D81A462846F6F7FBFF2046CB
:1015000070BD0000F8030020F8B50D46044603F056
:10151000DDFB0646FDF71CFA07463046FDF738FAB4
:101520000646002C01D00020F8BD28461B4903F0D8
:1015300005F904462819394603F000F90419281959
:1015400017A103F0FBF8154904192819C91F03F066
:10155000F5F8041900270120009014E000980028F5
:1015600004D128190FA103F0E9F80419F00708D0F5
:101570000D49B8000958281903F0E0F804190020B3
:10158000009076087F1C002E01D0052FE6D3281985
:1015900003A103F0D3F80019F8BD000013560100B1
:1015A0000D0A00002C2000009C57010070B50C466D
:1015B000002801D0002070BD01256D02294620467B
:1015C000F7F740F80648F6F723FF0246044920469D
:1015D000F6F790FF29462046FDF7E4F970BD0000BC
:1015E0001B560100F8B5094D06460F462846F6F78A
:1015F0000FFF0446002E01D00020F8BD0246294608
:101600003846F6F777FF2046F8BD00005C6301001E
:1016100010B5012464020B46002801D0002010BD43
:10162000224603491846F6F765FF204610BD000024
:10163000A006002004490A6A0260CA6942608969FA
:1016400081600021C16070474080044010B50846A9
:1016500054022146F6F7F6FF204610BD70B5234D23
:1016600000246878A978E443884201D0012000E092
:101670000020FF22FA321EA1FCF7FEFA6878022849
:1016800004D0002816D0012818D020E02348FF24D9
:101690000078F53400281AD0012809D0022816D085
:1016A000032814D01E4A12A10020FCF7E5FA0EE030
:1016B0001C4C0CE0A878022808D008E0A878022882
:1016C00002D0002802D002E0174C00E00024601C89
:1016D00005D1134A06A11032FCF7CEFA0024A868FF
:1016E000A04201D9012070BD002070BDB8E8FF1FE5
:1016F0002E5C736F757263655C6461706C696E6B90
:101700005C647261672D6E2D64726F705C766673B7
:101710005F6D616E616765722E630000F0030020EB
:101720000B020000204E0000C409000070B5034603
:1017300000200246012509E0DC0704D08E1A2C4661
:10174000761EB44020435B08521CD2B28A42F3D3C7
:1017500070BD000010B525210848F6F773FF074853
:1017600025212530F6F76EFF05480021C160017084
:1017700041708170C170818010BD00008401002023
:10178000A8E8FF1F0146EFF31080C207D20F72B620
:101790000868002801D003680B60002A00D162B6F7
:1017A0007047000070B50D4600280FD00849094C5D
:1017B000884204D222680146104600F0D1FA20681F
:1017C0004570054800F0FBF800F090FB70BD00008C
:1017D000FFFF0000DCEEFF1F2C26002070470000FA
:1017E00070B51B4EF068002831D0B08A401EB08220
:1017F000002526E0A068002808D061684160606884
:10180000002802D0A16881606560A560104821466B
:10181000183800F0CDFAA08AB0826078042804D18C
:101820000C49E08A09884018A082012060702021BC
:101830000855E068F060E068002801D00661E560C6
:101840002561B08A002802D1F468002CD2D170BD85
:1018500044260020E4EEFF1F70B504000ED00C4DAE
:10186000A17828680126827891420BD900F0BEFA4F
:1018700028684670204600F039FB70BD054800F02E
:101880009EF8F8E766702146024800F091FA70BDB4
:10189000DCEEFF1F2C26002010B50321FFF782FF8E
:1018A00010BD000001480068408B7047DCEEFF1F50
:1018B00010B50446008B084320836278618B062AAA
:1018C00015D0052A12D1084210D00A460240628380
:1018D00088432083204600F0ABFA0120607002218B
:1018E000202001552146044800F062FA10BD0A4646
:1018F0008243EDD010BD00002C2600200246880057
:1019000070B5144940188038C46F002C1DD0208B4E
:10191000104320836178658B062917D0052914D1DF
:10192000284212D0294601406183A84320832046E3
:1019300000F07EFA208B0221A843208301206070F2
:10194000202001552046FFF787FF70BD29468143BF
:10195000EBD070BD6422002070B503460D480D46E3
:101960000468002A208B08D01946814301D0062143
:1019700009E098432083022070BD0146194001D040
:101980006183F6E7052163832846FFF70BFF0120FB
:1019900070BD0000DCEEFF1F814202D342688A4224
:1019A00001D801207047EFF31082D207D20F72B630
:1019B00003680B60016000D162B6002070470146E9
:1019C0004068002342684A600A78022A05D0012A4A
:1019D00003D0032A01D0436070474268002A01D037
:1019E000916043608360704770B5044615460020DF
:1019F000207001226270A1706060A060E0602061D0
:101A0000A082E082208323466083203318705870C0
:101A1000608C002803D10448FFF7B4FEA062294679
:101A2000204600F005F870BDA82100207047000096
:101A300030B5428C920803D10E4A12881204920CDF
:101A4000836A92009B185A0700D51B1F01221206B9
:101A5000403BDA630022996314469500521C5C51A6
:101A60000E2AFAD3C2691A624362C162806A0249CD
:101A7000016030BDB0600100A52E5AE20349044A5E
:101A80000968C8821288801888827047DCEEFF1FC0
:101A9000E4EEFF1F10B50848016808488A8A0088EC
:101AA000CB8A101AD21880B28A82010402D404218F
:101AB000FFF778FE10BD0000DCEEFF1FE4EEFF1F15
:101AC000F8B50446406800260F46002805D0607827
:101AD000022818D0A08900282FD0A089E189884247
:101AE0003ED2208980000019076172B6A089401C8F
:101AF000A08162B62089401C80B22081E1898842A1
:101B000000D12681F8BD66702046FFF758FF0546D4
:101B1000203006702189E86989000919086172B6C8
:101B2000A089401CA08162B62089401C80B220811F
:101B3000E18988420AD1268108E02046FFF73FFF6D
:101B40000546C069042107602020415501206870C6
:101B5000284600F06DF92946034800F029F9F8BD40
:101B60000320FEF71BFFF8BD2C2600200321017087
:101B7000002141704180416081607047F8B50446A2
:101B80004088002804D0254EA1683268914201D0D7
:101B9000FF20F8BD401E0004000C60803CD131687D
:101BA0006078887061680127002928D02046FFF7F7
:101BB00006FF0546052120300170284600F038F95F
:101BC0006780A560A87860701548316840688A7899
:101BD0008078824201D328460AE0114800F0E8F8F4
:101BE00029460F4800F0E4F8306847706F7011E044
:101BF000FFF732FE31680020203108700CE0084900
:101C000049688A783168824206D9054800F0D0F8E0
:101C1000306847700020EBE70020F8BDDCEEFF1FC6
:101C20002C26002070B50E46184D044641882868C1
:101C3000002907D0A168814208D16088401C6080DB
:101C4000002070BDA06080786070F6E7002E0FD095
:101C500062788078824203D28870A06800F0D0F861
:101C60006068002806D02046296800F0A1F808E046
:101C7000012070BD286860602968002048602868DD
:101C8000846009213046FFF78DFDF1E7DCEEFF1F90
:101C900070B51848012102685170006800F0A6F87C
:101CA000154D6C7813E0E000411948680278002A6D
:101CB00017D0012A1AD000F0EBF8E878641C8442AF
:101CC00000D1002472B6A878401EA87062B6A87829
:101CD0000028E8D16C700948FFF771FE00F006F9A2
:101CE00070BD098989B2FFF7E3FDE6E78968FFF770
:101CF000E7FEE2E7DCEEFF1F402200202C2600205A
:101D000005480178002902D0012141707047012067
:101D10000249000748607047D4EEFF1F00ED00E065
:101D2000F8B50E4EF778B41C354672B6B278BA42A2
:101D300007D2521C22702A78531CBB4200D10023C8
:101D40002B7062B6F378934204D9D2009219916055
:101D50005060F8BD0220FEF721FEF8BD40220020B1
:101D600010B5124AD368002B17D013469B8A04E0A3
:101D7000002C12D02246A48AE318D4688B42F7D3F1
:101D8000C460D0600261C468002C00D02061591A80
:101D90008182908A401A908210BD0024C460D06075
:101DA000C91A02619182848210BD0000442600207D
:101DB00030B502780023022A03D0012A01D0032A79
:101DC00000D101238C7800E010464268002A02D03E
:101DD0009578A542F8D24A604160002B04D0002AD1
:101DE00000D09160886030BD0020FBE703494A685D
:101DF0004260002282604860704700002C2600206C
:101E000010B583680446002B05D1607801280CD1F9
:101E1000064B03E09B6818780028FBD0204600F0B2
:101E20001DF821461846FFF7C3FF10BD2C260020E1
:101E300010B5016900290FD0C268CA60C3680022CA
:101E4000002B07D08B8A848A1B198B82C368196187
:101E5000C26000E08A82026110BD00008168002932
:101E600007D042684A604168002901D080688860D4
:101E70007047064906E04A68824202D140684860DD
:101E8000704711460029F6D1704700002C2600202B
:101E900010B5416800290ED0FFF791FD0446FFF709
:101EA000C7FF01206070032120200155214604480E
:101EB000FFF77EFF10BD4188491C418010BD000026
:101EC0002C26002010B507480068416A806A8142CC
:101ED00003D300680449884202D00120FEF75EFD6A
:101EE00010BD0000DCEEFF1FA52E5AE2024948603B
:101EF0000221417070470000DCEEFF1FF7B5154668
:101F0000394A002004463749128802E08300CC5049
:101F1000401C9042FAD33548302201883448FBF700
:101F200069FE344801210088C90780B2421832484E
:101F300001683248FBF75EFE3148082201883148CB
:101F40000068FBF757FE304FFF26FE707C842F4A57
:101F500000213846FFF748FD2D48042101704460F8
:101F60002C480170C46004618482786A2030F6F7DE
:101F7000EBF829482A490760022078702748047046
:101F800044700978C170FFF751FD2648016A320498
:101F900011430162C169026A5202920E9206114314
:101FA000C161FEF71FFD20490028086012DB82088E
:101FB0001E49920051180A688307DB0E9E40324387
:101FC0000A60C206D20E012191404011184A8000D9
:101FD0008018016000232A460199009800F084F8D7
:101FE000FEBD000064220020AE600100C46001005C
:101FF000DC200020B0600100C8600100A8210020A2
:10200000CE600100C4EEFF1F5C260020E109010044
:102010002C26002044260020DCEEFF1F402200205A
:10202000CC60010000ED00E0D8EEFF1F00E400E00E
:1020300000E100E010B50B48012102685170006812
:10204000FFF7D4FEFFF7CAFB07480168491C01608F
:10205000FFF7C6FB00F028F80448FFF7B0FCFFF7D5
:1020600045FF10BDDCEEFF1FE4EEFF1F2C26002015
:102070000148006870470000E4EEFF1F074C084F5E
:102080002089BC4680B200DF064FBC4600DF616895
:102090000029F9D000208847F6E70000C8EEFF1FAE
:1020A0007D1A0100951A010070B50D4D28680028B1
:1020B00015D0A8880B4E401EA8800AE0E088FEF7E5
:1020C000A8FCA088A8802068286021463068FFF717
:1020D00063FCA888002802D12C68002CEED170BDCA
:1020E000E8EEFF1FC4EEFF1FFFB5080681B01E46D5
:1020F00017460C46000E00D14C1C1648FFF742FB59
:10210000051E25D02002000CAF626884EE61E1B2AA
:102110002846019AFFF768FC104801240E490288FE
:1021200006E0A00040188038C06F002803D0641C6F
:102130009442F6D90024A00040188038C567EC709E
:102140002846FFF789FB06480068203004702046C7
:1021500005B0F0BDDC20002064220020AE6001004C
:10216000DCEEFF1F02480068002800D0C0787047EE
:10217000DCEEFF1F7047000070B50446FF22A53259
:102180000B490C48F6F7B6F90B4E0C490C480D4DAF
:10219000002C01D0012C04D08068F6F725F96E825E
:1021A00070BDC068F6F720F90348401C688270BD16
:1021B00018EBFF1F74E9FF1F0399000010EBFF1FCE
:1021C0000C55010018E0FF1FF8B500250024FDF7AD
:1021D00021FB064605215748F6F736FA21215648D5
:1021E000F6F730FA21215548F6F72CFA0921544820
:1021F000F6F72AFA05214F48F6F726FA00BF00BF86
:102200000AE0504BAA0099584B4A101902F070FA94
:102210000019C4B2681CC5B2042DF2DB00222046AE
:10222000611CCCB244490A54002400250AE0464B04
:10223000AA009958414A101902F05AFA0019C4B27A
:10224000681CC5B2042DF2DB00222146601CC4B21A
:102250003A48425400243A4908193C49096802F0B6
:1022600047FA0019C4B22046611CCCB2344900229E
:102270000A54FDF7BDFA0746042239462D48F6F701
:1022800039F92C490020087100243104080FFDF7AA
:10229000CFFB014622462E48641C81543105080FAD
:1022A000FDF7C6FB014622462948641C8154FCF711
:1022B0000FF9012803D0FCF7EFFC00280CD13111F5
:1022C000082211430807000FFDF7B2FB2146621CEC
:1022D000D4B21F4A505408E03106080FFDF7A8FB9E
:1022E0002146621CD4B21A4A50543007000FFDF741
:1022F0009FFB2146621CD4B2154A5054002220464E
:10230000611CCCB212490A540024302221461148E3
:10231000641C425432222146641C42543522214618
:10232000641C42542146641C425400222146641C11
:102330004254F8BD24E9FF1FBE0F0020DF0F00202C
:1023400000100020600F0020700F002010E9FF1F18
:1023500029E9FF1F2EE9FF1FF1B5394DA869416931
:10236000009888470746A86981690098884704460D
:10237000002F07D0002C05D00126B602B74209D89D
:10238000012008E0FF2236322EA10020FBF774FC6A
:102390000220F8BD0020FF223B322AA1FBF76CFC93
:1023A00039463046F6F763F9002909D00020FF22AC
:1023B0003C3224A1FBF760FCBC4203D3012002E0C5
:1023C0000120F4E70020FF223D321EA1FBF754FC60
:1023D00039462046F6F74BF900291AD00020FF2293
:1023E0003E3218A1FBF748FC21460098F6F73FF96A
:1023F0000098401AE8602C616860B44200D334460B
:10240000AC60A969096A002905D0884704000BD18E
:1024100001E00120E3E7287800280AD0A869C16814
:10242000E8688847040004D0A869406880472046CF
:10243000F8BDFF220F48A968F5F7CDFF0020F8BDD1
:1024400070E8FF1F2E5C736F757263655C6461706A
:102450006C696E6B5C647261672D6E2D64726F7057
:102460005C666C6173685F6D616E616765722E6337
:102470000000000084F9FF1F70B50025002400262D
:102480001148F5F7C5FFC6B27000801CC2B22146E4
:102490000E48641C425403222146641C425400BF6F
:1024A0000EE00948611C425D2046CCB207490A543F
:1024B00000222046611CCCB204490A54681CC5B2F3
:1024C000B542EEDB70BD0000800F00200910002037
:1024D00010B531210948F6F7B7F809490748F5F76B
:1024E0006EFF08490548F5F76AFF07490348F5F705
:1024F00066FF06490148F5F762FF10BD800F002016
:1025000024E9FF1F29E9FF1FBE0F00200010002053
:1025100010B50A4C2078002808D000F081F86068D7
:10252000C168074888470021217010BDC02205A15D
:102530000020FBF7A1FB022010BD000030E8FF1FC8
:1025400050F8FF1F2E5C736F757263655C64617079
:102550006C696E6B5C647261672D6E2D64726F7056
:102560005C66696C655F73747265616D2E630000F3
:1025700070B5134C05462078002801D0852202E072
:10258000022D06D38B220FA10020FBF775FB022042
:1025900070BDFEF7B5F9FF21A06005311448F6F7CC
:1025A00053F801200649207028010C314018606062
:1025B00041680F4888470028EAD00321217070BD88
:1025C00030E8FF1F2E5C736F757263655C64617029
:1025D0006C696E6B5C647261672D6E2D64726F70D6
:1025E0005C66696C655F73747265616D2E63000073
:1025F00050F8FF1FF8B5094D0E460746002420018C
:102600002A58314638469047002801D02046F8BD68
:10261000641CE4B2022CF2D30320F8BD3CE8FF1F97
:1026200010B5FEF76DF906498968884201D101208D
:1026300000E00020622203A1FBF71EFB10BD00009A
:1026400030E8FF1F2E5C736F757263655C646170A8
:102650006C696E6B5C647261672D6E2D64726F7055
:102660005C66696C655F73747265616D2E630000F2
:10267000014610B5083103220C4608A0F5F7EAFE22
:10268000002807D00322214605A0F5F7E3FE002825
:1026900001D0032010BD012010BD000042494E00B2
:1026A0004845580070B5154D064628780C46012857
:1026B00006D0A42212A10020FBF7DEFA022070BD92
:1026C000FFF7AEFF6868224683683146174898478F
:1026D0000446132807D0142C07D0002C05D0032063
:1026E0002870204670BD0220FAE72878012800D023
:1026F0000020B22202A1FBF7BFFAF2E730E8FF1F89
:102700002E5C736F757263655C6461706C696E6B6F
:102710005C647261672D6E2D64726F705C66696CAB
:10272000655F73747265616D2E63000050F8FF1F62
:1027300010B51E21002000F039FD002800D0012036
:1027400010BD0000F0B593B00D4604461E46174676
:1027500044216846F5F778FF189800970290199879
:1027600003900196201DF5F771FF0990204608306F
:10277000F5F76CFF0D902046F5F768FF0E900120ED
:10278000000610900F95684600F0C6FC00281DD08A
:10279000144D002411A9144800F004FA002814D0A4
:1027A0001198800314D56946002000F04FF90028E5
:1027B0000CD00E490C4800F04FFD002806D01A98A6
:1027C0000128009808D0002809D0002013B0F0BDDF
:1027D000641CAC42DED3F8E7B9198842F5D1012078
:1027E000F4E7000040420F00F0ED00E003005FA0BE
:1027F00010B5044600F0AEFF002801D1200E0006FF
:1028000010BD000070B5F7F72DF80948402444606A
:1028100020254560074942034A60436923434361D9
:1028200043692B434361486910434861012070BDEF
:10283000800000F800F00F40F8B50020411E009025
:1028400035486426016004274160002412E0002C12
:1028500010D00121002000F0A9FC012000F0D2F9E5
:102860000220FDF7F1FF002000F0CCF90220FDF777
:10287000EBFFEAE7FFF7C6FF28480068002803D00F
:102880008068002800D08047F7F718FF00283CD068
:10289000FFF74EFF002838D00021082000F086FC0A
:1028A000002832D005210907042000F07FFC002811
:1028B0002BD000250BE06946042000F01DF900280C
:1028C00021D0052000994007884302D06D1CB542F5
:1028D000F1DBB54219D0012C17D01149042000F0CA
:1028E00065FC002811D00D480068002803D000695D
:1028F000002800D080470021082000F057FC002865
:1029000003D00120F8BD0124E3E77F1E01247FB23C
:10291000002F9CDC0020F8BD50E9FF1FF0EEFF1FE8
:10292000000F0050074841694022914341614169CD
:1029300020229143416104484169D203914341619E
:1029400001207047800000F800F00F4038B50C46B9
:102950000546FFF74DFF2A46F0210A401043014685
:10296000082000F023FC002821D02D072D0F032084
:1029700005436946284600F001FB6946284600F0F9
:10298000FDFA00216A462160D1780906216092781B
:10299000120411436A4621605278120211436A46BA
:1029A0002160127811432160012800D0002038BD39
:1029B000F8B50D460446002A2CD09608164900208A
:1029C00000F0ECFA002826D00527042221466846AC
:1029D000FDF796FC6946384600F0D0FA012819D177
:1029E0000F270021384600F0C9FA012812D100242F
:1029F000761E07E02946384600F0C0FA012809D1C2
:102A0000641C2D1DB442F5D30E20294600F0B6FA01
:102A1000012800D00020F8BD5200002338B50D4633
:102A200004460949002000F0B9FA00280BD0694695
:102A3000204600F033F8002805D0A007C10E00980A
:102A4000C8402870012038BD50000023F8B50E465C
:102A5000014600246425104800F0FEFB002810D039
:102A60000D4F3F1F3146384600F09CF8002808D033
:102A70003068C00302D4641CAC42F3DBAC4201D129
:102A80000020F8BD04483146001D00F08BF80028F6
:102A9000F7D00120F8BD0000F4ED00E01CB50C46B5
:102AA0000146042201A8FDF72BFC052001A900F036
:102AB00065FA01281ED10F20694600F05FFA01284F
:102AC00018D10E20694600F059FA00216A462160AB
:102AD000D178090621609278120411436A46216078
:102AE0005278120211436A46216012781143216024
:102AF000012800D000201CBD38B50C460C21084030
:102B00006946801C00F03AFA00216A462160D178BB
:102B1000090621609278120411436A4621605278B6
:102B2000120211436A462160127811432160012884
:102B300000D0002038BDF8B514460F46054608E021
:102B400039462846FFF76AFF002829D0641E6D1C0D
:102B50007F1C002C23D0A807F2D112E0A905012088
:102B6000890D8002461AB44201D2A608B600324648
:102B700039462846FFF71CFF002811D0AD19BF19B0
:102B8000A41B032CEAD808E039462846FFF746FF85
:102B9000002805D0641E6D1C7F1C002CF4D1012080
:102BA000F8BD000070B50C4605460749002000F04E
:102BB000F5F9002806D021462846FFF76FFF0028C8
:102BC00000D0012070BD0000520000231CB5002081
:102BD0006A46FF211154401CC0B20828FAD311469E
:102BE0003320F8F7B7FA01201CBD00000149087036
:102BF0007047000048E9FF1F014948607047000026
:102C000048E9FF1F08490968002903D0C96900295C
:102C100000D00847012212050449002801D08A602B
:102C200070474A6070470000F0EEFF1F00F00F4051
:102C3000FEB5164F164E174C051E19D0FFF7FCFDBA
:102C400069463846FFF782FE0098B04201D1012163
:102C500016E011480190042201A9104800F0C6FABC
:102C60002046F5F7F3FC010001D028468847FEBD59
:102C700069463846FFF76AFE0098B042F0D100215D
:102C80000120000600F08AF9EAE70000FC000001DC
:102C900000008802AA5501000400FA050CED00E0CE
:102CA000F8B502240546062801D0FFF7ABFD4E49D2
:102CB0004E4E4F1C2B00FAF72DFF080516095C5EDF
:102CC000758C93950120FFF79DFF89E00120FFF7A8
:102CD00099FF0220FDF7B8FD0020FFF793FF0220C7
:102CE000FDF7B2FD7AE0FFF7A7FD002879D0404D4F
:102CF000287801280BD00FE0641E64B2002C71DD2F
:102D00000120FFF77FFF0220FDF79EFD0020FFF767
:102D100079FF0220FDF798FD3946304600F09CFA15
:102D20000028E9D0314C01210C34204600F094FAFF
:102D3000002856D02878002805D10120FFF762FF2F
:102D40000220FDF781FD0020FFF75CFF0220FDF768
:102D50007BFD69463046FFF725FF002841D00098EB
:102D60008003F6D50021204600F076FA002838D0FE
:102D700036E03046F8E7F7F7A1FC002831D0FFF73E
:102D8000D7FC00282DD00021082000F00FFA0028E1
:102D900027D005210907042000F008FA002820D0D8
:102DA0003946E6E7FFF748FD00281AD00E493046BD
:102DB000C91C00F051FA002813D069463046FFF7CD
:102DC000F1FE00280DD000988003F6D508E008E059
:102DD00008E0304600F040FA002802D0FFF7A2FDDC
:102DE0000120F8BD0020F8BD00005FA0F0ED00E07C
:102DF00048E9FF1FF8B502240546062801D0FFF771
:102E000001FD5A495A4ECF1C2B00FAF783FE0805E4
:102E10002409787A93A9A6AD0120FFF7F3FE9CE080
:102E20000120FFF7EFFE0220FDF70EFD0020FFF767
:102E3000E9FE0220FDF708FD0021042000F0B6F9AC
:102E4000002876D069460420FFF756FE002870D08F
:102E5000FFF768FD81E0FFF7EFFC00287ED00FE070
:102E6000641E64B2002C7FDD0120FFF7CBFE022040
:102E7000FDF7EAFC0020FFF7C5FE0220FDF7E4FCA9
:102E80003946304600F0E8F90028E9D06946304676
:102E9000FFF788FE002861D000988003F6D5344CF7
:102EA00001210C34204600F0D7F9002856D0304DCF
:102EB0006946E43D2846FFF775FE00284ED000988D
:102EC000610D08402B4941182B48406801432846B2
:102ED00000F0C2F9002841D00220FDF7B5FC694698
:102EE0003046FFF75FFE002838D000988003F6D503
:102EF0000021204600F0B0F900282FD02DE0304608
:102F0000F8E7F7F7DBFB002828D0FFF711FC0028D3
:102F100024D00021082000F049F900281ED0052106
:102F20000907042000F042F9002817D00F49491C76
:102F3000E5E713E0FFF780FC00280FD03946304664
:102F400000F08AF9002809D069463046FFF72AFECA
:102F5000002803D000988003F6D50120F8BD03E0D7
:102F6000304600F079F971E70020F7E700005FA034
:102F7000F0ED00E00000FA0548E9FF1F70B50D46CE
:102F80000646002429463046F7F7FEFD022803D105
:102F9000641CE4B2642CF5D370BD000038B50D4656
:102FA0000446FFF725FC2246F0210A401043014663
:102FB000082000F0FBF8002806D0002C06D10E48AF
:102FC0004168A94201D1012038BD45600C20044070
:102FD000042229466846641CFDF792F9694620469A
:102FE000FFF7CCFF012805D10E200021FFF7C6FF17
:102FF0000128E9D0002038BD50E9FF1FF8B50D4683
:103000000446002A25D0960813490020FFF7C6FF82
:1030100000281FD00527042221466846FDF770F9D5
:1030200069463846FFF7AAFF012812D10D27002470
:1030300007E029463846FFF7A1FF012809D1641CA3
:103040002D1DB442F5D30E200021FFF797FF012874
:1030500000D00020F8BD00005200002370B50C46DF
:10306000054608490020FFF799FF002809D0A80766
:10307000C00E21468140284600F02EF8002800D0DE
:10308000012070BD5000002373B50646002464255E
:103090001048019900F0E0F8002815D00120000444
:1030A000314601430B48001F00F0D6F800280BD032
:1030B000084E083E01A93046FFF774FD002803D0F2
:1030C0000198C00301D501207CBD641CAC42F1DB3A
:1030D00000207CBDF8ED00E038B50C460146042226
:1030E0006846FDF70DF905206946FFF747FF0128FF
:1030F00010D1042221466846FDF702F90D206946E9
:10310000FFF73CFF012805D10E200021FFF736FF15
:10311000012800D0002038BD38B505460021082020
:1031200000F044F800283AD00024A0002958204696
:10313000FFF7AAFF002832D0641C042CF5D3092025
:10314000696AFFF7A1FF002829D00D24A0002958A3
:103150002046FFF799FF002821D0641C102CF5D3DE
:103160001020296CFFF790FF002818D00E4C0D4955
:10317000204600F071F8002811D00A492046891E27
:1031800000F06AF800280AD069460420FFF7B4FC72
:10319000002804D00098A021084201D0002038BDAA
:1031A000012038BD0B005FA0F0ED00E0F8B50E4F38
:1031B00004460E46082802D13868B04211D00C20CF
:1031C0002546054004226846FDF79AF869462846D8
:1031D000FFF7D4FE012801D00020F8BD082C00D153
:1031E0003E600120F8BD000050E9FF1FF8B514460D
:1031F0000D46064608E029783046FFF72FFF0028E5
:1032000029D0641E6D1C761C002C23D0B007F2D18F
:1032100012E0B1050120890D8002471ABC4201D29B
:10322000A708BF003A4629463046FFF7E7FE0028C8
:1032300011D0F619ED19E41B032CEAD808E029781F
:103240003046FFF70BFF002805D0641E6D1C761C6E
:10325000002CF4D10120F8BD70B50C460546074995
:103260000020FFF79BFE002806D021462846FFF7E6
:1032700033FF002800D0012070BD00005200002361
:1032800010B5FDF73DFB06494968884201D1012090
:1032900000E00020FF226A3202A1FAF7EDFC10BD27
:1032A000B8E8FF1F2E5C736F757263655C646170B4
:1032B0006C696E6B5C647261672D6E2D64726F70E9
:1032C0005C7666735F6D616E616765722E63000088
:1032D00010B503480021C068FDF7D0FA10BD00000A
:1032E000B8E8FF1F10B50248C068FDF7DDFA10BD51
:1032F000B8E8FF1F02480078012800D0002070477E
:103300008CE8FF1F02480078012800D00020704799
:1033100058E9FF1FFEB527480646F5F797F900283C
:1033200046D0002504460C3429E03846FCF790FAD4
:10333000002804D03830F5F789F940071ED420461C
:10334000F5F784F900F0B6F900282ED10120FBF73B
:10335000ADFF050029D11848476838460830F5F711
:1033600075F9014600200090019003460246029044
:1033700038461830FFF7E6F9002817D014342046F5
:10338000F5F764F90700D0D1201DF5F75FF90028A3
:10339000CBD13046F5F75AF9FF30A13080780028BC
:1033A00002D000F087F805462846FEBD1020FEBD7D
:1033B0000120FEBD4C55010058E9FF1F3EB50546F2
:1033C0001848F5F743F9002829D017484468002C1D
:1033D00009D0284600F02AF801462846F5F747F9B3
:1033E00000291AD101E002203EBD0120FBF75EFF5B
:1033F0000028F9D120460C30F5F728F901460020C5
:10340000009001900346029020462A461830FFF7AC
:1034100099F9002801D000203EBD0F203EBD0120BB
:103420003EBD00004C55010058E9FF1F70B5054630
:103430001448F5F70BF9061E18D030460830F5F79A
:1034400005F9002815D0441E13D4301DF5F7FEF8F9
:10345000E1004018F5F7FAF8A84208D8301DF5F752
:10346000F5F8E100091D4018F5F7F0F870BD641E8D
:10347000EBD5FF228D3204A10020FAF7FDFB0020DE
:1034800070BD00004C5501002E5C736F7572636552
:103490005C6461706C696E6B5C696E7465726661A8
:1034A00063655C7461726765745F666C6173682ED6
:1034B0006300000070B518480446F5F7C7F8002807
:1034C00027D0164D002068706860012000F04EF98A
:1034D000002805D02046F5F7B9F804460C340AE078
:1034E000072070BD20460830F5F7B0F8C00701D0BE
:1034F000AC600AE014342046F5F7A8F80028F1D1B2
:10350000201DF5F7A3F80028ECD101202870002039
:1035100070BD012070BD00004C55010058E9FF1F2F
:10352000F7B586B015465548F5F790F800287DD0D8
:1035300053484768002F12D052480068002808D02E
:103540004369002B05D02A46079906989847012819
:1035500008D00220FBF7AAFE002801D164E0022077
:1035600009B0F0BD0D20FBE738463430F5F76EF8B2
:10357000A84201D92C4600E0044638462430039086
:10358000F5F764F822460799FFF730FE002866D069
:103590000398F5F75BF8064638461030F5F756F80D
:1035A00000210191029101463846183023460096C9
:1035B000069A0490FFF7C6F8002817D0FAF7B8FE6D
:1035C00000282AD0384614300090F5F73FF800283C
:1035D0004FD00320FBF76AFE0028C1D138463830AF
:1035E000F5F734F8C00703D0012602E01120B7E751
:1035F00000260398F5F72AF801900098F5F726F8C9
:10360000019A002101910092014623460296069AF2
:103610000498FFF797F800281FD006980019069025
:10362000079800192D1B0790002D00E024E09BD186
:10363000002095E7102C01D2264600E010263246E5
:1036400069460698FFF777FA002808D0324669469F
:103650000798F4F787FE002803D0122080E70A209D
:103660007EE70698AD1B8019069007988019A41B69
:103670000790002CD8D0DDE7012071E74C55010000
:1036800058E9FF1FF0EEFF1F70B505460848F4F734
:10369000DDFF00280BD0FF2401342846FFF7C6FECB
:1036A000A04203D22846FFF7C1FE0446204670BD63
:1036B0004C550100F8B5FCF7CBF804001FD0124DB3
:1036C0006868A04219D00020FBF7F0FD002815D152
:1036D00020462C30F4F7BAFF074620463030F4F786
:1036E000B5FF064620462830F4F7B0FF3A4631468B
:1036F000FFF77CFD002804D06C600020F8BD092095
:10370000F8BD0820F8BD000058E9FF1F10B50F48AC
:10371000F4F79CFF002817D00020FBF7C7FD002816
:1037200011D1FAF7FDFD002801D0022000E00120B0
:1037300000F01CF8072000F019F805490020087077
:10374000FFF7F0F8002010BD012010BD4C5501001E
:1037500058E9FF1F04480068002802D0806A00284A
:1037600000D1002070470000F0EEFF1F70B5054645
:103770001648F4F76BFF010001D02846884714482B
:103780000468002C1FD0A169002902D02846884770
:1037900070BDA078012803D0022805D0012070BD9B
:1037A0002846FFF77DFA70BD0848001DF4F74EFF6C
:1037B000002802D16068002801D0FFF71DFA2846D2
:1037C000FFF718FB70BD002070BD0000AE55010072
:1037D000F0EEFF1F884203D3904201D801207047CA
:1037E0000020704770B5094C02212069FDF764F88C
:1037F000E06803210546F4F73AFF6D1CE5600029F7
:1038000003D101212069FDF757F870BD34E9FF1F8E
:10381000F8B51F4C1646E0780D46002806D00B225E
:1038200092011CA10020FAF727FAF8BDF0051FD07D
:103830000020B122920017A1FAF71EFA6078204A00
:1038400014A1FAF719FA31462846FEF72BFF012793
:10385000054613280ED0142D16D0002020710C48D8
:103860002038416989194161284600F0C9F8F8BD3E
:103870000120DEE7FEF74CFE054600206070E77091
:103880002771FAF7BFFBEAE700252771E7E7000099
:10389000F00300202E5C736F757263655C64617069
:1038A0006C696E6B5C647261672D6E2D64726F70F3
:1038B0005C7666735F6D616E616765722E63000092
:1038C000C5020000F8B51A4C074660780D4600287E
:1038D00012D00020174A18A1FAF7CEF9681C00D0C0
:1038E0000120144A14A1521CFAF7C6F9104E203ECA
:1038F0007068401C02D002E00120EBE77560E079BF
:10390000032800D1E7717068A84202D1E079B8427B
:1039100001D0032008E03846FEF72AFE002803D134
:103920000121F5606170A17000F06AF8F8BD000037
:10393000F0030020850200002E5C736F75726365D2
:103940005C6461706C696E6B5C647261672D6E2D76
:1039500064726F705C7666735F6D616E61676572CD
:103960002E63000070B5194C2578032D05D025462F
:10397000203D2E68002E06D006E0154A15A1002035
:10398000FAF77AF970BD2860A868401C00D1A960D8
:10399000E079032800D1E371A869904206D9E8696B
:1039A000904203D9002A01D003200BE0481C02D02A
:1039B000A8688842F8D1032B02D0E0799842F3D16D
:1039C0000020AA6100F01CF870BD0000F003002088
:1039D000350200002E5C736F757263655C64617004
:1039E0006C696E6B5C647261672D6E2D64726F70B2
:1039F0005C7666735F6D616E616765722E63000051
:103A0000FEB50546132803D0142D01D0012000E097
:103A100000205D22D20045A1FAF72EF94E4C207805
:103A2000032810D02246203A1168002912D0D36909
:103A3000906983420ED300280CD093685068984256
:103A400008D1012007E0BB22920038A10020FAF73C
:103A500013F9FEBD00206071A3790193002902D102
:103A6000E179032901D0012100E000210091002823
:103A700004D02179002901D0012600E00026E17858
:103A8000002903D0002801D0012000E0002002908E
:103A900010690027401C13D02F4820384068401C74
:103AA00000D001202D4A21A1FAF7E6F82A48203853
:103AB000426801694069891A4902884200D9012790
:103AC0000320002D01D020701DE0019900290AD0AB
:103AD000002F01D00625F6E700990029F3D0002E2B
:103AE000F1D10425EFE702990029ECD1002E01D095
:103AF000022003E00098002802D00120207011E08D
:103B0000207803280BD16078002806D0FEF700FD4E
:103B100000216170002D00D1054611480570019803
:103B2000002896D101F0C0F8FEBD00002E5C736F36
:103B3000757263655C6461706C696E6B5C64726104
:103B4000672D6E2D64726F705C7666735F6D616E4B
:103B5000616765722E630000F00300200A03000015
:103B6000B8E8FF1F70B50D20F9F7EEFF1D48816B17
:103B700042151143816341680322120791430122D8
:103B8000120711434160174838300168D2111143C0
:103B90000160154CA0680325AD04A843A060A0688F
:103BA000052149058843A060FAF77EFB0F48A9125A
:103BB0008160C160A0682843A060A06841214905D8
:103BC0000843A0600A490868FF22120290432A11A4
:103BD000104308600D20F9F7ABFF0D20F9F7D0FF77
:103BE000012070BD0080044000500540409004401A
:103BF0000CE400E00A4610B501460248FAF72AFB39
:103C000010BD0000E813002010B50D20F9F79CFF4F
:103C1000064881680122D20591438160FAF744FB8E
:103C20000D20F9F7ADFF012010BD00000050054048
:103C3000F8B5064600252F460D20F9F785FF1E4CE6
:103C4000A068052149058843A060A168032080047D
:103C50008143A160FAF728FB71790020012902D085
:103C6000022903D004E001252F4600E001250120B0
:103C70000001690008433843A060306801010F4823
:103C80000068F4F7F4FC2168C004490B4903C00C38
:103C900001432160A068032189040843A0600D202E
:103CA000F9F746FF0D20F9F76BFFA06801214905E0
:103CB0000843A0600120F8BD00500540CCECFF1F78
:103CC00010B50A488168032292049143816081689B
:103CD0004522520591438160FAF7E6FA04480168EB
:103CE0000122520591430160012010BD00500540A2
:103CF0003880044070B50A4601460C48FAF7BFFA0E
:103D00000546EFF31080C407E40F72B60748FAF7D0
:103D100010FA002805D0064881680122D205114317
:103D20008160002C00D162B6284670BDD8110020F9
:103D30000050054010B50248FAF7EAF910BD00003E
:103D4000D811002010B50F4C2078002807D0002093
:103D50002070F9F7DDFE002808D01F2010BD832257
:103D600009A10020F9F788FF022010BD6078002823
:103D700003D1FAF710FD002801D0002010BD252046
:103D800010BD00008CE8FF1F2E5C736F75726365B9
:103D90005C6461706C696E6B5C647261672D6E2D22
:103DA00064726F705C6961705F666C6173685F6993
:103DB0006E74662E63000000F8B50F460446F4F7F3
:103DC00041FC2046A2A100F0B9FC05466019ADA156
:103DD00000F0B4FC45196019AEA100F0AFFC451924
:103DE0006019B0A100F0AAFC4519FAF799FA002869
:103DF00001D0B0A100E0B0A1601900F09FFC45190E
:103E00006019AEA100F09AFC45196019ACA100F050
:103E100095FC4519FAF78CFA002801D0A5A100E01D
:103E2000A5A1601900F08AFC45196019A3A100F052
:103E300085FC45196019A8A100F080FC4519FAF726
:103E400087FA002801D09BA100E09BA1601900F037
:103E500075FC4519601999A100F070FC45196019AD
:103E6000A3A100F06BFC4519FAF76AFA002801D00B
:103E700090A100E090A1601900F060FC4519601964
:103E80008EA100F05BFC45196019A1A100F056FC61
:103E90004519FAF739FB002801D086A100E086A178
:103EA000601900F04BFC4519601984A100F046FC34
:103EB0004519FAF770FC002801D099A600E09BA6EE
:103EC00060199DA100F03AFC45196019314600F0D7
:103ED00035FC4519601979A100F030FC45196019CD
:103EE000314600F02BFC4519601997A100F026FC23
:103EF0004519FAF750FC002815D1FCF725F90028E0
:103F000011D0601994A100F019FC4519FCF72EF9A5
:103F100001466019042200F040FC4519601967A1B0
:103F200000F00CFC4519FAF738FC002815D1FCF715
:103F30003BF9002811D060198DA100F0FFFB451955
:103F4000FCF746F901466019042200F026FC4519E9
:103F500060195AA100F0F2FB4519601989A100F01F
:103F6000EDFB451960198AA100F0E8FB45196019BD
:103F700052A100F0E3FB4519601990A100F0DEFBAF
:103F800045196019002100F0E2FB451960194BA1A9
:103F900000F0D4FB451960198CA100F0CFFB451946
:103FA00060198FA100F0CAFB451960198DA100F0BE
:103FB000C5FB451960198DA100F0C0FB45196019BA
:103FC0008CA100F0BBFB451960193CA100F0B6FBC9
:103FD0004519FCF7B9F8002810D0601988A100F045
:103FE000ADFB4519FCF7CCF80146601900F080FBE9
:103FF0004519601931A100F0A1FB4519601985A18F
:1040000000F09CFB4519FCF7C1F80146601900F06F
:104010006FFB4519601929A100F090FB4519601943
:1040200081A100F08BFB844945196019496800F0B3
:104030008EFB4519601921A100F080FB4019201862
:104040007EA100F07BFB39462046FAF7ABFCF8BDB9
:1040500023204441504C696E6B204669726D776134
:104060007265202D207365652068747470733A2F13
:104070002F6D6265642E636F6D2F6461706C696E65
:104080006B0D0A00556E697175652049443A2040F0
:10409000550D0A004849432049443A2040440D0A3E
:1040A000000000004175746F2052657365743A20FA
:1040B0000000000031000000300000000D0A000088
:1040C0004175746F6D6174696F6E20616C6C6F7790
:1040D00065643A20000000004F766572666C6F7769
:1040E00020646574656374696F6E3A200000000097
:1040F000496E636F6D70617469626C6520696D6192
:10410000676520646574656374696F6E3A200000AA
:10411000506167652065726173696E673A200000BF
:10412000426F6F746C6F616465720000496E7465F4
:1041300072666163650000004461706C696E6B209B
:104140004D6F64653A2000002056657273696F6E8A
:104150003A2040560D0A0000426F6F746C6F616424
:1041600065722056657273696F6E3A200000000018
:10417000496E746572666163652056657273696F16
:104180006E3A2000476974205348413A20000000ED
:10419000313433366264636336373032396664668D
:1041A00063306666303362373365313230343562BE
:1041B0006236613966323732000000004C6F63614D
:1041C0006C204D6F64733A2000000000555342206C
:1041D000496E74657266616365733A200000000081
:1041E0004D5344002C204344430000002C204849F8
:1041F000440000002C205765625553420000000027
:10420000426F6F746C6F61646572204352433A2051
:1042100030780000496E74657266616365204352B0
:10422000433A20307800000052656D6F756E74203F
:10423000636F756E743A2000C8E8FF1F55524C3A00
:104240002040520D0A00000010B5064C0448606082
:10425000002060800448F5F7ABFB0120207010BD02
:104260004218002034EFFF1F8C260020F0B54BA32E
:104270000ECB9DB06D460EC5474F0024384609222F
:104280006946F4F737F90925FAF722F9464E01286D
:1042900073D0FAF701FD00286FD0747120460190A9
:1042A00001247D19182241A102A8F4F711F8172260
:1042B00002A92846F4F71EF90198A870202500F0FD
:1042C000A3F934702746641C33497470491900916E
:1042D00044223C490CA8641CF3F7FAFF42220CA9C3
:1042E0000098F4F707F90099781C8F70009942350F
:1042F0008F721F31CF7008718873F7F7ADF92649B7
:10430000347149190091671C20222FA102A8F3F7EC
:10431000DFFF202202A90098F4F7ECF8009920357D
:104320008C7000F003F9B7712FA10EC91A480392DF
:10433000401902917C1C04930090092202A9F4F711
:10434000D9F8009809358770174818220C30877300
:104350001148B470451927A102A8F3F7B9FF172235
:1043600002A92846F4F7C6F80F48AC70B6300471BD
:10437000FFF76AFF1DB0F0BDFFE730890649401E18
:10438000308108718B2088700022CA701F493A540E
:1043900008881738088094E7F81500200902A20061
:1043A0000601008096000000FCECFF1F09040000DD
:1043B00002080650080705820240000007050202B5
:1043C000400000006C6001000904000002030000CE
:1043D0000609210001000122210007058103400098
:1043E00001070501034000010904000000FF03006C
:1043F000070000000904000002FF0000090705058E
:1044000002400000070585024000000006EDFF1F86
:1044100002484078002800D001207047DCEFFF1FE1
:1044200010B5F7F753FA10BD002070477CB51C4655
:10443000154601281ED1002C01D0012C1AD101AA49
:1044400069460D48F5F794FA00280ED0019A402AE3
:1044500005DD4F2209A10020F9F70EFC0AE02846ED
:104460000099F4F747F840207CBD012C02D10C499B
:104470000120087000207CBDE82700202E5C736FAF
:10448000757263655C7573625C6869645C757362A0
:10449000645F757365725F6869642E630000000075
:1044A000A0EFFF1FF8B507461A481646008882425B
:1044B00001DD0020F8BD184800780028FAD0174C1C
:1044C0000122E26001E0002814D06288002AFAD1BB
:1044D000134D32462F70681CF4F70CF820466561C6
:1044E0000024848046800F490978012908D86D1C72
:1044F000456108E00020E0606061A0806080D8E74E
:104500004188491C41800020F7F706FD0648C45544
:104510000120F8BD745E0100DDEFFF1F7CEFFF1F7F
:1045200000170020725E0100A0EEFF1F10B50349C6
:10453000012008700248F5F73BFA10BDA0EFFF1FFD
:10454000E82700200178832902D14078002801D093
:1045500000207047012070477047000038B50124E3
:104560001D461146022814D1002D12D008780728C4
:104570000CD06B462A461148F5F7CCF9002813D029
:104580000098FFF7DFFF012804D004E00C49012068
:10459000087038BD00240B4D2878002809D0FBF79F
:1045A0006BFA0020287004E0852207A10020F9F7AB
:1045B00063FB2046FBF79AFF38BD0000E827002088
:1045C0002FE8FF1FA0EFFF1F2E5C736F75726365EE
:1045D0005C7573625C6869645C757362645F757353
:1045E00065725F6869642E630000000010B50549BC
:1045F0000020C870FFF73AFEF8F7E8FDF7F76AFF0A
:1046000010BD0000DCEFFF1F10B5FCF779F9074C77
:1046100060600020FCF73CF9E060F9F709FD00203C
:104620006070A0700249A060086010BDB8E8FF1F6C
:10463000A8EFFF1F70B514460D460646FEF720FE94
:10464000064B1868002807D00120FBF757FF2246C9
:104650002946304600F0AEFB70BD0000A8EFFF1FFA
:1046600070470000F8B515460E460746FEF708FEEF
:104670000D480068002816D00C4900200C4C8860BA
:10468000207803280FD00120FBF738FF2A46314657
:10469000384600F0ADFD2078032804D02A46314684
:1046A0003846FAF77FFAF8BDA8EFFF1FB8E8FF1FFA
:1046B000F00300200548074A01780548C180002121
:1046C00001704170C160826001617047645E0100E9
:1046D000DCEFFF1F0100010010B5EFF31080C407ED
:1046E000E40F72B6F9F7AAFE002C00D162B610BD35
:1046F00070B50D460446090E00F014F8064628026F
:10470000010EA01900F00EF886192804010EA01958
:1047100000F008F88619E9B2A01900F003F8801932
:1047200070BD00000B09044A0907D35C0370090F30
:10473000515C417002207047FE5A01000346002080
:1047400001E01A54401C0A5C002AFAD17047F3B504
:1047500081B0074600242546029805E00A21F3F7B8
:1047600086FF0021641C4D410028F7D120462843D4
:1047700001D101240025002609E00A210298F3F75F
:1047800076FFA21B3031521EB954761C02900020D5
:10479000311BA841F1D32046FEBDF8B515460E46A3
:1047A0000746FFF7D4FF0446A8420AD23022294622
:1047B0003846F3F710FE281BC0193146FFF7C7FF34
:1047C0002846F8BDF1B5304882B00068002808D00E
:1047D000016A002905D002988847002800D00120EE
:1047E000FEBD2A480190F3F731FF04004AD00020B3
:1047F0000425074600902A4668460299F3F77AFE98
:10480000D4340AE0201DF3F721FF02463146009818
:10481000FEF7E0FF012832D014342046F3F716FFEC
:104820000600EFD1201DF3F711FF0028EAD1002F79
:1048300028D024E002980026411904226846F3F7A4
:1048400059FE0198F3F702FF04460C340AE0201DDC
:10485000F3F7FCFE024639460098FEF7BBFF01283D
:104860000CD014342046F3F7F1FE0700EFD1201DE1
:10487000F3F7ECFE0028EAD1002E03D02D1D0C2DFD
:10488000D8D9ACE70020FEBDF0EEFF1F4C5501006B
:104890000C490968002903D0496A002900D008475B
:1048A00001783A290AD1007A302809D0322807D075
:1048B000332805D0342803D0352801D00020704794
:1048C00001207047F0EEFF1FFFB583B00398FAF7A1
:1048D000A5F9FF22963241A1F9F7CEF94A48019095
:1048E000417A007A090201434748C01E407B414398
:1048F00006984018401EF3F7BAFE054606980027B2
:10490000424E002819D00024681EF76800900AE083
:10491000F168481C82B23E4800F064FDF068401C1B
:10492000F0600098641C8442F2D33A4A3848F16837
:1049300000F058FDF068401CF0603069202802D378
:10494000FF22AB321FE04101334A401C8C1830611A
:10495000202232492046F3F7CDFD0B222046039951
:10496000F3F7C8FD21461C310698F3F73DFD380CDE
:104970002075000A6075A776380AE076B1681029BC
:1049800008D3FF22B93215A10020F9F775F90020EC
:1049900007B0F0BD08460C2250431F4A204BC03AD6
:1049A0001350204B87187B60049B002B00D01350C2
:1049B0000598002800D078600198491C427A037A53
:1049C0001002114A1843D21E527B50436843B8600C
:1049D000B1603078401C30702046D9E72E5C736F90
:1049E000757263655C6461706C696E6B5C64726146
:1049F000672D6E2D64726F705C7669727475616C70
:104A00005F66732E63000000A3060020D0E8FF1F3E
:104A1000A0080020FFFF0000600B0020005A0100EA
:104A20004D16010009550100C07A704710B51C30C1
:104A3000F3F70CFE10BD000010B50446FFF7F6FFBB
:104A4000002812D0E07EA17E040209480C43017BBD
:104A5000C07A0902014307484069F3F708FE044998
:104A6000A41E497B6143081810BD0020C04310BD3F
:104A7000A0060020D0E8FF1FC172704770B50F4933
:104A8000087DCA7C0402087BC97A050214430D43E1
:104A9000002C01D06C430FE008482030F3F7D6FD1E
:104AA000002802D06843044606E00024FF228A3230
:104AB00003A12046F9F7E0F8204670BDA0060020CB
:104AC0002E5C736F757263655C6461706C696E6B8C
:104AD0005C647261672D6E2D64726F705C766972B2
:104AE0007475616C5F66732E63000000F3B5012678
:104AF0000F46760281B031464D48F3F7A5FD3146A9
:104B00004C48F3F7A1FD4C4C0025C0214B48E56013
:104B1000F3F79AFD49487100C030F3F795FD256120
:104B20002570A56046486561606032464549404849
:104B3000F3F7CEFB3E4E307BF27A010201200004F7
:104B400011433818F61CF3F792FD0446F71E797BE3
:104B50003D484843A04208D9FF2257323BA10020DC
:104B6000F9F78AF87C7B38480BE043484143A1427F
:104B700008D2FF225A3235A10020F9F77DF87C7B5C
:104B80003D4844432A49012000042031844204D393
:104B90003574280A7074204603E03474200A707457
:104BA0000020F3F721FC797B2046F3F760FD3249C2
:104BB000000211394018040CFC8230222F491F4892
:104BC000F3F786FB60021D491B4C48610862042014
:104BD0006561A06000200C2242435218926863690C
:104BE000401CD21862610428F5D3234A2946673253
:104BF0001048E56000F0F6FBE1681F4A491C6E3280
:104C00000C48E16000F0EEFBE06825610B4D401CB4
:104C10001A49E060C035284620223031F3F76AFC9B
:104C200028460B220199F3F765FC01202061FEBDA7
:104C3000A0060020A0080020D0E8FF1FA00A002046
:104C4000D5EA0000B05701005A1000002E5C736FC7
:104C5000757263655C6461706C696E6B5C647261D3
:104C6000672D6E2D64726F705C7669727475616CFD
:104C70005F66732E6300000091FF0000B0590100D1
:104C800010B50446FEF724FB0649002C07D08878AF
:104C9000002801D102208870FEF724FB10BD0020FF
:104CA000F9E70000B8E8FF1F10B5FEF711FBF9F7B0
:104CB00023FA002805D104484178022901D10121B5
:104CC0008170FEF70FFB10BDB8E8FF1F10B5FEF7AF
:104CD000D7FA0148007810BDB8E8FF1FF8B50446C0
:104CE000FEF7CEFAFEF7F4FAF9F706FA002810D02C
:104CF000FCF7B4FC204A214B9168994201D2091972
:104D00009160002805D0947855785470012C05D115
:104D100002E0FEF7E7FAF8BD0220907000269660E8
:104D2000FEF7E0FA0127002D16D0012D14D0022D38
:104D300012D1134D2878032803D0AF710020FEF75D
:104D40005FFE2878032812D00020FF2212320DA126
:104D5000F8F792FF00F058F9154D002C09D0012CFE
:104D600007D0022CD7D1F9F763F92F60F8BD0120E5
:104D7000EBE72E60F8BD0000B8E8FF1F60EA000016
:104D8000F00300202E5C736F757263655C64617064
:104D90006C696E6B5C647261672D6E2D64726F70EE
:104DA0005C7666735F6D616E616765722E6300008D
:104DB000A8EFFF1FF7B582B0044615460026510242
:104DC0000398F3F73FFC002031460C2251430F4A71
:104DD0008B189B685B0AC318009384420CD39C42D7
:104DE0000AD21F1BAF4200D32F465358201A3A460F
:104DF00003999847E419ED1B002D04D0761CF6B2F8
:104E00000098102EE0D305B0F0BD0000A00A0020ED
:104E10000149486070470000D0E8FF1F1CB5314CC5
:104E2000E07F002802D020461F3000E02EA00121A4
:104E30008906FFF75BFE2F48FAF702FD0346207D47
:104E4000002802D02748143000E02BA00022294976
:104E5000FFF73AFD2B48FAF7F3FC034600222949F5
:104E600029A0FFF731FDFFF731FF002808D02948BE
:104E7000FAF7E6FC03460022264927A0FFF724FDA7
:104E8000284B41219A1C2848F9F7E6FA00280BD054
:104E90002648FAF7D5FC0346002224492448FFF7A8
:104EA00013FD0021FFF7E8FD002001900120C00361
:104EB0000090F9F772FC002810D0FF22013200990F
:104EC0000198F3F74FFA002808D11A48FAF7B8FC0E
:104ED00003460022174918A0FFF7F6FC00F032F84D
:104EE0001CBD00003C5501004441504C494E4B2034
:104EF00020202000AD1501004D42454420202020F7
:104F000048544D00CD14010044455441494C5320B0
:104F100054585400091501004641494C20202020D6
:104F200054585400C8E8FF1F5C06002079130100A4
:104F30000F570100E51501004E4545445F424C20E6
:104F40005458540010B5FFF7C1FE0146FF31F5314A
:104F500000282BD01D4A1446203CE0691154090A50
:104F6000101841701A480068FAF7A4FA002805D012
:104F70002322120117A10020F8F77EFE134900201A
:104F8000A269FAF7F5F9002806D0FAF703FB1B4AE5
:104F900010A10020F8F770FEFAF7FCFA002805D0FF
:104FA000164A0CA1521D0020F8F766FE1448F3F7CC
:104FB0004DFB034612480F38C17C002904D0002263
:104FC0001049001DFFF780FC10BD000038E0FF1FF6
:104FD000F05A01002E5C736F757263655C626F61DD
:104FE00072645C6D6963726F62697476325C6D695C
:104FF00063726F62697476322E63000036020000BD
:1050000027E8FF1FA914010010B5F9F7C4FB002819
:1050100005D0FFF75BFE002801D1F6F7FBF8F9F7A2
:10502000BCFB002809D0F9F767FA002803D1F9F78B
:105030004FFA012801D1F6F7EDF802484168491C02
:10504000416010BDC8E8FF1FF8B50C46074600F0E8
:10505000ADF8002855D1FAF73DFC002803D1FAF746
:1050600031FC002800D00120002803D1F9F760F9B5
:10507000002846D0022C44D0002C0BD0012C40D16B
:105080000B223E493846F3F76DF9002839D1FFF776
:1050900023FB70E0012069460870851E384600F049
:1050A00087F8002863D1354E00240D36E0003158D2
:1050B0000B223846F3F756F9002800D12546641C28
:1050C000102CF3D3681C0024002818D02B00F8F70C
:1050D00021FD1009114E1924262A2C303236383C75
:1050E0003E424448F9F759FB002840D00120F9F727
:1050F00045FA3CE0F62222A10020F8F7BDFD684603
:105100000470F8BD284C206800688047206800695A
:10511000804720684068804729E0012000E00020A7
:10512000F9F788FA23E0012000E00020F9F78CFA73
:105130001DE0012000E00020F9F79AFA17E00020B6
:1051400000E00120F9F714FA11E0012000E000204E
:10515000F9F784FA0BE0012000E00020F9F714FAD7
:1051600005E0FF22253206A10020F8F785FD6846FC
:1051700000780028C5D0FFF797FDF8BD0F57010054
:105180002E5C736F757263655C6461706C696E6BC5
:105190005C647261672D6E2D64726F705C766673ED
:1051A0005F757365722E6300F05A0100002070472E
:1051B00010B50B2209A1F3F7D5F800280BD10A4846
:1051C00081684068F3F753FA02460121074B49040E
:1051D0000548F4F721FC002010BD00004552415362
:1051E0004520202041435400181100206B66656B58
:1051F000F7B50446002682B0154630461CE00C2167
:1052000032464A430F4952189168490A41180091A1
:1052100084420CD38C420AD20F1BAF4200D32F46DC
:105220005368201A3A4603999847E419ED1B002D5C
:1052300006D0761C0098F6B2034989688E42DED308
:1052400005B0F0BDA00A0020D0E8FF1FF7B5054665
:1052500004462035287C84B01646302801D3606B84
:1052600032E030210F1AB74200D3174600193A46F0
:105270000599F3F73FF9287CC019C1B22974302988
:1052800002D2002007B0F0BD05980023C019059098
:10529000F61B1A462046F9F7B1FD00281FD002A9D7
:1052A0000022009101AB1146F9F7FEFD0028E9D17B
:1052B000019860632A7C2146F9F72EFF0028E1D18E
:1052C000297C606B4018606332460599F9F724FF2A
:1052D0000028D7D1606B801960631420D2E71C20AE
:1052E000D0E70000F7B58118012349029B0288B07E
:1052F000994207D99F2292002DA10020F8F7BCFC0B
:105300000BB0F0BD41024B095102049149090691CD
:1053100032495A01511802910391099901910028CB
:1053200001D000263BE0012639E0019970014418C4
:10533000039900904518202221462846F3F712F8D9
:1053400000282BD0214628460B22F3F70BF8002823
:1053500011D00020224F05907F6823462A46204620
:105360000221B84701990098085CE52805D0059806
:10537000002807D012E00120ECE72A462346104619
:10538000012108E02046F9F749FC002806D0234611
:105390002A4618460021124C6468A047761C0698DD
:1053A0008642C2D3049A09990298F3F7A3F8A7E7B3
:1053B0002E5C736F757263655C6461706C696E6B93
:1053C0005C647261672D6E2D64726F705C766972B9
:1053D0007475616C5F66732E63000000600B0020C3
:1053E000D0E8FF1F10B54B000124591C6402A142F4
:1053F00006D3FF223A3204A10020F8F73DFC10BD8D
:10540000C254120A425410BD2E5C736F75726365EC
:105410005C6461706C696E6B5C647261672D6E2D8B
:1054200064726F705C7669727475616C5F66732EFE
:1054300063000000F0B587B0002416460F4605460D
:10544000039404940594FF2004AA03A90130029256
:10545000019100906B1C05AA31463846FBF7DAFA39
:1054600000280DD0022814D001281FD0042829D0EC
:10547000052801D00628E6D1052825D0012024E002
:10548000049A002A27D0691C0398F9F745FE0446C0
:1054900021E0049A002A05D0691C0398F9F73CFE24
:1054A000040018D10598361A3F18CCE7049A002A50
:1054B00004D0691C0398F9F72FFE0446002C0AD18A
:1054C000132408E0152406E00020FF22613203A126
:1054D000F8F7D2FB1624204607B0F0BD2E5C736FA0
:1054E000757263655C6461706C696E6B5C6472613B
:1054F000672D6E2D64726F705C66696C655F737486
:105500007265616D2E6300007047000001000000AD
:10551000010000003863010040630100000000004A
:1055200000000000000000004C6301005063010017
:105530005863010048630100546301000100023612
:1055400000000000000000000000000074E9FF1FE0
:105550004D4943524F42495448544D4D4943524F8F
:1055600042495400000068747470733A2F2F6D69BB
:1055700063726F6269742E6F72672F6465766963F8
:10558000652F3F69643D404226763D40560000004D
:10559000000000000000000000000000000000000B
:1055A000000000000000290E0100000000000000C3
:1055B0000000000000000000010000002D020100BA
:1055C000453D01003D0F010051E80000C1E700002A
:1055D000891001001DE90000F53201000000000003
:1055E000BC55010000000000FFFFFFFFFFFFFFFFB1
:1055F000FFFFFFFFFFFFFFFF0000000000000000B3
:1056000000000000000000000000000374797065D5
:105610003A20006572726F723A20003C21646F6319
:10562000747970652068746D6C3E0D0A3C212D2DD7
:10563000206D62656420506C6174666F726D2057D6
:1056400065627369746520616E6420417574686574
:105650006E7469636174696F6E2053686F727463EE
:105660007574202D2D3E0D0A3C68746D6C3E0D0A3C
:105670003C686561643E0D0A3C6D65746120636839
:1056800061727365743D227574662D38223E0D0A71
:105690003C7469746C653E6D626564205765627325
:1056A0006974652053686F72746375743C2F7469F4
:1056B000746C653E0D0A3C2F686561643E0D0A3CC2
:1056C000626F64793E0D0A3C7363726970743E0DBB
:1056D0000A77696E646F772E6C6F636174696F6EA1
:1056E0002E7265706C6163652822405222293B0D41
:1056F0000A3C2F7363726970743E0D0A3C2F626F0F
:1057000064793E0D0A3C2F68746D6C3E0D0A0041B1
:10571000535345525420205458540000C05A01009D
:10572000000000004C64010001000000586401000A
:105730000200000040640100030000003464010026
:10574000040000002864010005000000EC63010073
:10575000060000001064010007000000E063010083
:10576000080000000464010009000000C863010093
:105770000A000000D46301000B000000F863010080
:105780000C0000001C6401000D00000064640100B6
:105790000E000000706401000F000000886401002A
:1057A000A4640100946401009C6401007C64010015
:1057B000EB3C904D53443053342E3100020801002D
:1057C000022000501FF8010001000100000000004D
:1057D00000000000000029741902274441504C4980
:1057E0004E4B2D444E444641543136202020FAB8C9
:1057F000C0070520018ED0BC0010B8C0078ED8BEEF
:105800006D00E80B00EBFEB40EB700B307CD10C37C
:105810008A044608C07405E8EDFFEBF4C3504C451C
:105820004153452052454D4F56452054484520414F
:10583000524D204D424544204441504C494E4B204E
:105840005553422044455649434520414E44205239
:1058500045424F4F54205448452053595354454DC9
:105860002E2E0000000000000000000000000000DC
:105870000000000000000000000000000000000028
:105880000000000000000000000000000000000018
:105890000000000000000000000000000000000008
:1058A00000000000000000000000000000000000F8
:1058B00000000000000000000000000000000000E8
:1058C00000000000000000000000000000000000D8
:1058D00000000000000000000000000000000000C8
:1058E00000000000000000000000000000000000B8
:1058F00000000000000000000000000000000000A8
:105900000000000000000000000000000000000097
:105910000000000000000000000000000000000087
:105920000000000000000000000000000000000077
:105930000000000000000000000000000000000067
:105940000000000000000000000000000000000057
:105950000000000000000000000000000000000047
:105960000000000000000000000000000000000037
:105970000000000000000000000000000000000027
:105980000000000000000000000000000000000017
:105990000000000000000000000000000000000007
:1059A000000000000000000000000000000055AAF8
:1059B00011160100095501000002000055130100F5
:1059C00009550100000000005513010009550100B0
:1059D00000000000D9120100E5520100000400009F
:1059E000000000000000000000000028000000008F
:1059F000000000000000418EBB32000000000000EB
:105A00000000000000000000000000010000000095
:105A1000764876480000DC837648000000000000ED
:105A20004C6C0100F06B0100D06B0100A86C010010
:105A300084680100986B01009C680100E86A01001D
:105A4000886A0100686C0100446B01000C6A010067
:105A5000486A0100D06C0100086C0100386901003F
:105A60000C690100E468010068690100246B010011
:105A70008C6C010018660100D86501009C6501006E
:105A8000986901001468010070670100386701001F
:105A900060660100486801003C6501007065010016
:105AA00010650100B0640100E0640100D0670100EE
:105AB000B0660100EC660100246D0100AC670100D6
:105AC00053544152545F424C41435400B534010099
:105AD0000D37010021350100BD33010015330100F0
:105AE000893601002D34010005330100B53601006F
:105AF000CC5A01000000000000000101010030311B
:105B00003233343536373839616263646566000094
:105B100000BE0AE00D782D0668400824400000D33E
:105B20005840641EFAD1491C521E002AF2D1704717
:105B3000002070470020704770B5264C022060603E
:105B40000120E060244D2868C00702D0002060607A
:105B500070BD00F02CF8F6E770B51E4C02216160B4
:105B60001E49884202D30120606100E0A0601A4D06
:105B700000F01DF82868C007FAD00020606070BDF2
:105B8000F8B505468E081348012114464160124FAE
:105B900001CC01C53868C00706D0761EF8D10D4883
:105BA000002141600846F8BD00F001F8F2E70C481A
:105BB00040680006000E0BD00A494968002907D04A
:105BC00009490A4AC30700D00A60091D4008F9D1F3
:105BD0007047000000E5014000E4014000100010A3
:105BE0000004014000050140000601403546526EA8
:105BF0000000000000BE0AE00D782D066840082471
:105C0000400000D35840641EFAD1491C521E002A9D
:105C1000F2D17047002070470020704770B52B4CC0
:105C2000022020602949012008310860284D286899
:105C3000C00702D00020206070BD00F033F8F6E706
:105C400070B5224C02212160B0F1102F03D31F49FF
:105C50000120103101E01D49091D08601C4D00F0B4
:105C600021F82868C007FAD00020206070BD2DE917
:105C7000F041DFF858808E08012114460546C8F827
:105C80000010134F01CC01C53868C00707D0761E3D
:105C9000F8D10021C8F800100846BDE8F08100F0F6
:105CA00001F8F1E70B48006810F0FF000CD00A493A
:105CB0000968002908D00849084AFC31C30700D008
:105CC0000A60091D4008F9D17047000004E5014051
:105CD00000E4014004040140040501403546526ED1
:105CE000000000000000000000040000210000206F
:105CF000250000202900002049000020710000201C
:105D000000000000010000207001002000100020B1
:105D1000000200200000002050010000105B010084
:105D20000002000000000000000000000010000061
:105D30002100002025000020290000204D00002027
:105D40007B00002000000000010000207001002006
:105D50000010002000020020000000205001000080
:105D6000F45B0100000200000000000002360200A7
:105D7000040000000000000000000000000000001F
:105D80000000000000000000312C010000000000B5
:105D900000000000000000000800100018002000B3
:105DA0003000400060008000C0000001800100025F
:105DB000000300040006000080841E0000127A0028
:105DC00000B003401B003C1000F005401F003810DD
:105DD0000809000006003410070034100060064077
:105DE000007006401400160018001A001C001E0067
:105DF000220028001C002000240028002C00300075
:105E0000380044003000380040004800500058007E
:105E10006800800050006000700080009000A000CA
:105E2000C000F000A000C000E0000001200140011F
:105E30008001E00140018001C001000240028002B7
:105E40000003C003800200038003000480040005F7
:105E50000006800700050006000700080009000A88
:105E6000000C000F00000140010101004000400053
:105E700040000101400040000202400000024000DA
:105E8000040440004000400040002120050540007F
:105E90000002400001DA00000000000000000000E5
:105EA0001DDA000000000000A1B90000F1C00000F0
:105EB00041C8000013B60000F9B50000B5B30000FA
:105EC00000000000000000000000000000000000D2
:105ED00000000000000000000000000000000000C2
:105EE0000000000000000000C3B800000000000037
:105EF000000000000600FF0901A101150026FF00B7
:105F000075089540090181029540090191029501AA
:105F10000901B102C000210012011002EF0201408C
:105F2000280D04020010010203010000050F3900D2
:105F3000021810050038B60834A909A0478BFDA047
:105F4000768815B665000121001C100500DF60DDB4
:105F5000D88945C74C9CD2659D9E648A9F000003EA
:105F6000064A01200000040309040803410052000E
:105F70004D003403220042004200430020006D0027
:105F80006900630072006F003A00620069007400EB
:105F9000200043004D005300490053002D004400F1
:105FA0004100500022001A03300030003000310060
:105FB0004100300030003000300030003000300050
:105FC00022036D006200650064002000530065003C
:105FD0007200690061006C00200050006F007200C8
:105FE000740022036D00620065006400200053000D
:105FF00065007200690061006C00200050006F00B5
:10600000720074001A0343004D005300490053000E
:106010002D00440041005000200076003100240390
:106020005700650062005500530042003A0020000E
:1060300043004D005300490053002D00440041002F
:10604000500010035500530042005F004D00530004
:1060500043001A0343004D005300490053002D0034
:10606000440041005000200076003200080B00027E
:1060700002020104090400000102020104052400D7
:106080001001052401030204240206052406000071
:106090000705830310002009040000020A00000520
:1060A00007050402400000070584024000000400C8
:1060B00088000401FF5207000100000010270000C3
:1060C00000000000CC000000980000000400000068
:1060D00001000100000000000000000000000000BE
:1060E00000000000000000000000000000000000B0
:1060F000000000000000000000000000020002009C
:10610000010000000000000000000000000000008E
:10611000000000000000000000000000000000007F
:106120000000000000000000030002000400000066
:10613000000000000000000000000000000000005F
:10614000000000000000000000000000000000004F
:10615000000000000000000000000000000000003F
:10616000000000000000000000000000000000002F
:10617000000000000000000000000000000000001F
:10618000000000000000000000000000000000000F
:1061900000000000000000000000000000000000FF
:1061A00000000000000000000000000000000000EF
:1061B00000000000000000000000000000000000DF
:1061C00000000000000000000000000000000000CF
:1061D00000000000000000000000000000000000BF
:1061E00000000000000000000000000000000000AF
:1061F000000000000000000000000000000000009F
:10620000000000000000000000000000000000008E
:10621000000000000000000000000000000000007E
:10622000000000000000000000000000000000006E
:10623000000000000000000000000000000000005E
:10624000000000000000000000000000000000004E
:10625000000000000000000000000000000000003E
:10626000000000000000000000000000000000002E
:10627000000000000000000000000000000000001E
:10628000000000000000000000000000000000000E
:1062900000000000000000000000000000000000FE
:1062A00000000000000000000000000000000000EE
:1062B00000000000000000000000000000000000DE
:1062C00000000000000000000000000000000000CE
:1062D00000000000000000000000000000000000BE
:1062E00000000000000000000000000000000000AE
:1062F000000000000000000000000000000000009E
:10630000000000000000000000000000000000008D
:10631000000000000000000000000000000000007D
:10632000000000000000000000000000000000006D
:106330000000000000000000393930330000000088
:10634000393930340000000048544D0042494E00B5
:106350005458540057415600435356004120626F31
:106360006F746C6F61646572207570646174652010
:106370007761732073746172746564206275742030
:10638000756E61626C6520746F20636F6D706C65F3
:1063900074652E0D0A52656C6F6164207468652007
:1063A000626F6F746C6F6164657220746F206669D0
:1063B000782074686973206572726F72206D6573DE
:1063C000736167652E0D0A004D53445F4F4E2020C8
:1063D000434647004D53445F4F46462043464700DF
:1063E0004F56464C5F4F4E20434647004155544F51
:1063F0005F4F4E2043464700434F4D505F4F4E2066
:10640000434647004F56464C5F4F4646434647007B
:106410004155544F5F4F464643464700434F4D500A
:106420005F4F464643464700484152445F525354EB
:10643000434647004155544F5F525354434647002B
:106440004552415345202020414354004153534578
:10645000525420204143540052454652455348204F
:1064600041435400504147455F4F4E204143540043
:10647000504147455F4F464641435400696E74653D
:106480007266616365000000696E7465726E616CAE
:10649000000000007573657200000000746172678F
:1064A000657400007472616E7369656E740000003B
:1064B000496E206170706C69636174696F6E2070E1
:1064C000726F6772616D6D696E6720736563746F5B
:1064D00072206572617365206661696C65642E0067
:1064E000496E206170706C69636174696F6E2070B1
:1064F000726F6772616D6D696E67206D6173732075
:106500006572617365206661696C65642E000000C8
:10651000496E206170706C69636174696F6E207080
:10652000726F6772616D6D696E67207772697465ED
:10653000206661696C65642E00000000496E206170
:1065400070706C69636174696F6E2070726F6772CE
:10655000616D6D696E6720696E697469616C697AD5
:106560006174696F6E206661696C65642E0000005D
:10657000496E206170706C69636174696F6E207020
:10658000726F6772616D6D696E6720756E696E6995
:1065900074206661696C65642E0000005468652093
:1065A0006865782066696C652063616E6E6F742023
:1065B00062652070726F6772616D6D65642E204C2C
:1065C0006F676963206661696C757265206F6363CC
:1065D00075727265642E00005468652068657820C5
:1065E00066696C652063616E6E6F742062652064FD
:1065F00065636F6465642E20506172736572206CF0
:106600006F676963206661696C757265206F63638B
:1066100075727265642E0000546865206865782084
:1066200066696C652063616E6E6F742062652064BC
:1066300065636F6465642E20436865636B73756D75
:106640002063616C63756C6174696F6E206661694B
:106650006C757265206F636375727265642E0000DD
:10666000546865206170706C69636174696F6E2035
:1066700066696C6520666F726D6174206973207540
:106680006E6B6E6F776E20616E642063616E6E6FED
:10669000742062652070617273656420616E642F7E
:1066A0006F722070726F6365737365642E000000F3
:1066B000496E206170706C69636174696F6E2070DF
:1066C000726F6772616D6D696E67206E6F74207393
:1066D0007570706F72746564206F6E207468697372
:1066E000206465766963652E00000000496E2061B4
:1066F00070706C69636174696F6E2070726F67721D
:10670000616D6D696E67206661696C6564206265A4
:106710006361757365207468652075706461746564
:106720002073656E742077617320696E636F6D707E
:106730006C6574652E000000546865207374617286
:1067400074696E67206164647265737320666F722A
:106750002074686520696E74657266616365207572
:1067600070646174652069732077726F6E672E00A4
:10677000546865207374617274696E672061646423
:106780007265737320666F722074686520626F6F24
:10679000746C6F61646572207570646174652069E2
:1067A000732077726F6E672E0000000054686520BA
:1067B000626F6F746C6F6164657220435243206432
:1067C0006964206E6F7420706173732E0000000086
:1067D000496E206170706C69636174696F6E2070BE
:1067E000726F6772616D6D696E672061626F72743E
:1067F00065642064756520746F20616E206F757408
:10680000206F6620626F756E6473206164647265C8
:1068100073732E00546865206865782066696C651E
:10682000206F6666736574206C6F616420616464B8
:1068300072657373206973206E6F7420636F727258
:106840006563742E00000000546865206170706CF0
:1068500069636174696F6E20696D61676520697332
:10686000206E6F7420636F6D70617469626C652057
:106870007769746820746865207461726765742E26
:1068800000000000546865207472616E7366657262
:106890002074696D6564206F75742E0046696C659F
:1068A0002073656E74206F7574206F66206F72643C
:1068B00065722062792050432E205461726765749E
:1068C000206D69676874206E6F7420626520707235
:1068D0006F6772616D6D656420636F72726563745A
:1068E0006C792E00466C61736820616C676F726909
:1068F00074686D20777269746520636F6D6D616E69
:1069000064204641494C555245000000466C617375
:106910006820616C676F726974686D20657261735D
:106920006520616C6C20636F6D6D616E6420464103
:10693000494C555245000000466C61736820616CFB
:10694000676F726974686D20657261736520736525
:1069500063746F7220636F6D6D616E642046414990
:106960004C55524500000000466C61736820616C14
:10697000676F726974686D207772697465207665D7
:106980007269667920636F6D6D616E64204641495E
:106990004C55524500000000546865206865782019
:1069A00066696C6520796F752064726F70706564BC
:1069B0002069736E277420636F6D70617469626CF7
:1069C0006520776974682074686973206D6F6465E9
:1069D000206F72206465766963652E2041726520A0
:1069E000796F7520696E204D41494E54454E414E98
:1069F0004345206D6F64653F205365652048454CD5
:106A000050204641512E48544D00000054686520E6
:106A1000696E74657266616365206669726D77611F
:106A20007265204641494C454420746F20696E6967
:106A30007469616C697A6520746865207461726735
:106A40006574204D4355000054686520696E746577
:106A50007266616365206669726D77617265204652
:106A600041494C454420746F20756E696E697469A4
:106A7000616C697A652074686520746172676574F9
:106A8000204D43550000000054686520696E746510
:106A90007266616365206669726D77617265204612
:106AA00041494C454420746F20646F776E6C6F6170
:106AB000642074686520666C6173682070726F670B
:106AC00072616D6D696E6720616C676F7269746861
:106AD0006D7320746F2074686520746172676574CB
:106AE000204D43550000000054686520696E7465B0
:106AF0007266616365206669726D776172652046B2
:106B000041494C454420746F2072657365742F6849
:106B1000616C742074686520746172676574204DBF
:106B200043550000456E64206F6620737472656182
:106B30006D20686173206265656E207265616368AF
:106B40006564000054686520696E746572666163EF
:106B500065206669726D77617265204641494C45D2
:106B60004420746F20646F776E6C6F61642074686A
:106B70006520666C617368206461746120636F6E68
:106B800074656E747320746F2062652070726F6715
:106B900072616D6D65640000506F737369626C653E
:106BA000206D69736D6174636820626574776565D3
:106BB0006E2066696C652073697A6520616E642059
:106BC00073697A652070726F6772616D6D656400BC
:106BD000416E20696E7465726E616C206572726FB1
:106BE0007220686173206F63637572726564000060
:106BF000416E206572726F7220686173206F6363EB
:106C0000757272656400000054686520696E746571
:106C10007266616365206669726D77617265204690
:106C200041494C454420746F20756E6C6F636B2036
:106C30007468652074617267657420666F72207075
:106C4000726F6772616D6D696E6700004F7065727B
:106C50006174696F6E207761732073756363657308
:106C60007366756C0000000054686520666C617383
:106C70006820616C676F206D697373696E67206649
:106C80006F72206120726567696F6E00456E6420C7
:106C90006F662073747265616D20697320756E6B09
:106CA0006E6F776E00000000416E206572726F7229
:106CB000206F6363757272656420647572696E67B4
:106CC00020746865207472616E73666572000000DE
:106CD00054686520696E74657266616365206669D3
:106CE000726D776172652041424F52544544207065
:106CF000726F6772616D6D696E672E20496D616795
:106D00006520697320747279696E6720746F2073CF
:106D10006574207365637572697479206269747330
:106D200000000000000000004D42454420202020CB
:106D300056465320202020202020202020202020C4
:106D4000302E3100646D010000E0FF1F00100000D4
:106D500024880000F073010000F0FF1FD03B00000A
:106D600004810000011C120112FFB6FFC8010108D6
:106D700023E0071A740421250220B5021ADD041A43
:106D8000DF041AE1041AE3041AE50401101AE714F7
:106D90005AE9181AEB081AED040A75EF0481092A5A
:106DA0002CA934A90801FC101110B5054C23783327
:106DB000B9044B13B10448AFF320098001232370B9
:106DC00010BD744220236007380A08B5034B1BB17D
:106DD000034903204308BD1A7820291C13154B10C2
:106DE0000C2B08BF134B9D46A3F5803A100C218B4A
:106DF000460F461348144A121A1DF047FA0F1E1187
:106E00005DD098470E081954132104120D130D4834
:106E10003D2802D00C501115F00FFA20222914F051
:106E2000EDF914F0F5F91ABF72313A028041298C5C
:106E30005A90904110130649074A074B9B1A03DDED
:106E4000043BC858D050FBDC2008F02FF8FFF7B9FE
:106E5000FF1A6C94312A20340B10FEE7022813BF6E
:106E6000F34F8F0549064BCA6802F4E0621343CB27
:106E70006012111CBFFDE77812ED13E0041011FA47
:106E800005034B1868A0F10D035842584170471490
:106E9000BF3001100E1008B5FFF7F3FF40B14FF0FF
:106EA0008043180922C3F80C21C3F81004173825B1
:106EB000FFF7E7FF1C2846D01A180F52594BD2F89B
:106EC0000414C3F82015D2F808081A24081A0C086C
:106ED0001A28081A10081A2C081A14081A30081A46
:106EE00018081A34081A1C081A40081A20081A44EC
:106EF000081A24081A48081A28081A4C081A2C08D4
:106F00001A50081A30081A54081A34081A60081A55
:106F100038081A64081A3C081A68081A40081A6CDB
:106F2000081E4424C3F870963C9CFF48AE13D3F867
:106F3000180B24D10744BF6FF00102C30C180C31A9
:106F40004AD2F8883043F47003C20829FE1814BFEF
:106F5000F36F8F4FF01023D3F80C22D2071ED529E0
:106F60004B01E22B04253A111B2AFBDA1B1022C825
:106F70001D3223F001341F0C32214B1A461C12140F
:106F80001429FBD01A212A197611123418082BFB68
:106F9000D0FFF74FFF1A122210082A03DBD3F804A0
:106FA000320D112B23DA164E151221C2F89A121245
:106FB0002B2312240B17220B5A100BD1E7054B057C
:106FC0004A1A6008BD12BF12C0124012ED12E0341E
:106FD000E001401220100890D0031F2886BF13F054
:106FE0001F100B044A4FF0A042012303FA1808F0C7
:106FF000C2F808057047301203100C50805CC1F1D4
:1070000004010841C04313F00119162A23281383F1
:10701000421DDB7047D268180E0133F8E738B51C03
:1070200020FFF7DAFF0B061CD7FF1F061CD4FF2535
:10703000061808D1FF0B4C0B4D1E0A13CCFF18107D
:10704000220120135D1F2B86BF03F01F0329464634
:10705000144101323010FA03F3052AC1F80C35F05F
:10706000D138BD54071974100B2DE9F84F80463BF9
:10707000483B4DC8082282460324135C381812038B
:10708000F5E0730132052A41F82340F0D13348314D
:1070900028091E26100BFFF7ACFF4FF00109284C02
:1070A00014263227180925254B585DFFF780141147
:1070B00068120B2A46594620461AF80B30FFF7870C
:1070C000FFA0BB482B1B4AEC1A09A41AC2A2184302
:1070D0000BF1010BBBF1050FE7D144F62060013540
:1070E000FFF779FFFFF781FF052DD8D1013FD5D1FB
:1070F00013480136FFF76FFF042ECCD031466423CE
:107100000A2202E0013993FBF2F30129FAD198FB3C
:10711000F3F30C1018F402FB1434094B04EB840451
:107120001C44BAE71846FFF73EFFD1E75BBF4AFCB5
:107130001A54081A4F041440420F1A1808100B086A
:10714000B5034B9888FFF775FF142008BD23BF04D3
:10715000100A2008B5074B044613B11421AFF310F1
:107160000E80054B1868836A03B19847204614F0D7
:1071700031F842BF1A5C3C100B70B50D4E0D4CA49B
:107180001BA410100A25A54209D10B4E0C4C6CF023
:1071900022F812680F05D170BD56F82530984701C6
:1071A00035EEE70A1CF2E76C6469041A70041702F2
:1071B0004403469342180BD1704703F8011BF9E7CB
:1071C000FEB01BF8B504A808BC08BC9E4670470C6E
:1071D000182E0C9252524C048C84848E1C824C903B
:1071E0001E1EC244924C06CA525FE21FF01EC13EF0
:1071F00002448ED12E1FE24488100ED12ED12E05CE
:10720000100AC4881C0B1F251E1B1B30080E1115ED
:10721000160F18131A0C744146DCFAFF7F0100099F
:107220006390D003DEC0CEFA462325021A0104186B
:107230000A646C766B4441544120011442494E1A51
:10724000F889E303991B9FE730130801144D52019D
:107250002311E31AB1101A2D10143554011A191004
:10726000018D380801010206020208013A04063FB6
:10727000010106060604017A10010D230B99969769
:107280004E021201022B0414E45C0189437A040CBF
:107290001AEC1801B712201A400401C552015C28EB
:1072A0005D010A417A080C1A301801B71A20DC195E
:1072B0000401C40212010C146CDC02F61508280249
:1072C000D28012BF401CFAE7BFF34F8F30BFBFF32D
:1072D0006F8F70471206126B520A1603064A010896
:1072E000294512A012141203A757494E55534212B2
:1072F0008412041207122A12441265127612691AB5
:1073000063081249126E1A7408127212663A6112F8
:1073100012471A5516124432731250127B12391248
:10732000321243124512361A340412321A2D121236
:10733000431A37023A2D121A461C29141A33021A1C
:10734000420A12331A31203A422612351A410229D2
:10735000181239527D0950A01A430C3A4264296E22
:107360001A44823A328E298C29A01A360C5A2D885A
:107370001A360A3A310C3A451C29043A33CC5A36AB
:10738000A02114286D0140292C03016F732E6D621A
:1073900065642E636F6D2F7765627573622F6C6104
:1073A0006E64696E672D706167652F3F6269643D29
:1073B000CA132C01251A5501013814D060011AFC9A
:1073C00004142861011A54041A80041AAC041AD84F
:1073D00004140462011A3004146C5D011A5C081A6A
:1073E00088041AB4041AE00404D10C6301000000FC
:1073F000FFFFFFFFFFFFFFFFFFFFFFFFFFFFFFFF9D
:10740000FFFFFFFFFFFFFFFFFFFFFFFFFFFFFFFF8C
:10741000FFFFFFFFFFFFFFFFFFFFFFFFFFFFFFFF7C
:10742000FFFFFFFFFFFFFFFFFFFFFFFFFFFFFFFF6C
:10FBF000FFFFFFFFFFFFFFFFFFFFFFFFF5C05C5BA5
:00000001FF
